:100000000C945D4C0C94F74C0C94F74C0C94F74CFE
:100010000C94F74C0C94F74C0C94F74C0C94F74C54
:100020000C94F74C0C94F74C0C94F74C0C94F74C44
:100030000C94F74C0C94B44D0C94F74C0C94F74C76
:100040000C94F74C0C94F74C0C94F74C0C94F74C24
:100050000C94F74C0C94F74C0C94F74C0C94F74C14
:100060000C94F74C0C94F74C0C94F74C0C94F74C04
:100070005A5501200101003808000000000000006E
:100080000000000000000000000000000000000070
:100090009556A3567E57675B515BA656B556C45618
:1000A000385BD256E05600020800085504085A0092
:1000B00000F8000990000A1E32050000FF00000051
:1000C000A60000000000000000000000000000008A
:1000D0000000000000000000000000000000000020
:1000E0000000000000000000000000000000000010
:1000F0000000000000000000000000000000000000
:1001000000000000000000000000000000000000EF
:1001100000000000000000000049000000495252A9
:10012000000052525C2D00000000000000000000A2
:100130000000000000000040000000494A52004951
:1001400052525B1C52531C25241B2425251B0A0AD2
:100150002D1C12120A0A0000000000000000404995
:1001600049494949525B5B5B525B1C1C1312241CBE
:100170001209090912090909090A0A0A0A0A0A13CD
:10018000120A0A12130A0000000000009252525292
:10019000525213121309001C0A1212401B65090A5D
:1001A0000009241B120000251C1C010025241C1C16
:1001B0000024252424240000000000005249494066
:1001C00000001B1352494900641C1C5B4A481C6513
:1001D0001C2552491C1C652464491C1C6525644966
:1001E0001C1C6D2E5C490000000000000000000097
:1001F0000049000000005352000000535225000047
:100200004A52252500005B251300005B53000A1CA1
:10021000095B1C657F374052522E2E1C525C2E25E6
:100220001B1324251C1C12002525120000121B0084
:1002300000132E37001B37372E2E37372E2E2E2E3B
:100240002E2E6E6E6E1C1313120009131200001274
:1002500013130012251C13132E371C131313361CF3
:10026000131B1B1B25131C1C1B1B1B1C1C1C1C1CDD
:100270001C1C1C1C1C131312121313001313131C2D
:10028000000913131C010037131C13002E2E1C1C15
:10029000001C772E2500137F251C010A37241C1C07
:1002A0000A2E25250900132E242525252E25252552
:1002B000252525252D2E251B2E2E251C1325251CF9
:1002C0001C1C1C011C1C1300011C0A000165775C2E
:1002D000016E7F6E521B25256D1C524925251C136E
:1002E00053001C1C1C524A001B135B5B000009528C
:1002F0005C0000005B5C000000001B0000000000D0
:10030000000000000000135B7F776E6E1365777648
:100310006E6E1B65777676761B5BBF76B6760913B5
:100320006DBFB7B6001B125C76BF0000121B125BDC
:1003300000000000090A6E6E6E77241C6E6E772531
:100340001C1C6E776E1C1C1C76761C1C2425B76545
:10035000646D6D1B766D6D5B09125B5C5B125B649B
:100360001213131B12121C1C1C1C1C241C1C2425E5
:1003700025242425251B00002513000064BF000947
:100380006EBFBF6D6EBF6D5B12135B12131209005F
:100390000901000000002E1C0900096E0100097609
:1003A0007F7F12777F7F6412BF775B121B095B121E
:1003B0001B0900001B0900000000000000000000F5
:1003C0000000000000007F7F5313130064121B0124
:1003D00000001B12000000000000000000000000F0
:1003E000000000000000000000000000000000000D
:1003F00000000000000000000000000026000000D7
:1004000026002F0000002F00370000003700FF00FB
:100410000000FF00BF000000BF00370000370000F1
:1004200000262600000000000000000026262626E8
:100430002600000000002F00000000370000000030
:10044000FF00000000BF00000000370000000000B7
:100450002626262626000000000000002626262646
:1004600026002F0000000000370000000000FFFF02
:10047000FFFF0000BF000000000037000000000088
:100480002626262626000000000000002626262616
:1004900000002F0000002F00370000003700FFFF92
:1004A000FFFF0000BF000000BF0037000000370062
:1004B0002626262600000000000000000000262658
:1004C0002600002F00002F00370000003700FF003B
:1004D0000000FF00BF000000BF0037000037000031
:1004E0002626260000000000000000002600000074
:1004F00026002F0000002F0000370037000000000A
:10050000FF00000000BF00BF000037000000370000
:10051000260000002600000000000000000000008F
:1005200000000000000000000000000000000000CB
:100530000000000000000000009B000000529BA48F
:1005400000005B9B6D7700000000000000000000D1
:10055000000000000000005B000000E4F6FF099BC3
:10056000EDF6FFBFA4ADBFBFBFBF767F7FB7B7BFFC
:100570007F766EB7B7BF00000000000000005BB6DA
:10058000F6F6F6FFFFFFFFBFFFFFFFBFBFAEFFFFA7
:10059000FFB7AD65FFFFB7B6AD65FFFFBFB7AE6E86
:1005A000FFFFBFB7B765000000000000F6F6EDEDF5
:1005B000ADA4B66D6D5C526E6565655265765C5C2A
:1005C00052536E246552526E25255B52772D252598
:1005D000526E6E2D2525000000000000A49B9B4953
:1005E00000006564A49B92006D2525649349656EA7
:1005F000652E9B5224256D25655225246D2D65524F
:1006000025256E2E6452000000000000000000004E
:10061000004A000000005B9B0000005B5B2D0000B7
:10062000525B2E2E00015B2D1C01005C5B014A65B4
:100630004A5B1C6E7F77495B9B77776D5B65776E56
:1006400065656D2D25255C522E25130949641C090D
:10065000095C7F7F091C7F7F777F777F77777F7F3C
:100660007776777F7F6E656E6EA4B6FF655BA4B705
:10067000BFFF526DBFBFBFFF7FBFBFBFBFFFBFBFC9
:10068000B7BFFFFF7FB7BFBFFFFF6EB7BFBFFFFFA3
:1006900077BFBFBFFFFFFFFFBFBFB75BFFFFBFBF9E
:1006A000A464FFFFBFADA47FFFFFBFA4BF7FFFBF58
:1006B000ADBFBFBFFFB6BFBFBF77F7BFBFBF7777C5
:1006C000FFBFBFBF64526D7F6E2E2D2D7F766E6E85
:1006D0006E2E777777762E1C7F776E251C257765B3
:1006E00025251C096E6E1C0949255B494A6E7F64ED
:1006F0005377BF775B5C256E6E255B4A25651C1BB7
:100700005B002524245B53001C1B5B5C00000A5B20
:10071000640000006464000000005C000000000051
:100720000000000000005B5C7FBF77765C6D7FB7E8
:1007300077775C6D7FBF77775C64BFBFBFBF0A5CB4
:100740006EBFBFBF0065646DBFBF00005B6D646DB1
:1007500000000000125B7777777F6E6E77777F7689
:100760006D7677BF776D6E76BF7F6D6E767FBF7665
:1007700076BFBF76BFBFBFB664ADADB6B6ADBFFF87
:10078000646DADB6AD6477BFBFBFFFFF77BFBFBFBE
:10079000FFFF7FBFBFBFFFF6BFB7ADF6FFFFA4AD42
:1007A000FFFFFFFFFFFFFFFFFFFFFFFFFFF6A400BC
:1007B0005B5200000000BFBFAD5B64BFB6ADADBF14
:1007C000FFBFFFFFFFFFBF64FFFFBFB6765BFFBF4A
:1007D000BF5B0000FF5C00000000000000000000A4
:1007E000000000000000BFBF645C5C006E5C6549F7
:1007F00000006D5B00000000000000000000000031
:1008000000000000000000000000000000000000E8
:1008100000000000000006000400000001000200CB
:1008200003000400050006000700080009000A0094
:100830000B000C000D000E000F0010000000110056
:10084000120013001400150016000600030000003B
:100850001700180019001A001B001C001D001E00C4
:100860001F00200021002200230024002500260074
:10087000000000B0073F005C00000B7F00C00000DC
:10088000902B4000B2073F005C00000B7F00C200CD
:10089000009235407A902B40009237401E902940BC
:1008A0000092304010902B40009232400F9029402F
:1008B000009230400F902B4000923240109029401F
:1008C000009230400F902B40009232400F90294010
:1008D000009230400F902B400092324010902940FF
:1008E000009230400F902B40009232400F902B40EE
:1008F000009232401090304000923C400F903040C7
:1009000000923C400F90324000923E4010FF0601A2
:100910005300902B40009237402D90304000923C85
:10092000401F903040009240400F90304000923C79
:10093000401090324000923E400F902B4000923782
:10094000402E90304000923C401E9030400092403B
:10095000401090304000923C400F90324000923E58
:10096000400F902940009230401090304000923764
:10097000400F902940009230400F90304000923755
:10098000400F902940009230401090304000923744
:10099000400F902940009230400F90304000923735
:1009A0004010902B40009232400F9032400092391C
:1009B000400F902B40009232400F9032400092390D
:1009C0004010902B40009232400F903240009239FC
:1009D000400F902B400092324010903240009239EC
:1009E000400F902B40009237402E90304000923CB8
:1009F000401E903040009240401090304000923CA9
:100A0000400F90324000923E400F902B40009237B2
:100A1000402E90304000923C401F90304000924069
:100A2000400F90304000923C400F90324000923E88
:100A30004010902B40009237402D90304000923C67
:100A4000401F903040009240400F90304000923C58
:100A5000401090324000923E400F902B4000923761
:100A6000402E90304000923C401E9030400092401A
:100A7000401090304000923C400F90324000923E37
:100A8000400F902940009230401090304000923743
:100A9000400F902940009230400F90304000923734
:100AA000400F902940009230401090304000923723
:100AB000400F902940009230400F90304000923714
:100AC0004010902940009230400F90304000923703
:100AD000400F9029400092304010903040009237F3
:100AE000400F902940009230400F903040009237E4
:100AF000400F90294000922E4010902A4000922FE3
:100B0000400F902B40009237402E90304000923C96
:100B1000401E903040009240401090304000923C87
:100B2000400F90324000923E400F902B4000923791
:100B3000402E90304000923C401F90304000924048
:100B4000400F90304000923C400F90324000923E67
:100B50004010902940009230400F90304000923772
:100B6000400F902940009230401090304000923762
:100B7000400F902940009230400F90304000923753
:100B8000400F902940009230401090304000923742
:100B9000400F902B40009232400F9032400092392B
:100BA0004010902B40009232400F9032400092391A
:100BB000400F902B40009232400F9032400092390B
:100BC0004010902B40009232400F903240009239FA
:100BD000400F902B40009237402E90304000923CC6
:100BE000401F903040009240400F90304000923CB7
:100BF000400F90324000923E4010902B40009237C0
:100C0000402E90304000923C401E90304000924078
:100C1000400F90304000923C401090324000923E95
:100C2000400F902B40009237402E90304000923C75
:100C3000401F903040009240400F90304000923C66
:100C4000400F90324000923E400F902B4000923770
:100C5000402E90304000923C401F90304000924027
:100C6000400F90304000923C400F90324000923E46
:100C70004010902940009230400F90304000923751
:100C8000400F902940009230401090304000923741
:100C9000400F902940009230400F90304000923732
:100CA0004010902940009230400F90304000923721
:100CB000400F902940009230400F90304000923712
:100CC0004010902940009230400F90304000923701
:100CD000400F9029400092304010903040009237F1
:100CE000400F90294000922E400F902A4000922FF2
:100CF000400F902B4000922B4010903040009237D4
:100D0000406BFF06014500FF2F000002060000FFB8
:100D100000FF00020800085504085A0000F8000906
:100D200090000A1E32050000FF00020800083C0087
:100D3000009C00FF0002060008390000CE00FF0002
:100D4000020300084608085208085E0000F800FF89
:100D500000020600083E0808320000F000FF000014
:100D6000000A0D00000000000000120D000000004D
:100D7000000000290D00000000000000340D0000FC
:100D800000000000003F0D00000000000000500DBA
:100D9000000000004E414D452054484520534D4130
:100DA000525445535420414E494D414C3B444F47CA
:100DB0001D3B4D4F4E4B4559153B444F4C504849F8
:100DC0004E103B4341540E3B464F58053B484F5253
:100DD0005345043B504152524F5403000000000061
:100DE0000000000000000000000000004E414D45E2
:100DF0002041205245434F524420434F4D50414ED5
:100E0000593B5243413C3B4D4F544F574E0B3B4394
:100E1000415049544F4C0A3B434F4C554D42494178
:100E2000043B4445434341043B412026204D033BC2
:100E30004150504C4503000000000000000000003D
:100E4000000000004E414D4520534F4D4554484948
:100E50004E472054484154204D454C545320454161
:100E600053494C593B425554544552243B49434500
:100E700020435245414D1D3B4943450E3B434845A8
:100E8000455345083B43484F434F4C415445083B6D
:100E9000534E4F57033B5741580200005245414CB7
:100EA000204F462046494354494F4E414C2C204E3A
:100EB000414D45204120435245415455524520570C
:100EC0004849434820484154455320434154533BEB
:100ED000444F4753383B4D494345153B42495244E3
:100EE00053093B414C46083B48554D414E53040085
:100EF000000000004E414D452041204352554E43D5
:100F0000485920464F4F443B4348495053293B439F
:100F1000454C4552590F3B434152524F54530B3BA2
:100F200043455245414C0A3B504F50434F524E05AA
:100F30003B4150504C4553043B4E555453033B43A7
:100F40005241434B45525302000000004E414D4573
:100F5000204120464F4F4420594F55205041434B8C
:100F600020464F52205448452042454143483B5378
:100F7000414E44574943484553293B434849505300
:100F8000193B434849434B454E0F3B484F5420447F
:100F90004F47530A3B465255495405000000000094
:100FA000000000004E414D45204120434152442065
:100FB00047414D4520504C41594544204259204B12
:100FC0004944533B474F2046495348293B4F4C44E3
:100FD000204D414944223B4352415A5920454947FB
:100FE000485453073B574152063B47494E20525500
:100FF0004D4D59043B554E4F030000004E414D45A9
:10100000204120504C4143452057484552452050EF
:10101000454F504C452022434845434B20494E22E2
:101020003B484F54454C483B484F53504954414C22
:10103000093B414952504F5254083B444F43544F8F
:10104000522753204F4646494345053B574F524B85
:10105000050000004E414D4520414E20414E494D76
:10106000414C205345454E20494E204D455849435B
:101070004F3B425552524F343B4C495A4152440D1A
:101080003B42554C4C073B444F47053B484F52535E
:1010900045043B41524D4144494C4C4F033B434175
:1010A00054023B434F570200000000004E414D45A3
:1010B00020534F4D455448494E47204120574F4DEE
:1010C000414E204B4545505320425920484552201F
:1010D0004245443B414C41524D1A3B5449535355B0
:1010E0004553163B424F4F4B133B54454C455048DC
:1010F0004F4E450E3B4C414D500300000000000098
:10110000000000004E414D4520534F4D4554484985
:101110004E4720594F55204C49434B3B49434520AE
:10112000435245414D263B43414E4459203B535485
:10113000414D5053143B454E56454C4F5045033B93
:101140004C495053033B46494E47455253023B538B
:10115000504F4F4E02000000000000004E414D4530
:101160002041204B494E44204F46204E45543B469B
:101170004953484E4554363B48414952204E455408
:10118000183B54454E4E4953204E4554083B564F4C
:101190004C4C455942414C4C204E4554043B424135
:1011A000534B455442414C4C204E455403000000E3
:1011B000000000004E414D4520534F4D45544849D5
:1011C0004E47205343484F4F4C53204255592041DE
:1011D000204C4F54204F463B424F4F4B53313B50D6
:1011E000415045521A3B4348414C4B083B50454EF9
:1011F00043494C4553073B4445534B53033B464FF0
:101200004F44030000000000000000004E414D4527
:1012100020534F4D455448494E472054484154208F
:101220005350494E532041524F554E443B544F501A
:101230004B3B544845204541525448053B4D45528F
:10124000525920474F20524F554E44043B57484572
:10125000454C033B46414E023B57494E444D494C99
:101260004C0200004E414D452041204B494E442048
:101270004F462054414E4B3B46495348223B474141
:10128000534F4C494E451B3B534845524D414E1020
:101290003B4F585947454E053B5741544552043B37
:1012A000534550544943033B544F494C4554033B29
:1012B0004F494C0300000000000000004E414D4526
:1012C00020534F4D455448494E47205448415420DF
:1012D000474554532053435255424245443B464CA4
:1012E0004F4F523C3B42415448545542093B504FAA
:1012F0005453083B4241434B063B46414345053B63
:10130000504F5441544F4553033B4B494402000056
:10131000000000004E414D452041205155494554A3
:1013200020414E494D414C3B434154243B4D4F5588
:1013300053450D3B5241424249540D3B44454552B1
:10134000073B47495241464645063B4649534805F7
:101350003B534E414B45043B48414D53544552038A
:101360000000000000000000000000004E414D455C
:1013700020534F4D455448494E472050454F504CFF
:101380004520534156453B4D4F4E4559393B434F00
:10139000494E53093B434F55504F4E53073B50481E
:1013A0004F544F475241504853073B5354414D50BF
:1013B00053073B414C554D494E554D2043414E53EB
:1013C000030000004E414D4520534F4D45544849C0
:1013D0004E4720594F5520425559204259205448D4
:1013E000452051554152543B4D494C4B443B4F498C
:1013F0004C0C3B49434520435245414D093B4D412F
:10140000594F4E4E41495345063B4A5549434502C3
:101410000000000000000000000000004E414D45AB
:1014200020534F4D455448494E4720594F5520456C
:1014300041542057495448205045414E555420426C
:1014400055545445523B4A454C4C593D3B425245FC
:1014500041440C3B435241434B455253093B4241AB
:101460004E414E4153073B43454C455259070000FE
:10147000000000004E414D4520534F4D4554484912
:101480004E4720494D504F525445442046524F4DEF
:10149000204745524D414E593B42454552303B4312
:1014A0004152531F3B434C4F434B53083B43484F20
:1014B000434F4C415445053B48554D4D454C204606
:1014C0004947555245530300000000004E414D4529
:1014D00020534F4D455448494E4720594F552042BF
:1014E00055592053414C5445443B4E5554534C3B65
:1014F000504F50434F524E083B505245545A454C62
:1015000053053B504F5441544F20434849505303D7
:101510003B504F524B020000000000000000000052
:10152000000000004E414D4520534F4D4554484961
:101530004E47204B4944532054414C4B2041424F8D
:1015400055543B5343484F4F4C163B47414D455331
:101550000D3B53504F5254530B3B54560A3B4D5581
:10156000534943083B504152454E54530800000034
:101570000000000000000000000000004E414D454A
:1015800020534F4D455448494E4720594F552057F9
:1015900049534820594F552048414420494E20592D
:1015A0004F5552204241434B594152443B504F4FBB
:1015B0004C523B484F5420545542033B464C4F57E6
:1015C000455253023B5357494E47023B54524545FF
:1015D000530200004E414D45204120225448494EBF
:1015E0004B494E47204D414E27532047414D452200
:1015F0003B43484553533F3B5452495649414C2085
:10160000505552535549540C3B4A454F5041524452
:1016100059063B425249444745043B5343524142D9
:10162000424C45043B5249534B0300004E414D454B
:1016300020534F4D455448494E472054484154206B
:101640004B49445320474554204452455353454445
:1016500020555020464F523B434855524348413B4A
:1016600048414C4C4F5745454E0D3B504152545903
:101670000A3B454153544552053B5049435455524A
:10168000450500004E414D45204120464F4F442026
:101690005448415420434F4D455320494E20494E14
:1016A0005354414E5420464F524D3B504F54415499
:1016B0004F45531F3B4F41544D45414C193B434F00
:1016C000464645450F3B50554444494E470A3B5317
:1016D0004F5550073B524943450500004E414D458B
:1016E00020534F4D455448494E47205448415420BB
:1016F0004445434159533B5445455448513B465258
:10170000554954053B4C4541564553043B574F4FB3
:1017100044043B424F4459023B4D454154020000B2
:1017200000000000000000000000000000000000B9
:10173000000000004E414D45204120464F4F4420BF
:10174000544841542753204841524420544F204B81
:10175000454550204F4E20594F555220464F524B31
:101760003B504541532D3B53504147484554544904
:10177000253B52494345073B534F5550033B434F8D
:10178000524E020000000000000000004E414D4596
:101790002041205350454349464943204C55585514
:1017A0005259204954454D205448415420594F55D1
:1017B000204F574E204D4F5245205448414E204F08
:1017C0004E45204F463B5456303B434152173B5603
:1017D00043520B3B52494E47093B57415443480340
:1017E000000000004E414D4520534F4D455448499F
:1017F0004E4720594F5520535445414D3B56454780
:10180000455441424C4553423B434C414D530B3BA5
:10181000434C4F54484553063B52494345053B53BF
:101820004852494D50040000000000000000000034
:101830000000000000000000000000004E414D4587
:1018400020534F4D455448494E472050454F504C2A
:10185000452046414C4C204F5554204F463B4C4F61
:101860005645293B424544263B54524545530D3B82
:10187000414952504C414E45023B48414D4D4F432A
:101880004B0200000000000000000000000000000B
:10189000000000004E414D4520534F4D45544849EE
:1018A0004E4720594F5520505554204F4E2041202F
:1018B000424142593B44494150455253513B4241B8
:1018C000425920504F57444552063B42414259200D
:1018D0004C4F54494F4E033B424942033B534F4305
:1018E0004B53020000000000000000004E414D4537
:1018F00020534F4D455448494E47205448415420A9
:101900004749564553204F464620484541543B538E
:10191000554E1E3B53544F56451D3B4649524513A9
:101920003B524144494154494F4E053B484541547F
:101930004552043B434152204D4F544F5203000047
:10194000000000004E414D45204120504C41434590
:1019500020574845524520594F5520534545204D65
:10196000414E592050454F504C4520524541444925
:101970004E473B4C494252415259523B41495250C9
:101980004C414E45043B5041524B033B5343484F5F
:101990004F4C033B545241494E0200004E414D45CD
:1019A00020534F4D455448494E47204153534F43D0
:1019B00049415445442057495448204120545552E8
:1019C000544C453B5348454C4C3C3B4245494E47A3
:1019D00020534C4F571A3B48415245053B534F55F6
:1019E00050033B57415445520200000000000000E4
:1019F000000000004E414D45204120464F4F4420FD
:101A000054484154275320474F4F44204F4E2041C4
:101A100020484F54204441593B49434520435245B7
:101A2000414D343B4D454C4F4E113B53414C41448D
:101A3000103B53414E44574943484553043B484F9C
:101A40005420444F47530300000000004E414D45D1
:101A5000204F4E45204F462054484520534D454C7D
:101A60004C53204F462053554D4D45523B464C4F0D
:101A700057455253203B4355542047524153531B23
:101A80003B4241524245435545133B5241494E0565
:101A90003B53554E54414E204C4F54494F4E03003A
:101AA000000000004E414D4520534F4D45544849DC
:101AB0004E47205448415420594F55205345543BDC
:101AC000434C4F434B393B48414952123B544142EE
:101AD0004C450E3B564352063B54494D455202007D
:101AE00000000000000000000000000000000000F6
:101AF00000000000000000000000000054454C4CB5
:101B0000204D4520534F4D455448494E4720434FA3
:101B10004C4F52454420424C55453B534B59443B56
:101B20004A45414E53093B45594553043B5741549F
:101B30004552043B53484952540300000000000042
:101B40000000000000000000000000000000000095
:101B5000000000004E414D4520534F4D455448492B
:101B60004E47205448415420414C5741595320413D
:101B70005454524143545320412043524F57443B05
:101B80004143434944454E54273B46495245193B3E
:101B90004649474854073B504152414445053B5351
:101BA000414C450200000000000000004E414D4540
:101BB0002041204B494E44204F4620454E47494E38
:101BC0004545523B454C454354524943414C243BC7
:101BD0005241494C524F4144193B434956494C0EDE
:101BE0003B4D454348414E4943414C073B434845E3
:101BF0004D4943414C063B4145524F5350414345AB
:101C0000030000004E414D4520534F4D4554484977
:101C10004E472050454F504C4520444F204F4E20BA
:101C200054484520464C4F4F523B45584552434936
:101C300053451F3B44414E43450C3B534954450AD1
:101C40003B57415443482054560A3B534C4545505A
:101C50000800000000000000000000004E414D455B
:101C600020534F4D455448494E4720544841542035
:101C70004120444F43544F52204749564553205921
:101C80004F553B505245534352495054494F4E3A99
:101C90003B53484F54530D3B42494C4C0C3B54452D
:101CA0005354093B41445649434507000000000096
:101CB000000000004E414D4520534F4D45544849CA
:101CC0004E472041204D4147494349414E204D4117
:101CD0004B4553204449534150504541523B52419A
:101CE000424249542F3B50454F504C451C3B4249C2
:101CF00052440B3B434F494E093B525542424552D9
:101D00002042414C4C020000000000004E414D4575
:101D100020534F4D455448494E4720544841542084
:101D2000474F455320475245415420574954482076
:101D30004348454553453B435241434B4552533C31
:101D40003B57494E45103B48414D083B4150504C94
:101D50004553073B5041535441030000000000002D
:101D6000000000004E414D4520534F4D4554484919
:101D70004E4720594F5520444F204F4E20594F5524
:101D800052204B4E4545533B50524159443B434CE6
:101D900045414E20464C4F4F52143B47415244451B
:101DA0004E063B424547033B435241574C0300001C
:101DB0000000000000000000000000004E414D4502
:101DC00020412053554D4D455220564143415449E1
:101DD0004F4E2053544154453B43414C49464F528A
:101DE0004E4941233B464C4F524944411B3B4841DD
:101DF00057414949073B434F4C4F5241444F063BE3
:101E00004F5245474F4E0300000000000000000005
:101E1000000000004E414D452041204B494E4420DA
:101E20004F4620545542453B494E4E45522054554D
:101E30004245263B544553542054554245213B547A
:101E40004F4F544850415354450F3B54562050492E
:101E50004354555245083B46414C4C4F5049414E26
:101E60000200000000000000000000004E414D454F
:101E700020534F4D455448494E4720594F55205304
:101E800045452041542041204255532053544F5042
:101E90003B42454E43483A3B50454F504C450F3B23
:101EA0004255532053544F50205349474E0C3B4208
:101EB0005553093B5343484544554C4504000000E5
:101EC000000000004E414D4520534F4D45544849B8
:101ED0004E472054484154204745545320504153C5
:101EE0005345442041524F554E4420544845204FBD
:101EF00046464943453B474F53534950243B4D4584
:101F00004D4F530D3B4A4F4B45530A3B434F4C44B7
:101F1000083B434152445304000000005245414CE9
:101F2000204F462046494354494F4E414C2C204EA9
:101F3000414D4520412046414D4F55532050524977
:101F40004E43453B434841524C4553383B4348413F
:101F5000524D494E47173B56414C49414E54083B60
:101F6000414C42455254043B5048494C49500300AF
:101F7000000000004E414D4520534F4D4554484907
:101F80004E472057495448204120484F4C4520494E
:101F90004E20544845204D4944444C453B444F4E07
:101FA0005554543B54495245053B424147454C0426
:101FB0003B4C4946455341564552033B5245434FDE
:101FC0005244023B52494E47020000004E414D45EB
:101FD00020534F4D455448494E472050454F504C93
:101FE00045204355542054484549522046494E47C0
:101FF000455253204F4E3B4B4E4946452C3B50419A
:10200000504552263B474C4153530C3B4752415499
:102010004552023B52415A4F52020000000000005C
:10202000000000004E414D4520534F4D4554484956
:102030004E4720544841542050454F504C45202293
:1020400050554C4C205550223B50414E54532E3B42
:10205000534F434B53133B5745454453103B50415B
:102060004E5459484F5345043B534841444553044B
:102070003B434F5645525302000000004E414D4530
:1020800020534F4D455448494E4720544841542011
:1020900055534553204241545445524945533B46BC
:1020A0004C4153484C494748542A3B524144494FBC
:1020B0001F3B544F59530D3B434152063B434C4F3A
:1020C000434B04000000000000000000000000007E
:1020D000000000004E414D4520414E20494E5354D2
:1020E00052554D454E5420494E2041205245414CB9
:1020F000202248494C4C42494C4C59222042414EE6
:10210000443B42414E4A4F323B464944444C4512BF
:102110003B57415348424F4152440D3B4A55470AB1
:102120003B47554954415204000000004E414D4583
:10213000204120434F554E54525920544841542079
:1021400057415320494E564F4C56454420494E2046
:10215000574F524C44205741522049493B55534117
:10216000283B4745524D414E591F3B4A4150414E35
:10217000113B454E474C414E44083B4652414E436D
:10218000450200004E414D4520534F4D45544849AE
:102190004E472050454F504C4520574F52525920E2
:1021A00041424F5554204C4F53494E473B484149BB
:1021B000521D3B4D4F4E4559123B4A4F420A3B4B35
:1021C000455953093B57414C4C455407000000000A
:1021D0000000000000000000000000004E414D45DE
:1021E0002041204348494C44275320504554205413
:1021F00048415420594F5520444F4E2754205045B4
:10220000543B46495348373B534E414B45183B548A
:102210005552544C45083B46524F47063B53504994
:1022200044455202000000000000000000000000D1
:10223000000000004E414D452041204B494E4420B6
:102240004F4620434849503B504F5441544F383B30
:1022500043484F434F4C415445103B504F4B455220
:102260000B3B434F4D5055544552063B434F524E46
:102270000600000000000000000000000000000058
:102280000000000000000000000000004E414D452D
:1022900020534F4D455448494E47205448415420FF
:1022A000474F4553204752454154205749544820F1
:1022B000535445414B3B504F5441544F4553493B78
:1022C00053414C4144083B4D555348524F4F4D5399
:1022D000063B4F4E494F4E53043B4245414E53033C
:1022E000000000004E414D452041205045542054EF
:1022F0004841542044524157532043524F5744536E
:1023000020544F205045542053544F524520574994
:102310004E444F57533B50555050593F3B4B4954F7
:1023200054454E0E3B4D4F4E4B45590D3B534E4180
:102330004B45053B42495244530200004E414D4536
:1023400020534F4D455448494E472050454F504C1F
:102350004520504F554E443B4E41494C53293B4D2F
:10236000454154233B464953540A3B504156454D41
:10237000454E54043B4445534B023B444F5547485C
:10238000020000000000000000000000000000004B
:10239000000000004E414D4520534F4D45544849E3
:1023A0004E4720544841542050454F504C452043FF
:1023B00048454154204F4E3B494E434F4D452054D4
:1023C0004158433B54455354103B44494554083B02
:1023D00053504F555345073B43415244530200006D
:1023E0000000000000000000000000004E414D45CC
:1023F0002041204445434953494F4E2054484520ED
:1024000057484F4C452046414D494C59204D414B72
:10241000455320544F4745544845523B564143414C
:1024200054494F4E3E3B4D4F56494E470D3B45415B
:10243000540B3B504554053B434152033B54560318
:10244000000000004F4E2041204441494C59204299
:10245000415349532C205748415420444F20594F51
:102460005520574F5252592041424F5554204D4FFD
:1024700053543F3B4D4F4E4559393B46414D494CD6
:1024800059103B4845414C5448073B574F524B0667
:102490003B57454947485405000000004E414D4513
:1024A00020534F4D455448494E47205448415420ED
:1024B0004B4E4F434B533B4341523C3B50454F5097
:1024C0004C45103B574F4F445045434B4552093BF9
:1024D000444F4F52204B4E4F434B4552073B4B4EC0
:1024E000454553053B4F50504F5254554E49545952
:1024F000020000004E414D4520534F4D4554484980
:102500004E4720412046414D494C5920444F4553A8
:1025100020544F4745544845523B4541543C3B5657
:1025200041434154494F4E0E3B4348555243480D99
:102530003B5049434E4943053B574154434820547F
:1025400056053B4152475545020000004E414D455E
:102550002041204B494E44204F4620534541464F91
:102560004F44205553454420494E20534F55503B2E
:10257000434C414D433B534852494D500C3B4F59FE
:10258000535445520A3B43524142043B4C4F425341
:10259000544552040000000000000000000000004C
:1025A000000000004E414D4520534F4D45544849D1
:1025B0004E47205448415420434C5542204D454DF0
:1025C0004245525320564F5445204F4E3B4F4646AE
:1025D00049434552532E3B4D454D424552531F3BB7
:1025E00052554C4553093B4D4F4E4559063B4455BA
:1025F0004553050000000000000000004E414D451D
:1026000020534F4D455448494E4720594F55205768
:10261000415348204556455259204441593B44496D
:10262000534845531E3B464143451C3B4841495294
:10263000143B48414E4453113B434C4F544845537F
:102640000300000000000000000000000000000087
:102650000000000054454C4C204D4520534F4D4543
:102660005448494E4720414E4E4F59494E472054F9
:10267000484154204341545320444F3B534352411B
:102680005443483C3B52554220414741494E5354E4
:1026900020594F55083B4D454F57073B434C494D3B
:1026A00042043B534845440300000000574841544E
:1026B000204F4E45205448494E47204D414B4553ED
:1026C00020594F555220484F555345204120484FDF
:1026D0004D453F3B4C4F56452B3B46414D494C5990
:1026E000203B4655524E4954555245073B504554A0
:1026F000053B5049435455524553023B5456020042
:10270000000000004E414D4520534F4D455448496F
:102710004E4720535045434946494320594F552081
:102720004D4947485420484944453B4D4F4E455933
:10273000443B4A4557454C5259073B44494152593D
:10274000053B4749465453033B4B45595302000050
:102750000000000000000000000000004E414D4558
:10276000204120574849544520414E494D414C3B5A
:10277000504F4C415220424541523F3B5241424210
:102780004954123B434154073B484F525345043B85
:102790005345414C02000000000000000000000012
:1027A0000000000000000000000000000000000029
:1027B000000000004E414D4520534F4D45544849BF
:1027C0004E4720544841542050454F504C452054CA
:1027D000554E453B5049414E4F2D3B47554954417D
:1027E00052163B524144494F153B434152073B541B
:1027F00056033B56494F4C494E0200000000000072
:102800000000000000000000000000004E414D45A7
:1028100020534F4D455448494E4720544845204683
:10282000414D494C592054414B4553205455524E2B
:1028300053205553494E473B42415448524F4F4D08
:10284000443B4341520D3B48414952204452594573
:1028500052063B50484F4E45043B54560200000080
:10286000000000004E414D4520594F555220464131
:10287000564F5249544520465249454420464F4FF1
:10288000443B504F5441544F45532B3B43484943DD
:102890004B454E253B46495348053B534852494D0D
:1028A00050043B48414D425552474552023B4F4E22
:1028B000494F4E2052494E47530200005748415459
:1028C000204C4956494E47204352454154555245A4
:1028D00020465249474854454E5320574F4D454E88
:1028E000204D4F53543F3B534E414B45303B53508B
:1028F00049444552123B4D4F555345083B444F47C1
:10290000043B425547043B534841524B03000000EF
:10291000000000004E414D4520534F4D455448495D
:102920004E47205448415420445249564553204371
:10293000415453204352415A593B4341544E49500C
:10294000353B444F4753163B4D4943450C3B59419A
:10295000524E043B42415448033B424952445302C5
:102960000000000000000000000000004E414D4546
:102970002041204B494E44204F462053434F504561
:102980003B54454C4553434F5045423B4D494352C0
:102990004F53434F50450E3B5249464C45205343FD
:1029A0004F5045083B5045524953434F5045063B15
:1029B00053434F5045204D4F5554485741534804B9
:1029C000000000004E414D4520534F4D45544849AD
:1029D0004E47205448415420434F4D455320494EC3
:1029E0002050414952533B53484F4553453B534F69
:1029F000434B53163B50414E5453023B53414C54AE
:102A0000202620504550504552023B5457494E53C2
:102A10000200000000000000000000004E414D4593
:102A200020534F4D455448494E47204E45574C5929
:102A300057454453205341564520464F523B484F3B
:102A40004D45443B4655524E49545552450E3B4226
:102A5000414259093B5641434154494F4E043B437F
:102A600041520200000000000000000000000000D1
:102A7000000000004E414D4520534F4D45544849FC
:102A80004E4720594F552045415420425920544823
:102A9000452048414E4446554C3B504F50434F52C1
:102AA0004E313B4E555453243B4348495053073B0A
:102AB00043414E4459063B475241504553020000A2
:102AC0000000000000000000000000004E414D45E5
:102AD00020534F4D455448494E4720594F552744A0
:102AE0002046494E4420494E2041204241524E3B0F
:102AF0004841593E3B434F57133B484F52534507BC
:102B00003B434F524E023B54524143544F520200FA
:102B100000000000000000000000000000000000B5
:102B2000000000004E414D4520534F4D455448494B
:102B30004E472050454F504C452054494E54204F4D
:102B40005220434F4C4F523B48414952433B574917
:102B50004E444F5753113B455945474C41535345FC
:102B600053083B43414B45023B454153544552209A
:102B70004547475302000000000000004E414D450C
:102B800020534F4D455448494E472050454F504CD7
:102B900045205741583B434152403B464C4F4F52D2
:102BA00053153B4655524E4954555245043B534BE1
:102BB0004953033B4D4F5553544143484502000090
:102BC0000000000000000000000000000000000005
:102BD000000000004E414D4520534F4D455448499B
:102BE0004E4720544841542048415320504F434BB6
:102BF0004554533B50414E5453413B434F4154166F
:102C00003B504F4F4C205441424C45063B415052A3
:102C10004F4E023B4B414E4741524F4F023B5348B0
:102C20004952540200000000000000004E414D4592
:102C300020534F4D455448494E4720494E20594F47
:102C4000555220484F555345205448415420435233
:102C500045454B533B464C4F4F52363B53544149ED
:102C60005253153B444F4F520B3B43484149520688
:102C70003B524F4F460200000000000000000000E1
:102C8000000000004E414D45204120464F4F44205A
:102C900054484154275320534F4D4554494D4553B3
:102CA00020474C415A45443B444F4E5554363B48CF
:102CB000414D1A3B43414B45073B434152524F5410
:102CC00053063B535745455420504F5441544F45AC
:102CD0005302000000000000000000004E414D457E
:102CE00020534F4D455448494E4720594F55205386
:102CF0004545204F4E204120545241434B3B5452B6
:102D000041494E3D3B484F525345193B43415204C4
:102D10003B52554E4E4552043B47524559484F553C
:102D20004E4402000000000000000000000000000F
:102D3000000000004E414D4520534F4D4554484939
:102D40004E47205749544820535452495045533B0D
:102D5000464C41473C3B5A45425241183B554E492F
:102D6000464F524D073B43414E44592043414E4547
:102D7000043B544947455203000000000000000096
:102D80000000000000000000000000004E414D4522
:102D900020412053504F5254205749544820524FFD
:102DA00057445920535045435441544F52533B4686
:102DB0004F4F5442414C4C1E3B484F434B45591CCE
:102DC0003B534F43434552173B57524553544C498D
:102DD0004E470C3B524F44454F030000000000009B
:102DE000000000004E414D4520534F4D4554484989
:102DF0004E4720464F554E4420494E204120504CCE
:102E0000415947524F554E443B5357494E47483B13
:102E1000534C494445103B4D4552525920474F2091
:102E2000524F554E44043B534545534157043B5381
:102E3000414E44424F580300000000004E414D45B2
:102E400020534F4D455448494E4720544841542043
:102E500043414E20424520504F505045443B504F37
:102E600050434F524E3E3B42414C4C4F4F4E133B12
:102E70004348414D5041474E45063B50494D504C0B
:102E800045043B425542424C45030000000000000F
:102E9000000000004E414D4520534F4D45544849D8
:102EA0004E47204D494E5420464C41564F524544C2
:102EB0003B47554D403B49434520435245414D0B0F
:102EC0003B544F4F54485041535445073B414E5497
:102ED00041434944053B4D4F5554485741534805DC
:102EE0003B54454103000000000000004E414D45A9
:102EF00020534F4D455448494E4720544841542093
:102F0000434F4D4553204F5554204154204E49477F
:102F100048543B4D4F4F4E183B5354415253163B70
:102F200042415453143B4F574C53143B5445455462
:102F30004803000000000000000000000000000046
:102F4000000000004E414D4520414E20494E475261
:102F5000454449454E5420594F5520505554204919
:102F60004E20414E204F4D454C45543B454747531D
:102F70003F3B434845455345103B48414D063B4781
:102F80005245454E20504550504552053B4D494C09
:102F90004B033B4F4E494F4E530200004E414D45AF
:102FA00020534F4D455448494E47205448415420E2
:102FB000414C5741595320434F5354532041204CC7
:102FC0004F5420544F205245504149523B434152A7
:102FD0004B3B5456063B484F555345053B524546DF
:102FE000524947455241544F52023B57415443487E
:102FF000020000004E414D45204120504C414345C8
:10300000204F4E20594F555220424F445920574887
:1030100045524520594F5527442046494E442047A4
:103020004F4C443B48414E443C3B4D4F5554481750
:103030003B4E45434B093B45415253043B57524994
:103040005354040000000000000000004E414D45B4
:1030500020534F4D455448494E472050454F504C02
:10306000452050494E2055503B504F535445523601
:103070003B48414952123B434C4F544845530C3B4B
:1030800043414C454E4441520700000000000000FF
:103090000000000000000000000000000000000030
:1030A000000000004E414D4520534F4D45544849C6
:1030B0004E4720594F55205345543B434C4F434BAB
:1030C000393B48414952123B5441424C450E3B5614
:1030D0004352060000000000000000000000000055
:1030E00000000000000000000000000000000000E0
:1030F00000000000000000000000000047495645A5
:10310000204D45204120574F5244205448415420DF
:1031100041204241534542414C4C20554D5049526B
:103120004520555345533B4F55542D3B535452491D
:103130004B45283B534146450B3B464F554C0200FF
:10314000000000000000000000000000000000007F
:10315000000000004E414D452041204B494E442087
:103160004F46204B4559205445454E414745525303
:1031700020484156453B484F5553453E3B434152FD
:10318000123B4C4F434B45520D3B4449415259036E
:10319000000000000000000000000000000000002F
:1031A0000000000000000000000000004E414D45FE
:1031B00020534F4D455448494E47204D454E2044DD
:1031C0004F205748454E20412050524554545920D5
:1031D0004749524C205041535345533B574849535C
:1031E000544C453C3B4C4F4F4B1E3B534D494C457B
:1031F00005000000000000000000000000000000CA
:10320000000000004E414D45204120504C414345B7
:10321000205748455245204D454E2054524144497F
:1032200054494F4E414C4C592048414E47204F5530
:10323000543B424152463B504F4F4C2048414C4C2E
:10324000113B47594D053B424F574C494E47204192
:103250004C4C455902000000000000004E414D4515
:103260002041204B494E44204F4620504C4143457D
:103270002054484154204841532041204C4F424261
:10328000593B484F54454C543B5448454154524592
:10329000093B42414E4B033B484F53504954414C2C
:1032A000030000000000000000000000000000001B
:1032B000000000004E414D452054484520415050EB
:1032C0004C49414E43452054484154204C415354AD
:1032D0005320544845204C4F4E474553543B52458C
:1032E00046524947455241544F52303B53544F5632
:1032F000451C3B544F4153544552063B574153489C
:103300004552060000000000000000004E414D45FF
:103310002041204849474820504159494E47204FB5
:10332000434355504154494F4E3B504859534943EC
:1033300049414E313B4154544F524E4559233B5025
:10334000494C4F54053B50524F204154484C455432
:1033500045043B414354494E470300000000000030
:10336000000000004E414D4520534F4D4554484903
:103370004E472054484154204B45455053204B491B
:10338000445320494E444F4F52533B4241442057EF
:10339000454154484552463B494C4C4E4553530FCA
:1033A0003B5456083B434F4D505554455204000082
:1033B0000000000000000000000000004E414D45EC
:1033C00020534F4D455448494E47205448415420BE
:1033D00053484F554C44204841564520414E2049C2
:1033E0002E442E20544147204F4E2049543B5355E4
:1033F000495443415345343B414E494D414C253B93
:103400004348494C44043B42524945464341534595
:10341000020000004E414D4520534F4D4554484950
:103420004E472050454F504C452053454520574866
:10343000454E205448455920474F20534E4F524B3C
:10344000454C494E473B464953484C3B434F5241FC
:103450004C103B5348454C4C53033B534541574557
:1034600045440200000000000000000046524F4D9D
:103470002057484F4D20444F20594F55205448491C
:103480004E4B20594F552043415547485420594FE2
:103490005552204C41535420434F4C443F3B5350D2
:1034A0004F555345363B4348494C44213B465249CE
:1034B000454E44073B434F574F524B455205000082
:1034C000000000004E414D45204120464F4F442012
:1034D000594F55205041434B20464F5220544845A8
:1034E0002042454143483B53414E44574943484598
:1034F00053293B4348495053193B434849434B45A3
:103500004E0F3B484F5420444F47530A3B465255B9
:103510004954050000000000000000004E414D45E8
:1035200020534F4D455448494E4720412043484978
:103530004C4420504C415953205749544820494E3F
:1035400020544845204241434B594152443B535734
:10355000494E47343B42414C4C143B444F470D3B92
:1035600053414E44424F5807000000000000000045
:10357000000000004E414D4520534F4D45544849F1
:103580004E472050454F504C45205745415220460C
:103590004F522050524F54454354494F4E3B474F92
:1035A00047474C4553183B48454C4D4554143B52F6
:1035B00041494E434F41540D3B474C4F5645530BE9
:1035C0000000000000000000000000004E414D45DA
:1035D00020534F4D455448494E47204153534F4384
:1035E00049415445442057495448204144414D20C5
:1035F00026204556453B4150504C453A3B474152A9
:1036000044454E204F46204544454E103B534E41C5
:103610004B450C3B464947204C45414609000000BC
:10362000000000004E414D452041205041525420A1
:103630004F462054484520424F4459205448415455
:1036400020594F552042525553483B484149523129
:103650003B54454554482B3B4241434B043B464970
:103660004E4745524E41494C5302000000000000B5
:103670000000000000000000000000004E414D4529
:1036800020414E20455850454E5345205448415402
:1036900020474F4553205550205748454E20594FFD
:1036A0005520474554204D4152524945443B464FD1
:1036B0004F44503B494E535552414E4345093B43BD
:1036C0004C4F54484553033B54454C4550484F4E8E
:1036D000450200004E414D452041204A4F422049BD
:1036E0004E2057484943482050454F504C4520579D
:1036F0004541522057484954452048415453204F92
:103700005220434150533B4E55525345313B434861
:103710004546273B42555443484552023B53414995
:103720004C4F520200000000000000004E414D4589
:1037300020414E204F43434153494F4E2057484567
:103740004E204120574F4D414E204D49474854206F
:10375000574541522041204841543B574544444934
:103760004E47203B46554E4552414C1A3B4541532E
:10377000544552133B4348555243480F0000000044
:10378000000000004E414D4520534F4D45544849DF
:103790004E472050454F504C4520444F20574845F8
:1037A0004E2054484559204841564520544845200C
:1037B0004348494C4C533B5348414B45313B474FA1
:1037C00020544F20424544103B42554E444C452026
:1037D00055500F0000000000000000004E414D4514
:1037E0002041205350454349464943204954454DC3
:1037F00020594F552048415645204F4E20412050DA
:103800004154494F3B4241524245435545283B4371
:1038100048414952213B5441424C45103B504C4198
:103820004E54053B5357494E47020000000000002C
:10383000000000004E414D4520534F4D455448492E
:103840004E4720594F5520444F205748494C45205A
:10385000594F5520534F414B20494E205448452045
:103860005455423B52454144323B52454C41581B12
:103870003B53494E47083B5348415645030000001F
:103880000000000000000000000000004E414D4517
:1038900020414E20455850454E53495645204641FB
:1038A000425249433B53494C4B4B3B56454C564582
:1038B00054093B434153484D455245053B53415400
:1038C000494E043B535545444504000000000000A8
:1038D00000000000000000000000000000000000E8
:1038E000000000004E414D4520414E20414E494DC3
:1038F000414C20544841542050454F504C45205293
:103900004944453B484F525345533B43414D454C39
:10391000073B454C455048414E54043B444F4E4BA9
:1039200045590300000000000000000000000000F6
:103930000000000000000000000000004E414D4566
:1039400020534F4D455448494E4720544841542038
:1039500048415320524F4F54533B54524545413BED
:10396000504C414E540F3B484149520E3B54454543
:1039700054480300000000000000000000000000A8
:103980000000000000000000000000000000000037
:10399000000000004E414D4520534F4D45544849CD
:1039A0004E472054484154204953205345414C45EB
:1039B000443B4D41494C413B4D45444943494E45AB
:1039C000143B4D494C4B20434152544F4E033B4313
:1039D000455245414C02000000000000000000007C
:1039E0000000000000000000000000004E414D45B6
:1039F00020534F4D455448494E472050454F504C59
:103A00004520505554204F4E20412043414B453BCB
:103A10004943494E472D3B43414E444C45532C3B73
:103A200049434520435245414D0600000000000037
:103A30000000000000000000000000000000000086
:103A40000000000047495645204D4520414E4F5447
:103A500048455220574F524420464F5220224E4F45
:103A60004E53454E5345223B53494C4C59223B46FD
:103A70004F4F4C4953480E3B5249444943554C4FD4
:103A80005553083B41425355524406000000000084
:103A90000000000000000000000000004E414D4505
:103AA00020414E20554E555355414C20504C4143DA
:103AB00045205748455245204241424945532041FF
:103AC000524520534F4D4554494D455320424F5286
:103AD0004E3B4341524D3B414952504C414E4507AC
:103AE0003B484F4D45063B454C455641544F5206C9
:103AF000000000004E414D4520534F4D455448496C
:103B00004E472050454F504C452053544545523B5D
:103B10004341525A3B424F4154043B42494359436B
:103B20004C45023B47524F43455259204341525462
:103B30000200000000000000000000000000000083
:103B40000000000000000000000000004E414D4554
:103B5000204120504F50554C4152204D41494C205E
:103B60004F5244455220434154414C4F4755453BE9
:103B70005345415253353B5350494547454C103B03
:103B80004A4350454E4E59093B4C4C204245414E0C
:103B9000060000000000000000000000000000001F
:103BA000000000004E414D4520534F4D45544849BB
:103BB0004E47204153534F434941544544205749B0
:103BC000544820414E47454C533B48414C4F2D3BB8
:103BD00057494E4753203B48454156454E0E3B48BA
:103BE000415250530300000000000000000000009C
:103BF0000000000000000000000000004E414D45A4
:103C000020534F4D455448494E4720555345442075
:103C100041532041205441424C452043454E544598
:103C20005250494543453B464C4F57455253513BF3
:103C300043414E444C45530B3B424F574C204F465B
:103C400020465255495403000000000000000000C7
:103C5000000000005748415420444F455320412064
:103C6000574F4D414E20534159205748454E204112
:103C7000204D414E2050524F504F5345533F3B59DA
:103C800045534C3B49204C4F564520594F55043B1A
:103C90004E4F043B41524520594F55204B49444417
:103CA000494E470300000000000000004E414D4512
:103CB00020534F4D455448494E4720594F552050A9
:103CC0004C414E204D4F4E54485320494E204144C4
:103CD00056414E43453B5641434154494F4E403B6C
:103CE00057454444494E471E3B4348524953544D5F
:103CF0004153023B50415254590200000000000061
:103D0000000000004E414D4520534F4D4554484959
:103D10004E47205745204745542046524F4D20419D
:103D200020434F573B4D494C4B543B424545460879
:103D30003B434845455345033B4C45415448455258
:103D40000200000000000000000000000000000071
:103D50000000000000000000000000004E414D4542
:103D600020534F4D455448494E4720544841542014
:103D700053494E4B53204120534849503B544F52D6
:103D80005045444F383B494345424552471D3B4807
:103D90004F4C45093B434F52414C0200000000008C
:103DA0000000000000000000000000000000000013
:103DB00000000000574841542049532054484520F2
:103DC000424553542057415920544F20464C4154AA
:103DD00054454E20594F55522053544F4D4143485E
:103DE0003F3B4558455243495345563B444945544A
:103DF0000A3B5355434B20494E20425245415448BB
:103E0000023B474952444C45020000004245534999
:103E100044455320434F4F4B49455320262043529E
:103E200041434B4552532C204E414D4520534F4D5D
:103E3000455448494E47204B45505420494E204157
:103E400020434F4F4B4945204A41523B4D4F4E4531
:103E500059533B43414E44590A3B4B455953040087
:103E6000000000004E414D45204F4E45204F46205A
:103E700054484520524F4F534556454C54533B549C
:103E800048454F444F52453E3B4652414E4B4C49AC
:103E90004E2044183B454C45414E4F520D0000000A
:103EA0000000000000000000000000000000000012
:103EB0000000000000000000000000004E414D45E1
:103EC00020534F4D455448494E4720594F552044A3
:103ED0004F204F4E20544950544F453B44414E4390
:103EE000452A3B5245414348263B57414C4B093BF1
:103EF0004B49535305000000000000000000000083
:103F000000000000000000000000000000000000B1
:103F1000000000004E414D4520412053504F525467
:103F200020494E20574849434820594F5520574F64
:103F3000554C4420484541522054484520574F5243
:103F40004420225354524F4B45223B474F4C462F5F
:103F50003B524F57494E47193B5357494D4D494ED8
:103F600047183B54454E4E49530400004E414D45C1
:103F700020534F4D455448494E4720544841542002
:103F8000484F50533B524142424954493B46524F9D
:103F9000470D3B4752415353484F50504552073B02
:103FA0004B414E4741524F4F0400000000000000BB
:103FB0000000000000000000000000000000000001
:103FC000000000004E414D4520534F4D4554484997
:103FD0004E472054484154204245455320444F3BCE
:103FE0004D414B4520484F4E45592E3B5354494E69
:103FF000471A3B42555A5A103B504F4C4C494E4180
:1040000054450C000000000000000000000000000B
:104010000000000000000000000000004E414D457F
:1040200020534F4D455448494E4720544841542051
:1040300050454F504C452053484F5254454E3B53EA
:104040004B4952542F3B50414E5453163B4E414D19
:1040500045113B484149520B0000000000000000A0
:104060000000000000000000000000000000000050
:10407000000000004E414D4520534F4D45544849E6
:104080004E472C20424553494445532053484F4501
:10409000532C20534F4C442041542053484F45202B
:1040A00053544F5245533B534F434B53223B505570
:1040B000525345531F3B504F4C4953480D3B4C41C5
:1040C0004345530A00000000000000004E414D45EA
:1040D00020412043414E414C3B50414E414D4120F7
:1040E00043414E414C313B455249452043414E41AD
:1040F0004C223B5355455A2043414E414C0E3B4CBC
:104100004F56452043414E414C0200000000000044
:10411000000000000000000000000000000000009F
:10412000000000004E414D4520534F4D4554484935
:104130004E47205448415420574F554C4420424547
:1041400020494D504F535349424C4520544F204431
:104150004F20494E20544845204441524B3B524544
:104160004144453B5345570E3B5752495445083B44
:104170004452495645030000000000004E414D45A1
:1041800020534F4D455448494E47205448415420F0
:1041900044524F50533B5741544552313B54454D87
:1041A0005045524154555245153B544541525304D4
:1041B0003B50494E030000000000000000000000DA
:1041C00000000000000000000000000000000000EF
:1041D000000000004E414D4520534F4D4554484985
:1041E0004E472050454F504C4520434C454E434888
:1041F0003B46495354313B54454554482B3B4D4F66
:104200004E455903000000000000000000000000BF
:10421000000000000000000000000000000000009E
:104220000000000000000000000000004E414D456D
:1042300020534F4D455448494E47204B4944532045
:104240004C494B4520544F20434C494D42204F4E42
:104250003B5452454553323B4655524E49545552B4
:10426000451B3B4A554E474C452047594D0E3B5048
:10427000454F504C450300000000000000000000C6
:10428000000000004E414D4520594F5552204641F7
:10429000564F52495445205448494E4720544F20C8
:1042A000444F20415420414E20414D5553454D45EA
:1042B0004E54205041524B3B52494445534A3B4592
:1042C00041540F3B5741544348053B504C41592002
:1042D00047414D4553030000000000004E414D454D
:1042E000204120574F5252592054484154205045A4
:1042F0004F504C45204C4F534520534C4545502082
:104300004F5645523B4D4F4E45594D3B4A4F420B40
:104310003B46414D494C59063B4845414C544802A7
:10432000000000000000000000000000000000008D
:10433000000000004E414D4520544845204F4E4559
:10434000205448494E47205448415420594F552045
:104350004D4F5354204F4654454E204D4953504CD9
:104360004143453B4B455953463B474C41535345CD
:1043700053143B50454E43494C04000000000000DC
:104380000000000000000000000000004E414D450C
:1043900020534F4D455448494E4720594F552044CE
:1043A00052494E4B20484F543B434F4646454541AA
:1043B0003B434F434F41113B5445410F0000000028
:1043C00000000000000000000000000000000000ED
:1043D00000000000000000000000000000000000DD
:1043E000000000004E414D4520534F4D4554484973
:1043F0004E4720544841542050454F504C4520448E
:10440000554E4B3B444F4E555453443B4241534B06
:10441000455442414C4C0D3B50454F504C45073B99
:10442000434F4F4B494553053B4150504C45530278
:104430003B42524541440200000000004E414D45C0
:1044400020534F4D455448494E4720594F5520540D
:104450005259204F555420464F523B53504F5254BF
:1044600053205445414D263B504C41591D3B434838
:104470004545524C4541444552153B4A4F42050083
:10448000000000000000000000000000000000002C
:10449000000000004E414D4520534F4D45544849C2
:1044A0004E47204120434152204E45454453204928
:1044B0004E205448452057494E5445523B414E5496
:1044C0004920465245455A454A3B53484F57205488
:1044D00049524553103B484541544552053B4348DA
:1044E00041494E5303000000000000004E414D457D
:1044F00020412053494E47494E472047524F55507F
:1045000020544841542053504C49542055503B426C
:104510004541544C4553413B53555052454D4553ED
:104520000B3B534F4E4E5920262043484552043BE7
:104530004D4F4E4B45595303000000000000000052
:10454000000000004E414D4520534F4D4554484911
:104550004E47204245534944455320594F555253E5
:10456000454C462C205448415420594F5520574122
:1045700053483B4341522B3B434C4F5448455328EF
:104580003B4449534845530E3B57494E444F5753BC
:104590000200000000000000000000004E414D45F8
:1045A00020534F4D455448494E4720594F55204CB4
:1045B000494B4520544F20424520414C4F4E452009
:1045C000544F20444F3B524541443E3B42415448A6
:1045D00045093B5752495445053B434C45414E0420
:1045E00000000000000000000000000000000000CB
:1045F000000000004E414D4520534F4D4554484961
:104600004E4720594F5527442046494E4420494E95
:104610002041205343484F4F4C20504C4159475262
:104620004F554E443B5357494E4753503B534C49CB
:104630004445073B4348494C4452454E053B4D4F8A
:104640004E4B455920424152530500004E414D45C5
:10465000204120535045434946494320434F4D494B
:104660004320424F4F4B2053555045524845524FDF
:104670003B53555045524D414E4A3B53504944459A
:10468000524D414E0D3B4241544D414E073B444932
:10469000434B2054524143590200000000000000E7
:1046A000000000004E414D4520534F4D45544849B0
:1046B0004E4720544841542052554E53204F4E20CF
:1046C0004120545241434B3B545241494E5A3B487E
:1046D0004F525345043B444F47023B524143452010
:1046E00043415202000000000000000000000000F2
:1046F0000000000000000000000000005748415486
:10470000204F4E45205448494E47204D414B45537C
:1047100020594F5552204A4F4220574F5254485724
:1047200048494C453F3B4D4F4E4559413B50454F05
:10473000504C45083B42454E4546495453043B4284
:104740004F53530400000000000000000000000070
:10475000000000004E414D4520534F4D45544849FF
:104760004E47204E45574C595745445320474F20FC
:10477000494E544F204445425420544F20425559ED
:104780003B484F555345393B4655524E4954555277
:10479000451E3B434152093B52454652494745520B
:1047A00041544F520200000000000000574841549D
:1047B0002050415254204F4620594F5552205350BB
:1047C0004F555345275320424F44592049532041C8
:1047D0004C5741595320434F4C443F3B4645455469
:1047E0004F3B4E4F53450D3B48414E44530500004F
:1047F00000000000000000000000000000000000B9
:10480000000000004E414D4520534F4D455448494E
:104810004E4720594F5520444F20464F52204120AB
:10482000424142593B4348414E474520444941504B
:104830004552273B46454544204954263B42555264
:10484000502049540A3B4241544845204954043BB6
:104850004C4F564520495403000000004E414D4541
:1048600020534F4D455448494E47204D4F544845DD
:104870005253204E45454453204C4F5453204F46ED
:1048800020464F52205448454952204E4557424FEA
:10489000524E3B444941504552534F3B504154497D
:1048A000454E4345073B4C4F5645053B4D494C4B08
:1048B000030000004E414D4520534F4D455448499B
:1048C0004E4720544841542052455455524E53208F
:1048D000494E2054484520535052494E4754494D63
:1048E000453B4249524453323B464C4F5745525345
:1048F0001D3B4C4541564553053B53554E04000066
:104900000000000000000000000000004E414D4586
:1049100020534F4D454F4E4520594F552752452066
:10492000414C5741595320434C45414E494E472035
:1049300055502041465445523B4348494C443E3B28
:1049400048555342414E44183B444F47073B594F4B
:10495000555253454C460300000000000000000083
:10496000000000004E414D4520534F4D45544849ED
:104970004E472050454F504C4520444F2057484902
:104980004C45205741544348494E472054563B45D7
:1049900041545B3B4B4E4954033B52454144033B1E
:1049A00046414C4C2041534C45455002000000000C
:1049B0000000000000000000000000004E414D45D6
:1049C00020412050524F445543542050454F504CA5
:1049D000452042555920464F5220495453204649BC
:1049E000524D20535550504F52543B4D4154545208
:1049F000455353353B425241183B474952444C457D
:104A00000A3B50414E5459484F534508000000009E
:104A1000000000004E414D4520534F4D455448493C
:104A20004E4720544841542050454F504C45204457
:104A30004F204F4E20504159204441593B474F2071
:104A4000544F2042414E4B2B3B474F2053484F5031
:104A500050494E47133B5041592042494C4C531347
:104A60003B454154204F5554130000004E414D45E5
:104A700020534F4D455448494E47205448415420F7
:104A800048415320544F205741524D205550204209
:104A900045464F524520594F5520555345204954BE
:104AA0003B4F56454E1C3B49524F4E1B3B435552C4
:104AB0004C494E472049524F4E143B434152090046
:104AC000000000004E414D4520534F4D455448498C
:104AD0004E472050454F504C4520484154452054A6
:104AE0004F2047455420494E544F204946204954B1
:104AF000275320434F4C443B57415445523A3B4285
:104B00004544173B434152100000000000000000E4
:104B10000000000000000000000000004E414D4574
:104B200020534F4D455448494E4720544841542046
:104B300054414B455320504C41434520494E204160
:104B40002052494E473B424F58494E47463B434906
:104B500052435553113B57524553544C494E470805
:104B60003B42554C4C464947485403000000000066
:104B7000000000004E414D45204120535550455204
:104B80004845524F2057484F20574F52452041200B
:104B90004D41534B3B4241544D414E363B4C4F4EA1
:104BA000452052414E474552213B535049444552BE
:104BB0004D414E063B5A4F52524F06000000000036
:104BC0000000000000000000000000004E414D45C4
:104BD00020534F4D455448494E4720535045434973
:104BE000464943205448415420444F4753204C49A0
:104BF0004B4520544F2043484153453B4341545378
:104C0000303B43415253253B4D41494C2043415297
:104C100052494552043B42414C4C530300000000B2
:104C2000000000004E414D4520534F4D455448492A
:104C30004E4720594F552047455420414E2045535B
:104C400054494D415445204F4E204245464F524510
:104C500020594F552047455420495420464958452E
:104C6000443B434152563B524F4F46053B5456043A
:104C70003B504C554D42494E47030000474956456D
:104C8000204D45204120534C414E4720574F524420
:104C900020464F5220464143453B4D55474A3B50E5
:104CA000555353103B4B49535345520400000000E9
:104CB00000000000000000000000000000000000F4
:104CC00000000000000000000000000000000000E4
:104CD000000000004E414D4520534F4D455448497A
:104CE0004E4720544841542050454F504C45204792
:104CF00052494E443B5445455448373B434F464642
:104D00004545243B504550504552033B434F524E7E
:104D10000200000000000000000000000000000091
:104D20000000000000000000000000004E414D4562
:104D300020534F4D455448494E472053494E474C08
:104D400045204D454E204C4541524E20544F204465
:104D50004F20464F52205448454D53454C564553DD
:104D60003B434F4F4B433B5741534820434C4F54D9
:104D7000484553163B49524F4E053B534557030098
:104D8000000000004E414D45204120574F52442025
:104D900041204241534542414C4C20554D504952CF
:104DA0004520555345533B535452494B452B3B4F9C
:104DB0005554293B534146450B3B42414C4C040062
:104DC00000000000000000000000000000000000E3
:104DD0000000000000000000000000004E414D45B2
:104DE00020534F4D455448494E472050454F504C55
:104DF000452047524F57204649454C4453204F4683
:104E00003B434F524E383B5748454154163B434F66
:104E100054544F4E083B464C4F57455253050000E3
:104E20000000000000000000000000000000000082
:104E3000000000004E414D4520534F4D4554484918
:104E40004E472050454F504C452042555920534520
:104E5000434F4E442048414E443B434152423B4322
:104E60004C4F54484553123B4655524E49545552A7
:104E7000450C0000000000000000000000000000E1
:104E80000000000000000000000000004E414D4501
:104E900020534F4D455448494E47204C4954544C9B
:104EA00045204749524C53204452455353204153C7
:104EB0002041542048414C4C4F5745454E3B5749A3
:104EC000544348383B5052494E43455353123B419B
:104ED0004E47454C043B42414C4C4552494E4104DF
:104EE000000000004E414D4520534F4D4554484968
:104EF0004E47205448415427532053454C46205395
:104F00004552564943453B47415320535441544928
:104F10004F4E553B4C41554E44524F4D4154043B2E
:104F20004341522057415348023B53555045524D3F
:104F300041524B4554020000000000004E414D45D7
:104F400020534F4D455448494E4720544841542022
:104F50004849535345533B534E414B45483B4341CE
:104F6000540C3B464C4154043B5241444941544F3C
:104F700052030000000000000000000000000000DC
:104F80000000000000000000000000000000000021
:104F9000000000004E414D4520534F4D45544849B7
:104FA0004E4720412044454E5449535420534159C3
:104FB000533B4F50454E2057494445563B54484972
:104FC0005320574F4E27542048555254053B5249C1
:104FD0004E5345033B53504954030000000000006A
:104FE0000000000000000000000000004E414D45A0
:104FF00020412054595045204F4620504F5744459A
:10500000523B42414259493B47554E0E3B46414374
:1050100045093B42414B494E470200000000000059
:105020000000000000000000000000000000000080
:105030000000000000000000000000000000000070
:10504000000000004E414D4520412053504F525426
:1050500020504C4159454420494E2053484F52540A
:10506000533B54454E4E4953293B534F43434552BE
:105070001D3B4241534B455442414C4C193B564F0A
:105080004C4C455942414C4C0300000000000000CC
:1050900000000000000000000000000054454C4CDF
:1050A000204D4520534F4D455448494E4720594FB8
:1050B00055204D414B452041204C495354204F46EB
:1050C0003B53484F5050494E47204C495354533B53
:1050D0005448494E475320544F20444F0D3B584DA0
:1050E000415320474946545302000000000000008D
:1050F000000000004E414D4520534F4D4554484956
:105100004E47205448415420474F4553204752456D
:105110004154205749544820504F5441544F204344
:10512000484950533B44495053463B48414D4255F2
:105130005247455253083B484F5420424F4753086B
:105140003B534F4441060000000000004E414D45D6
:1051500020534F4D455448494E472050454F504CE1
:105160004520484156452041542054484549522045
:1051700046524F4E5420444F4F523B4D41544B3BAF
:10518000444F4F5242454C4C103B4C494748540405
:10519000000000000000000000000000000000000F
:1051A000000000004E414D45204120434F4D504FDF
:1051B000534552204F4620434C4153534943204DC1
:1051C000555349433B42454554484F56454E233B72
:1051D000424143481B3B4D4F5A4152541B3B4348AD
:1051E0004F50494E04000000000000000000000085
:1051F0000000000000000000000000004E414D458E
:10520000204120465249454E444C5920414E494D7B
:10521000414C3B444F47323B434154293B5241426E
:10522000424954033B474F41540200000000000034
:10523000000000000000000000000000000000006E
:10524000000000000000000000000000000000005E
:105250000000000050415354204F522050524553FB
:10526000454E542C204E414D4520412046414D4F46
:10527000555320552E532E20505249534F4E3B41EB
:105280004C43415452415A4C3B53494E4720534999
:105290004E470A3B464F4C534F4D073B53414E2020
:1052A0005155454E54494E05000000004E414D45B4
:1052B00020414E5920434956494C205741522047DE
:1052C000454E4552414C204F4620544845204E4FB4
:1052D000525448204F5220534F5554483B4C45455B
:1052E000463B4752414E54163B534845524D414E62
:1052F000043B4A41434B534F4E0300000000000063
:10530000000000004E414D4520534F4D4554484943
:105310004E4720594F55204D4947485420444F206F
:105320005748454E20544845205456204953204262
:10533000524F4B454E3B52454144393B4D555349E5
:1053400043133B4341524453093B4D4F5649450398
:105350000000000000000000000000004E414D452C
:1053600020534F4D455448494E47205448415420FE
:1053700048494748205343484F4F4C204B494453DA
:1053800020545259204F555420464F523B53504FB2
:10539000525453353B43484545524C454144455290
:1053A0001A3B504C4159113B42414E44040000000D
:1053B000000000004E414D4520414E20414E494DD8
:1053C000414C20544841542050454F504C452042B8
:1053D000524545443B444F4753463B484F52534543
:1053E00053163B434154544C45033B5241424249BE
:1053F0005453020000000000000000000000000004
:105400000000000000000000000000005748415468
:1054100020494E464C55454E43455320544845205F
:10542000434C4F5448455320594F552057454152FE
:105430002045414348204441593F3B57454154484A
:1054400045524B3B4D4F4F440A3B4A4F42053B5759
:10545000484154275320434C45414E03000000006F
:10546000000000004E414D4520534F4D45544849E2
:105470004E472041424F5554205748494348204108
:10548000204D414E20534159532022495427532047
:105490004D592057484F4C45204C494645223B4AE0
:1054A0004F42333B46414D494C59213B53504F529B
:1054B0005453063B43415205000000004E414D4508
:1054C00020534F4D455448494E4720464F554E4472
:1054D00020494E204120484F53504954414C2052BE
:1054E0004F4F4D3B4245444D3B42454450414E0D8C
:1054F0003B43414C4C20425554544F4E023B4F5875
:105500005947454E02000000000000000000000066
:10551000000000004E414D45204120524541534F6F
:105520004E20594F55204D49474854204E4F572043
:1055300057414E5420544F20474554204F55542036
:105540004F46204245443B5349434B263B544F4F23
:1055500020434F4C44173B5449524544113B48416A
:10556000544520574F524B08000000004E414D4516
:105570002041204C4157204D414E592050454F501D
:105580004C4520425245414B3B5350454544494EC2
:1055900047503B4A415957414C4B494E470A3B4CB7
:1055A0004954544552494E47053B53544F5020539C
:1055B00049474E53020000000000000000000000B8
:1055C000000000004E414D45204120464F4F4420F1
:1055D000594F55204255592053485245444445445B
:1055E0003B4348454553454A3B57484541540D3B8D
:1055F00043414242414745073B434F434F4E555479
:105600000400000000000000000000000000000096
:105610000000000000000000000000004E414D4569
:1056200020534F4D455448494E472054484154203B
:10563000594F552042554E444C452055503B424110
:105640004259413B4E455753504150455253193BE7
:10565000594F555253454C46043B444952545920E6
:105660004C41554E44525903000000000000000018
:10567000000000004E414D4520534F4D45544849D0
:105680004E4720594F552057415348204F4E4345D0
:105690002041205745454B3B4C41554E4452592ED5
:1056A0003B434152293B48414952063B4B495443F5
:1056B00048454E20464C4F4F520400000000000069
:1056C0000000000000000000000000004E414D45B9
:1056D00020534F4D455448494E472054484154208B
:1056E00048415320544F204452593B434C4F544857
:1056F0004553333B5041494E54173B484149520EA4
:105700003B4E41494C20504F4C495348043B544F69
:1057100057454C530200000000000000000000004C
:10572000000000004E414D4520534F4D455448491F
:105730004E4720594F55204252494E472042494E2C
:105740004F43554C41525320544F205741544348E6
:105750003B53504F5254494E47204556454E5442B4
:105760003B4249524453173B4F50455241073B433C
:105770004F4E434552540200000000004E414D453B
:1057800020534F4D454F4E452046414D4F555320D8
:1057900057484F5345204C415354204E414D4520CE
:1057A000495320224D415258223B47524F554348BE
:1057B0004F353B4B41524C1A3B484152504F0E3BE8
:1057C00052494348415244053B434849434F020034
:1057D000000000004E414D4520534F4D455448496F
:1057E0004E472050454F504C4520505554204F4E69
:1057F00020425245414B4641535420434552454176
:105800004C3B4D494C4B313B5355474152203B4259
:10581000414E414E41530D3B535452415742455224
:105820005249455304000000000000004E414D4520
:1058300020534F4D455448494E4720544841542029
:10584000594F552057494E442055503B434C4F43E8
:105850004B3D3B4D5553494320424F580D3B544F10
:1058600059530D3B575249535457415443480B0029
:105870000000000000000000000000000000000028
:10588000000000004E414D4520534F4D45544849BE
:105890004E4720594F55204D4541535552452049BB
:1058A0004E204D4541535552494E47204355505384
:1058B0003B464C4F5552333B53554741521E3B5785
:1058C00041544552093B4D494C4B07000000000034
:1058D0000000000000000000000000004E414D45A7
:1058E00020534F4D455448494E4720544841542079
:1058F000434F554C44205255494E20412044415974
:10590000204154205448452042454143483B5241A0
:10591000494E593B434C4F554453023B53554E421D
:1059200055524E0200000000000000000000000080
:10593000000000004E414D4520534F4D455448490D
:105940004E472054484154204B49445320434F5024
:10595000592046524F4D20544845495220465249FD
:10596000454E44533B484F4D45574F524B2F3B43B9
:105970004C4F54484553173B484149525354594C96
:10598000450B3B54414C4B0A000000004E414D4535
:1059900020534F4D455448494E472050454F504C99
:1059A0004520444F20494E204C4153205645474105
:1059B000533B47414D424C45583B57415443482087
:1059C00053484F5753083B4452494E4B023B4745BF
:1059D00054204D415252494544020000000000004D
:1059E000000000004E414D452041204B494E4420CF
:1059F0004F462053454520544841542050454F5070
:105A00004C45204541543B53554E464C4F5745520B
:105A1000473B50554D504B494E083B534553414D24
:105A200045083B504F505059050000000000000051
:105A30000000000000000000000000004E414D4545
:105A400020534F4D455448494E4720544841542017
:105A500046495245464947485445525320574541C7
:105A6000523B48454C4D45543A3B424F4F54531AD4
:105A70003B4F585947454E204D41534B083B5241EF
:105A8000494E434F41540600000000000000000052
:105A9000000000004E414D4520412022424F592731
:105AA00053204143544956495459222054484154A3
:105AB00020544F4D424F5953204C494B4520544F91
:105AC00020444F3B504C41592053504F525453386F
:105AD0003B434C494D42205452454553273B425588
:105AE000494C4420464F5254020000004E414D455F
:105AF00020534F4D455448494E4720535045434944
:105B00004649432054484154204D414B4553205968
:105B10004F5520495443483B494E53454354204236
:105B2000495445313B504F49534F4E204956591C1B
:105B30003B574F4F4C073B44525920534B494E045F
:105B4000000000004E414D4520414E204152544935
:105B5000434C45204F4620434C4F5448494E472024
:105B600050454F504C45204B4E49543B53574541AF
:105B70005445524D3B53434152460A3B4D495454C0
:105B8000454E53043B534F434B5304000000000069
:105B90000000000000000000000000004E414D45E4
:105BA00020534F4D455448494E4720574849434894
:105BB00020434F4D455320494E205457454C5645A0
:105BC000533B45474753513B444F4E5554530A3B73
:105BD000434F4F4B494553030000000000000000B5
:105BE00000000000000000000000000000000000B5
:105BF000000000004E414D4520534F4D454F4E454E
:105C0000204F5220534F4D455448494E4720544849
:105C10004154204841532057494E47533B42495233
:105C2000442D3B414952504C414E45113B414E475A
:105C3000454C103B425554544552464C59073B5035
:105C40004547415355530600000000004E414D4565
:105C5000204120524F4F4D2050454F504C4520463B
:105C600052455155454E544C5920414444204F4EC5
:105C700020544F204120484F5553453B44454E2F1B
:105C80003B424544524F4F4D223B42415448524FB4
:105C90004F4D063B504154494F06000000000000A4
:105CA000000000004E414D4520534F4D455448499A
:105CB0004E4720594F552046494E4420494E2041D9
:105CC0002042414259204E5552534552593B43526E
:105CD0004942443B444941504552530A3B544F5971
:105CE000530A3B42414259073B4348414E47494EC4
:105CF00047205441424C4502000000004E414D45B2
:105D000020534F4D455448494E4720544841542054
:105D1000594F5520444F20464F5220414E20555058
:105D20005345542053544F4D4143483B414E5441F9
:105D3000434944543B534F4441093B4D494C4B026A
:105D40003B4245440200000000000000000000004B
:105D5000000000004E414D4520534F4D45544849E9
:105D60004E472054484154204745545320544852EC
:105D70004F574E20425920414E204154484C4554E3
:105D8000453B42414C4C4B3B4A4156454C494E0CDD
:105D90003B4449534355530A3B53484F5450555481
:105DA0000300000000000000000000004E414D45CF
:105DB00020534F4D455448494E47204B49445320AA
:105DC0004C4541564520414C4C204F56455220549D
:105DD000484520484F5553453B544F59534D3B433D
:105DE0004C4F54484553103B53484F4553043B4692
:105DF0004F4F4402000000000000000000000000BF
:105E0000000000004E414D4520534F4D4554484938
:105E10004E4720594F552053455256452057495417
:105E20004820464953483B4348495053233B54413B
:105E300052544152205341554345223B4C454D4F0E
:105E40004E0C3B434F4C45534C415707000000005C
:105E500000000000000000000000000054454C4C11
:105E6000204D452041205741592050454F504C4529
:105E700020544F4C442054494D45204245464F52F2
:105E80004520434C4F434B53202620574154434811
:105E900045533B53554E4449414C323B5354415278
:105EA000532E3B484F5552474C415353030000007B
:105EB000000000004E414D452041205354415445BF
:105EC00020544841542047455453204D414E5920B9
:105ED000544F5552495354533B43414C49464F52FA
:105EE0004E4941273B464C4F52494441243B48418F
:105EF000574149490B3B4E455720594F524B0600DD
:105F00000000000000000000000000004E414D4570
:105F10002041204349545920494E20415553545261
:105F2000414C49413B5359444E4559493B4D454CE1
:105F3000424F55524E45153B5045525448033B4342
:105F4000414E424552524102000000000000000054
:105F50000000000000000000000000000000000041
:105F6000000000004E414D45204120574159205925
:105F70004F552043414E2054454C4C2054484154E9
:105F800020464F4F442048415320474F4E45204222
:105F900041443B534D454C4C4A3B4D4F4C44103BC8
:105FA000434F4C4F52063B544153544504000000AC
:105FB00000000000000000000000000057484154AD
:105FC000204252454544204F4620444F47205343EA
:105FD0004152455320594F5520544845204D4F5369
:105FE000543F3B5049542042554C4C353B444F4262
:105FF00045524D414E233B4745524D414E2053485B
:10600000455048455244053B53484F570300000054
:1060100000000000574845524520444F20594F5535
:10602000204B45455020594F55522053554E474C13
:1060300041535345533F3B434152353B50555253D7
:10604000451F3B48454144083B53484952540300CF
:106050000000000000000000000000000000000040
:106060000000000000000000000000004E414D450F
:1060700020534F4D455448494E47205448415427DA
:10608000532045415349455220544F20444F2057F7
:1060900048454E20495427532051554945543B52B9
:1060A0004541443C3B534C454550591A3B5354558C
:1060B00044590A3B5448494E4B030000000000007D
:1060C000000000004E414D45204120434F554E54A5
:1060D000525920574954482041204855474520509F
:1060E0004F50554C4154494F4E3B4348494E414611
:1060F0003B494E4449410E3B5553083B4A415041B0
:106100004E0600000000000000000000000000003B
:106110000000000000000000000000004E414D455E
:10612000204120465255495420464C41564F524535
:10613000442049434520435245414D3B535452412D
:106140005742455252593F3B5045414348103B430B
:106150004845525259083B4F52414E4745040000B2
:10616000000000000000000000000000000000002F
:10617000000000005748415427532054484520460A
:1061800049525354205245414C20574F52442054B9
:1061900048415420424142494553204C4541524ECA
:1061A00020544F205341593F3B4D414D412E3B44DC
:1061B000414441203B4E4F0E3B42594520425945F8
:1061C0000300000000000000000000004E414D45AB
:1061D000204120464F4F4420544841542041204301
:1061E0004F4F4B2053414D504C4553205748494C3D
:1061F00045204954275320434F4F4B494E473B536B
:10620000415543452F3B534F5550293B4348494C3B
:1062100049073B5350414748455454490300000047
:10622000000000004E414D452041204B494E442086
:106230004F46205448494E47204120574F4D414E2C
:10624000204255595320544F204348454552204839
:10625000455253454C462055503B434C4F544845BE
:1062600053503B4A4557454C5259063B464C4F57B5
:10627000455253053B464F4F440300004E414D45A8
:1062800020534F4D455448494E47205448415420CF
:1062900050454F504C452052494E53453B4841498B
:1062A000522D3B444953484553203B4C41554E44A5
:1062B00052590C3B4D4F5554480600000000000059
:1062C00000000000000000000000000000000000CE
:1062D000000000004E414D45204120534F5556458A
:1062E0004E495220594F552050555243484153452D
:1062F0002041542041204241534542414C4C2047CB
:10630000414D453B50454E4E414E54303B4341502C
:10631000263B42414C4C053B50524F4752414D04A5
:106320000000000000000000000000004E414D454C
:1063300020534F4D455448494E4720594F55274407
:106340002046494E44204F4E205448452042454166
:1063500043483B53414E44343B5348454C4C531CFB
:106360003B50454F504C45053B544F57454C53030C
:10637000000000000000000000000000000000001D
:10638000000000004E414D45204120504F535345E1
:106390005353494F4E20534F4D452050454F504C7D
:1063A0004520574F554C44204C494B4520544F20D5
:1063B00042452042555249454420574954483B4A9A
:1063C0004557454C52593D3B4D4F4E4559143B4363
:1063D0004152083B50455406000000004E414D45D7
:1063E00020534F4D455448494E472050454F504C3F
:1063F0004520505259204F50454E3B43414E273B7C
:106400004A41521E3B444F4F52083B57494E444F5E
:1064100057063B5348454C4C46495348033B454E71
:1064200056454C4F5045030000000000000000009E
:10643000000000004E414D45204120504C41434555
:106440002057484552452050454F504C4520444F19
:106450002041204C4F54204F462052454144494E44
:10646000473B4C494252415259463B424544524FA8
:106470004F4D0C3B42415448524F4F4D083B534304
:10648000484F4F4C05000000000000004E414D45B4
:1064900020412056454849434C4520544841542703
:1064A00053205045524D495454454420544F205395
:1064B000504545443B504F4C4943452043415229A8
:1064C0003B414D42554C414E4345283B4649524580
:1064D00020454E47494E450B3B52414345204341E1
:1064E000520400004E414D4520534F4D45544849FC
:1064F0004E47205448415420495320544F57454457
:106500003B4341524A3B424F4154113B5452414953
:106510004C4552053B574154455220534B49455237
:106520000200000000000000000000000000000069
:106530000000000000000000000000004E414D453A
:1065400020534F4D455448494E472054484154200C
:1065500041204D4F544F524359434C4953542057B7
:10656000454152533B48454C4D4554503B4A4143AD
:106570004B45540E3B474C4F564553033B474F4703
:10658000474C4553020000000000000000000000DE
:10659000000000004E414D4520534F4D45544849A1
:1065A0004E4720594F5520464F4355533B43414D8D
:1065B000455241533B42494E4F43554C4152530A79
:1065C0003B45594553043B54454C4553434F504577
:1065D00002000000000000000000000000000000B9
:1065E0000000000000000000000000004E414D458A
:1065F00020534F4D455448494E472050454F504C2D
:10660000452050415420544845495220504F434B57
:1066100045545320544F2046494E443B4B45595313
:106620004C3B57414C4C4554093B4D4F4E45590747
:106630003B50454E0200000000000000000000003A
:10664000000000004E414D4520534F4D45544849F0
:106650004E4720574F4D454E204841564520484112
:106660004420544F20464947485420544F2041432A
:1066700048494556453B524947485420544F2056B7
:106680004F54454E3B455155414C20504159123BCA
:106690004A4F425303000000000000004E414D45A8
:1066A00020414E2041525449434C45204F462043FF
:1066B0004C4F5448494E4720494E2057484943487B
:1066C0002050454F504C452048494445204D4F4EA1
:1066D00045593B425241213B534F434B1B3B53488F
:1066E0004F45103B434F41540E3B42454C5406002E
:1066F0000000000057484154204F4E45205448495F
:106700004E472041424F5554204120564143415469
:10671000494F4E20434F53545320544845204D4F2A
:106720005354204D4F4E45593F3B4C4F4447494EE3
:1067300047393B41495246415245133B464F4F442E
:10674000123B474153020000000000004E414D45FE
:1067500020534F4D455448494E472050454F504CCB
:10676000452043484557204F4E205748454E20541A
:10677000484559275245204E4552564F55533B46A2
:10678000494E4745524E41494C53473B47554D11A1
:106790003B50454E43494C083B4C495002000000D9
:1067A000000000004E414D4520534F4D455448498F
:1067B0004E4720594F55204F574E205448415420A2
:1067C000594F552043414E204C4F434B3B43415280
:1067D000493B484F555345103B53414645023B53B7
:1067E0005549544341534502000000000000000099
:1067F0000000000000000000000000004E414D4578
:106800002041204652554954205448415427532092
:106810004841524420544F20454154204E45415454
:106820004C593B57415445524D454C4F4E253B50DA
:10683000454143481D3B4F52414E4745123B47524D
:1068400041504546525549540500000000000000E3
:10685000000000004E414D452041204B494E442050
:106860004F4620414E494D414C2054484154204808
:1068700041532048454C504544204D414E205448FA
:10688000524F5547484F555420484953544F525939
:106890003B484F525345393B444F471C3B4D4F4EAD
:1068A0004B4559083B434F57020000004E414D45B0
:1068B000204120504C4143452057484552452050E7
:1068C000454F504C45205745415220574849544563
:1068D0003B484F53504954414C363B57454444493B
:1068E0004E47263B54454E4E495320434F55525434
:1068F0000600000000000000000000000000000092
:10690000000000004E414D45204120535045434971
:1069100046494320544F5050494E4720464F52203D
:10692000504945533B5748495050454420435245F0
:10693000414D353B4D4552494E475545153B494321
:106940004520435245414D113B4352554D420200B3
:106950000000000000000000000000004E414D4516
:1069600020534F4D455448494E47204D454E2042F7
:106970004F52524F572046524F4D204541434820D9
:106980004F544845523B544F4F4C532C3B4D4F4E68
:106990004559203B54494553073B434152043B4C26
:1069A00041574E204D4F574552043B434F4D4202F5
:1069B000000000004E414D4520412053504F52549D
:1069C00020594F55204D555354204841564520419C
:1069D000205241435155455420544F20504C415969
:1069E0003B54454E4E49535C3B52414351554554EF
:1069F00042414C4C053B4241444D494E544F4E039D
:106A00000000000000000000000000005748415452
:106A100020444F20524943482050454F504C452078
:106A2000574F5252592041424F55543F3B4D4F4EC4
:106A30004559313B5441584553103B5354415455EB
:106A400053073B524F4242455259053B4845414C42
:106A50005448033B53544F434B204D41524B4554F4
:106A6000030000004E414D4520412053504F5254E9
:106A70002041204C4F54204F462050454F504C450C
:106A800020424554204F4E3B484F525345205241DF
:106A900043494E47423B464F4F5442414C4C1B3BAF
:106AA000424F58494E47033B444F472052414349C8
:106AB0004E47030000000000000000004E414D451D
:106AC00020534F4D455448494E4720504152454E62
:106AD00054532054454C4C204B49445320544F2090
:106AE000444F204D4F52452051554945544C593B38
:106AF000504C41593F3B4C495354454E20544F2034
:106B00004D55534943123B54414C4B0B3B4541546B
:106B1000060000004E414D4520534F4D4554484915
:106B20004E47205448415420434F4E5441494E5300
:106B3000204341464645494E453B434F4646454521
:106B40004D3B534F44410E3B544541053B43484F59
:106B5000434F4C4154450400000000000000000079
:106B60000000000000000000000000004E414D4504
:106B700020534F4D455448494E47204D4F544845AA
:106B800052532053454E4420544F205448454952B7
:106B9000204B49445320494E2043414D503B464FE2
:106BA0004F44433B4C4554544552530B3B4D4F4E81
:106BB00045590B3B434C4F544845530800000000D7
:106BC000000000004E414D4520414E204F434341BF
:106BD00053494F4E2054484154204D494748542072
:106BE00042452053504F494C454420425920524180
:106BF000494E3B5049434E4943473B42414C4C2050
:106C000047414D45073B504152414445073B57459D
:106C10004444494E47070000000000004E414D45E6
:106C200020534F4D455448494E472054484154271E
:106C30005320444953415354524F555320464F52C9
:106C40002043524F50533B434F4C44223B494E53F9
:106C500045435453213B44524F55474854113B48F8
:106C600041494C0B00000000000000000000000043
:106C7000000000004E414D4520534F4D45544849BA
:106C80004E4720574F4D454E2053415920544841BF
:106C90005420414C4C20574F4D454E204C494B45BC
:106CA00020544F20444F3B53484F503F3B54414C9E
:106CB0004B0E3B454154083B4841495220444F4EFE
:106CC0004504000000000000000000004E414D455A
:106CD00020534F4D455448494E472050454F504C46
:106CE00045205249444520464F52204120544852A5
:106CF000494C4C3B524F4C4C455220434F4153540E
:106D00004552593B4D4F544F524359434C45053B17
:106D100046455252495320574845454C0200000011
:106D2000000000004E414D45204120464F4F442079
:106D3000594F5520454154204F4E20435241434B1B
:106D40004552533B434845455345543B5045414EBE
:106D50005554204255545445520C3B5341524449DA
:106D60004E4553020000000000000000000000003B
:106D70000000000000000000000000004E414D45F2
:106D8000204120504C414345205748455245205012
:106D90004F50434F524E20495320534F4C443B4D8C
:106DA0004F564945563B42414C4C5041524B063B95
:106DB0004341524E4956414C033B4349524355537C
:106DC00002000000000000000000000000000000C1
:106DD000000000004E414D4520534F4D4554484959
:106DE0004E4720544841542043414E204252494E80
:106DF00047204241434B205350454349414C204D8D
:106E0000454D4F524945533B534F4E472C3B5049FC
:106E100043545552451D3B4652414752414E5345FE
:106E2000063B4C4554544552020000004E414D452E
:106E300020534F4D455448494E4720534F4C442012
:106E40005448524F554748204D41494C204F5244D9
:106E50004552204144533B434C4F544845532D3BEE
:106E6000424F4F4B530E3B5245434F5244530B3B03
:106E70004449455420504C414E530400000000004A
:106E8000000000004E414D4520534F4D45544849A8
:106E90004E4720594F5520505554204F4E204120E9
:106EA000424147454C3B435245414D2043484545AF
:106EB0005345563B4C4F58053B425554544552039D
:106EC0003B4A414D030000000000000000000000AC
:106ED0000000000000000000000000004E414D4591
:106EE00020534F4D455448494E4720594F55205344
:106EF000454520494E534944452041204C41554E7B
:106F000044524F4D41543B5741534845524E3B44E8
:106F100052594552073B4348414E4745204D414356
:106F200048494E45063B434C4F54484553040000E6
:106F3000000000004E414D4520534F4D45544849F7
:106F40004E472047524F434552592053544F5245C4
:106F50005320474554204652455348204441494C0C
:106F6000593B4252454144323B4D494C4B173B50F3
:106F7000524F44554345143B4D45415404000000D5
:106F80000000000000000000000000004E414D45E0
:106F900020534F4D455448494E4720594F55205492
:106FA00055434B20494E3B5348495254443B534868
:106FB00045455453113B4348494C4452454E0D00FE
:106FC00000000000000000000000000000000000C1
:106FD00000000000000000000000000000000000B1
:106FE000000000004E414D4520534F4D4554484947
:106FF0004E47205448415420484153204120435299
:107000005553543B504945453B50495A5A410F3B13
:1070100042524541440D3B45415254480300000053
:107020000000000000000000000000000000000060
:107030000000000000000000000000004E414D452F
:1070400020534F4D455448494E4720544841542001
:10705000434F4D455320494E20464C414B45533BF1
:1070600043455245414C2F3B534E4F572E3B534FB8
:107070004150043B44414E445255464602000000F4
:107080000000000000000000000000000000000000
:10709000000000004E414D4520534F4D4554484996
:1070A0004E4720535045434946494320594F5527A1
:1070B00044204245204558434954454420544F20DC
:1070C00053454520494E20544845204F4345414EA5
:1070D0003B5748414C45323B534841524B133B448C
:1070E0004F4C5048494E1100000000004E414D45A4
:1070F00020534F4D455448494E472050454F504C22
:10710000452043525920494E544F3B48414E444B31
:10711000455243484945462E3B5449535355451C17
:107120003B50494C4C4F570B000000000000000042
:10713000000000000000000000000000000000004F
:10714000000000004E414D4520534F4D45544849E5
:107150004E472050454F504C4520534B49503B4DD6
:1071600045414C534D3B524F5045073B5343484FCD
:107170004F4C073B43485552434802000000000073
:1071800000000000000000000000000000000000FF
:107190000000000000000000000000004E414D45CE
:1071A0002041204B494E44204F46204255494C44F3
:1071B000494E47205448415420484153204D414EA8
:1071C00059204245445320494E2049543B484F538F
:1071D000504954414C363B484F54454C253B444F55
:1071E000524D49544F5259063B4241525241434B32
:1071F000530300004E414D4520414E204143544928
:10720000564954592054484154204255524E532017
:1072100041204C4F54204F462043414C4F5249454A
:10722000533B52554E4E494E47263B5357494D4DC1
:10723000494E47183B54454E4E4953093B41455230
:107240004F42494353070000000000004E414D45A6
:10725000204120465255495420534552564544201A
:10726000494E20435245414D3B53545241574245AC
:1072700052524945533A3B50454143484553213BBF
:107280004348455252494553043B42414E414E41C9
:1072900053023B424C554542455252494553020028
:1072A000000000004E414D45204120534F555243B0
:1072B00045204F4620454E455247592050454F5096
:1072C0004C452055534544204245464F5245204F9A
:1072D000494C3B434F414C1B3B574F4F44193B5785
:1072E00041544552113B57494E440A0000000000EA
:1072F0000000000000000000000000001000050079
:107300000100020002000200020003000400050068
:107310000600070008000200020002000200090047
:10732000020002000200020002000B000C000D002F
:107330000E000F0010000200020002000200020016
:1073400002000200020002001300140013001400E7
:1073500015001600170018000200020002000200CB
:1073600002000200020002001B001C001D001E00A3
:107370000B000C001F0020000200020002000200AF
:1073800021000200020002000200020002000200CE
:1073900002000200020002000200020002002500BA
:1073A000040004000100110012000900020019008D
:1073B0001A00020021002200230024000000000027
:1073C000000000000400020000002600270000006A
:1073D0002A002B002C002D000400020000002600D3
:1073E0002700000000002E002F0000000400020013
:1073F0000000280029000000300031003200330076
:1074000004000200000028002900000000003400F1
:107410003500000004000200360037003800390053
:1074200042004300440045000400020036003A00D8
:107430003B003900420046004700450004000200BE
:107440003C003D003E003F00480049004A004B0020
:10745000040002003C00400041003F0048004C0096
:107460004D004B001E0004004E004F0050004F0026
:1074700050004F0050005100520052005200520084
:10748000520052005200520052005200520052006C
:107490005200520053004F0050004F0050004F0068
:1074A000500054005600570058005700580057002D
:1074B000580059000200020002000200020002000F
:1074C00002000200020002000200020002000200AC
:1074D0005A005700580057005800570058005B00EA
:1074E00056005700580057005800570058005900E0
:1074F000020002000200020002000200020002007C
:107500000200020002000200020002005A005700BE
:10751000580057005800570058005B005C005700A7
:10752000580057005800570058005D005E005E008C
:107530005E005E005E005E005E005E005E005E005B
:107540005E005E005E005E005F005700580057005E
:1075500058005700580060000400030063006400F6
:10756000650066006700680069006A006B006C00D7
:107570006D006E00050305050505050305050505F8
:1075800005030505050505030505050505030505B1
:1075900005050503050505050503050505050503A1
:1075A000050505050503056161610503616161610B
:1075B0000561616161616161616161616161616117
:1075C00061616161616161616161616161616161AB
:1075D000616161616161616161616161616161619B
:1075E000616161616161616161616161616161618B
:1075F000616161616161616161616161616161617B
:10760000616161616161616161616161616161616A
:107610006161616161616161616161613F3F3F61C0
:1076200061613F703F6161613F703F6161613F70C7
:107630003F6161616161616161616161616161615C
:107640006161616161616161616161616161613F4C
:107650003F3F6161613F703F6161613F703F6161C8
:10766000613F703F6161616161616161616161613F
:107670006161616161616161616161613F3F3F3F82
:107680003F3F3F70707070703F3F3F3F3F3F6161D1
:1076900061616161616161616161616161616161DA
:1076A0006161616161616161616161613F3F3F3F52
:1076B0003F3F70707070703F3F3F3F70703F613F61
:1076C00070703F61616161616161616161616161AE
:1076D0006161616161616161616161613F3F3F3F22
:1076E0003F3F3F70707070703F703F3F3F3F3F7053
:1076F0003F6161616161616161616161616161619C
:107700006161616161616161616161613F3F3F3FF1
:107710003F3F70707070703F3F3F3F3F3F3F616140
:107720006161616161616105050561616161050515
:107730006161616161056161616161616161616195
:107740006161616161616161616161616161616129
:1077500061616161610AE80A0A0A610A0A0A010AAA
:10776000610A0A0A010A610A0A0A0A0A61610A052B
:1077700005056161610A050A61616161610A616112
:10778000616161503F703F6161613F703F61616164
:107790003F703F6161613F703F6161613F70703F69
:1077A0006161613F70703F3F61613F707070616106
:1077B000613F3F3F6161613F703F6161613F703F89
:1077C0006161613F703F6161613F703F61613F7026
:1077D000703F3F3F70703F617070703F61613F3F2D
:1077E0003F61616161616161616161616161613FCD
:1077F000616161613F706161613F707061613F70A3
:10780000703F613F70703F3F3F70707070703F3FDE
:107810003F3F3F3F3F70703F616170703F6161610A
:10782000703F616161613F6161616161616161617D
:1078300061613F3F3F3F3F3F70707070703F3F3F1F
:107840003F3F3F3F3F703F6161613F703F3F3F3F80
:107850003F70707070703F703F3F3F3F3F703F61BF
:1078600061613F703F3F3F3F3F70707070703F3FBE
:107870003F3F3F3F6161616161613F3F61616161C4
:10788000703F616161613F3F61616161616161613F
:1078900061613F3F3F3F3F3F70707070703F3F3FBF
:1078A0003F3F3F3F61616161616161616161616150
:1078B00061616161616161616161616561616161B4
:1078C000656561616165656561616565650A6165DB
:1078D0000A0A0A0A616161616161616161616161F4
:1078E0006161616161616565616161616565656570
:1078F00061616565656565616565650A65650A0A55
:107900000A0A0A653F3F3F3F3F3F3F70707070700B
:107910003F703F3F3F3F3F703F6161613F703F615C
:1079200061613F703F6161613F703F3F3F3F3F702A
:10793000707070703F3F3F3F3F3F70707070703F9E
:107940003F3F3F3F3F3F61616161616161616161F3
:1079500061616161616161613F3F61616161703F6E
:10796000616161613F3F3F6161613F703F616161A2
:107970003F703F6161613F703F6161613F703F6196
:1079800061613F703F6161613F703F6161613F7064
:107990003F6161616161613F3F3F6161613F703F94
:1079A0006161613F703F6161613F703F6161613F53
:1079B000703F6161613F703F6161613F703F616134
:1079C000613F703F3F3F3F3F3F3F3F70707070707F
:1079D0003F703F3F3F703F703F61613F3F703F618D
:1079E00061613F703F6161613F703F6161613F7004
:1079F0003F6161616161616161613F3F61616161DD
:107A000070703F6161613F70703F6161613F707094
:107A10003F6161613F70703F6161613F703F6161D3
:107A2000613F703F610AE80A0A0A610A0A0A010A0C
:107A3000610A0A0A010A610A0A0A0A0A61610A0A53
:107A4000050A6161610A0A0A61616161610A616135
:107A500061616150E80A0A0A0A650A0A0A0A0A0A02
:107A60000A0A0A0A0A0A0A0A0A0A0A0A0A0A0A0A76
:107A70000A610A0A0A0A0A610A0A0A0A0A610A0A61
:107A80000A0A0A503F703F3F3F3F3F703F616161CC
:107A90003F703F6161613F703F6161613F703F6175
:107AA00061613F703F6161613F703F6161613F3F74
:107AB0003F6161613F3F616161616161616161611C
:107AC00061616161616161616161616161616161A6
:107AD0006161616161616161616161616161616196
:107AE000616161613F703F3F3F3F3F703F61616156
:107AF0003F703F6161613F703F6161613F703F6115
:107B000061613F703F3F3F3F3F70707070703F3F1B
:107B10003F3F3F3F3F3F6161616161616161616121
:107B20006161616161616161616161616161616145
:107B300061613F3F3F3F3F3F70707070703F3F3F1C
:107B40003F3F3F3F3F703F6161613F703F61616117
:107B50003F703F6161613F703F6161613F703F61B4
:107B6000613F3F703F3F3F703F70707070703F3FAC
:107B70003F3F3F3F6161613F703F6161613F703FE7
:107B800061613F70703F613F70703F613F70703F57
:107B9000616170703F6161613F3F6161616161611D
:107BA00061616161616161616161616161616161C5
:107BB00061616161616161616161616161616161B5
:107BC0006161056161616161050361616161050375
:107BD0000561616161616150505061615050505068
:107BE0006150505050506150505050505050505073
:107BF0005050505050505250505050505250505081
:107C000050505250FF00FF00FF50500000005050F5
:107C10005000FF0050505050525050FF52505250A0
:107C2000FFFF5050525052525050525052525250E8
:107C300052505052505061616161505050506161DA
:107C4000505050505061505050505050FF50525072
:107C500050505250525050055250505205055050FD
:107C60005005050561616161616161616161616129
:107C700061616161616161616161616161616161F4
:107C800061616161616161056161616105056161F8
:107C9000610505050503050505050503050505053C
:107CA000050305050505050305050505050305058A
:107CB0000505050305050101050305010101050190
:107CC0000101010105030505050505030505050578
:107CD000050305050505050305050505050305055A
:107CE000050501030505050501010105050501015E
:107CF0000101010505030505050505030505050544
:107D00000503050505050503050505050503050529
:107D10000505050305052E2E0503052E2E2E052E21
:107D20002E2E2E2E05030505050505030505050563
:107D300005030505050505030505050505030505F9
:107D400005052E03050505052E2E2E0505052E2EEF
:107D50002E2E2E0505030505050505030505050160
:107D600005030505050105030505010105030505D5
:107D700001010503050501010503050501010503D1
:107D800005050101010101AFAFAF0101AF6BAFAF5D
:107D900001AFAFAFAFAF01AFAFAFAFA6AFAFAFAF58
:107DA000AFA6AFAFAFAFAFAF01AFAFAF050501014A
:107DB000AFAFAF05AFAFAF010101AF6BAFAF010127
:107DC000AFAFAFAFAF01AFAFAFAFAF01AFAFAFAF1F
:107DD000AFAFAFAFAFAFAFAF05AFAFAFAF01AFAF0B
:107DE000AFAF0101050305050505010305050505FF
:107DF0000103050505050103050505050101050547
:107E0000050501010505050501010505050501013A
:107E100005050505010101AFAFAF0101AF6BAFAFC4
:107E200001AFAFAFAFAF01AFAFAFAFA6AFAFAFAFC7
:107E3000AFA6AFAFAFAFAFAF05AFAFAF05050503AF
:107E4000AFAFAF05AFAFAF010101AF6BAFAF010196
:107E5000AFAFAFAFAF01AFAFAFAFAF01AFAFAFAF8E
:107E6000AFAFAFAFAFAFAFAF05AFAFAFAF05AFAF76
:107E7000AFAF050505030505050505030505052E39
:107E800005030505052E050305052E2E050305052D
:107E90002E2E050305052E2E050305052E2E0503A2
:107EA00005052E2E2E2E2EAFAFAF2E2EAF0AAFAF62
:107EB0002EAFAFAFAFAF2EAFAFAFAFA6AFAFAFAFDD
:107EC000AFA6AFAFAFAFAFAF2EAFAFAF05052E2EA2
:107ED000AFAFAF05AFAFAF2E2E2EAF0AAFAF2E2E86
:107EE000AFAFAFAFAF2EAFAFAFAFAF2EAFAFAFAFA4
:107EF000AFAFAFAFAFAFAFAF05AFAFAFAF2EAFAFBD
:107F0000AFAF2E2E0503050505052E030505050556
:107F10002E03050505052E03050505052E2E050571
:107F200005052E2E050505052E2E050505052E2E0B
:107F3000050505052E2E2EAFAFAF2E2EAF0AAFAF23
:107F40002EAFAFAFAFAF2EAFAFAFAFA6AFAFAFAF4C
:107F5000AFA6AFAFAFAFAFAF05AFAFAF050505038E
:107F6000AFAFAF05AFAFAF2E2E2EAF0AAFAF2E2EF5
:107F7000AFAFAFAFAF2EAFAFAFAFAF2EAFAFAFAF13
:107F8000AFAFAFAFAFAFAFAF05AFAFAFAF05AFAF55
:107F9000AFAF050505030505050505030505054006
:107FA0000503054040800503408080800503408034
:107FB00080800503408080400503408080400503A9
:107FC00040808040050305AFAFAF40404005AFAFF4
:107FD00080808040AFAF8080808040408080808003
:107FE000AFAF808080AFAFAF808080404040808066
:107FF00040808040AFAFAF050505AFAF05404040C2
:10800000AFAF40808080404080808080AFAF808074
:108010008080AFAFAF8080804040408080804080D3
:10802000804080800503050505054003050505051D
:1080300080404005050580808040050580808040A7
:108040000505408080400505408080400505408052
:1080500080400505050305AFAFAF40404005AFAF19
:1080600080808040AFAF808080AF40408080AFAFE5
:10807000808080AFAFAF8080804040408080804073
:1080800080408080AFAFAF050505AFAF05404040F1
:10809000AFAF408080804040AF8080808080AFAFB5
:1080A00080808080AFAFAF80808040404080808003
:1080B00040804080050305050505050305050510FD
:1080C00005030510101805031018181805031018DB
:1080D00018180503101818100503101818100503B8
:1080E00010181810050305AFAFAF10101005AFAF93
:1080F00018181810AFAF18181818101018181818EA
:10810000AFAF181818AFAFAF181818101010181814
:1081100010181810AFAFAF050505AFAF0510101060
:10812000AFAF10181818101018181818AFAF18188B
:108130001818AFAFAF18181810101018181810181A
:108140001810181805030505050510030505050594
:10815000181010050505181818100505181818101E
:108160000505101818100505101818100505101829
:1081700018100505050305AFAFAF10101005AFAF20
:1081800018181810AFAF181818AF10101818AFAF94
:10819000181818AFAFAF18181810101018181810BA
:1081A00018101818AFAFAF050505AFAF05101010C8
:1081B000AFAF101818181010AF1818181818AFAF64
:1081C00018181818AFAFAF18181810101018181882
:1081D000101810180503408080400503408080403F
:1081E00005034080804005030540808005030505A8
:1081F0004040050305050540050305050540050349
:10820000050505408040808040804080804080801F
:10821000808040808080804080808080408080801E
:10822000808080808080808080808080808080804E
:10823000808080808040808040808080408080403E
:1082400080808040808080808080408080808080AE
:10825000804080808080808080808080808080805E
:1082600080808080408080400505408080400505FA
:10827000408080400505808040050505404005059B
:1082800005054003050505054003050505054003F3
:1082900005050505408080408080408080408080CA
:1082A000808040808080804080808080408080808E
:1082B00080808080808080808080808080808080BE
:1082C00080808080808040808040808040808040AE
:1082D000808080408080808080804080808080801E
:1082E00080408080808080808080808080808080CE
:1082F00080808080050310181810050310181810CE
:1083000005031018181005030510181805030505B6
:1083100010100503050505100503050505100503E7
:10832000050505101810181810181018181018182E
:1083300018181018181818101818181810181818D5
:1083400018181818181818181818181818181818AD
:1083500018181818181018181018181810181810BD
:10836000181818101818181818181018181818189D
:108370001810181818181818181818181818181885
:1083800018181818101818100505101818100505D9
:10839000101818100505181810050505101005050A
:1083A0000505100305050505100305050505100362
:1083B00005050505101818101818101818101818A9
:1083C0001818101818181810181818181018181845
:1083D000181818181818181818181818181818181D
:1083E000181818181818101818101818101818102D
:1083F000181818101818181818181018181818180D
:1084000018101818181818181818181818181818F4
:1084100018181818050A0A0A0A0A0A0A0A0A0A0A89
:10842000050A0A0A0A0A05A5A5A5A5A505A5A5A5E3
:10843000A5A505A5A5A5A5A505A5A5A5A5A505A5CC
:10844000A5A5A5A50A0A0A0A0A0A0A0A0A0A0A0A20
:108450000A0A0A0A0A0AA3A3A3A3A3A3A3A3A3A382
:10846000A3A3A3A3A3A3A3A3A3A3A3A3A3A3A3A3DC
:10847000A3A3A3A30A0A0A0A0A0A0A0A0A0A0A0AF8
:108480000A0A0A0A0A0AA5A5A5A5A5A5A5A5A5A53E
:10849000A5A5A5A5A5A5A5A5A5A5A5A5A5A5A5A58C
:1084A000A5A5A5A50A0A0A0A0A0A0A0A0A0A0A0AC0
:1084B0000A0A0A0A0A0A4F4F4F4F4F4F4F4F4F4F6A
:1084C0004F4F4F4F616161614F4F616161614F4F2C
:1084D000616161610A0A0A0A0A0A0A0A0A0A0A0AA0
:1084E0000A0A0A0A0A0A4F4F4F4F4F4F4F4F4F4F3A
:1084F0004F4F616161616161616161616161616190
:10850000616161610A0A0A0A0A0A0A0A0A0A0A0A6F
:108510000A0A0A0A0A0A4F4F4F4F4F4F4F4F4F4F09
:108520004F4F616161614F4F616161614F4F6161A7
:1085300061614F4F0A0A0A0A0A050A0A0A0A0A0A68
:108540000A0A0A0A0A05A3A3A3A3A305A3A3A3A334
:10855000A305A3A3A3A3A305A3A3A3A3A305A3A3C5
:10856000A3A3A305BFBFBFBFBFBFBFBFBFBFBFBF29
:10857000BFBFB5BFBFBFBFBFBFB5BFBFBFB5BFBF29
:10858000BFBFBFBFB5BFBFBFBFBFBFBFBFBFBFBF05
:10859000BFBFBFBFBFA5A5A5A5A5BFA5A5A5A5A5EF
:1085A000BFA5A5A5A5A5BFA5A5A5A5A5BFA5A5A52D
:1085B000A5A5BFA5A5A5A5A5BFA5A5A5A5A5BFA51D
:1085C000A5A5A5A5A3A3A3A3A3A3A3A3A3A3A3A373
:1085D000A3A3A3A3A3A3A3A3A3A3A3A3A3A3A3A36B
:1085E000A3A3A3A3A3A3A3A3A3A3A3A3A3A3A3A35B
:1085F000A3A3A3A3A5A5A5A5A5A5A5A5A5A5A5A533
:10860000A5A5A5A5A5A5A5A5A5A5A5A5A5A5A5A51A
:10861000A5A5A5A5A5A5A5A5A5A5A5A5A5A5A5A50A
:10862000A5A5A5A54F4F616161614F4F6161616172
:108630004F4F616161614F4F616161614F4F616196
:1086400061614F4F616161614F4F616161614F4F86
:1086500061616161616161614F4F616161614F4F52
:10866000616161614F4F616161614F4F6161616142
:108670004F4F616161614F4F616161614F4F616156
:1086800061614F4FA3A3A3A3A3BFA3A3A3A3A3BFAE
:10869000A3A3A3A3A3BFA3A3A3A3A3BFA3A3A3A372
:1086A000A3BFA3A3A3A3A3BFA3A3A3A3A3BFA3A346
:1086B000A3A3A3BFBFA5A5A5A5A5BFA5A5A5A5A522
:1086C000BFA5A5A5A5A5BFA5A5A5A5A5BFA5A5A50C
:1086D000A5A5BFA5A5A5A5A5BFBFA5A5A5A5BFBFC8
:1086E000BFA5A5A54F4F616161614F4F6161616198
:1086F0004F4F616161614F4F616161614F4F6161D6
:1087000061614F4F616161614F4F4F4F4F4F4F4F0D
:108710004F4F4F4F61616161616161616161616191
:108720006161616161616161616161616161616139
:1087300061616161616161614F4F4F4F4F4F4F4FB9
:108740004F4F4F4F616161614F4F616161614F4FA9
:10875000616161614F4F616161614F4F6161616151
:108760004F4F616161614F4F4F4F4F4F4F4F4F4FD1
:108770004F4F4F4FA3A3A3A3A3BFA3A3A3A3A3BFE1
:10878000A3A3A3A3A3BFA3A3A3A3A3BFA3A3A3A381
:10879000A3BFA3A3A3A3A3BFA3A3A3A3BFBFA3A339
:1087A000A3BFBFBFE0C0E0E0E0E0E0C0E0E0E0E0A9
:1087B000E0C0E0E0E0E0E0C0E0E0E0E0E0C0E0E019
:1087C000E0E0E0C0E0E0E0E0E0C0E0E0E0E0E0C009
:1087D000E0E0E0E06161BF6161BF61BF6161BF6115
:1087E000BF6161BF61616161BF6161BF61BF6161A3
:1087F000BF61BF6161BF61616161BF6161BF61BF35
:108800006161BF61E0C0E0E0E0E0E0C0E0E0E0E046
:10881000E0C0E0E0E044E0C0E0E04444E0C0E04428
:108820004444E0C044444444E04444444444E044B8
:10883000444444E0E0C0E0444444444444444444A8
:10884000444444444444444444444444444444E04C
:10885000E0E044C0E0E0E0E0E0C0E0E0E0E0E0C014
:10886000E0E0E0E0444444E0E0E044444444444484
:10887000444444444444444444444444E0C0E04404
:108880004444E0C0E0E0E044E0C0E0E04444E0C054
:10889000E0444444E0C0E0E0E0E0E0C0E0E0E0E0EC
:1088A00044C0E0E0E0E04444E0E0E0E0444444E090
:1088B000E0E044444444E0E04444444444E044446C
:1088C000444444E0E044444444E044444444E0E05C
:1088D00044444444E0E044444444E0E044444444E8
:1088E000E0E044444444E0E044444444E0E0E04404
:1088F000444444E0E0C0E0E0E0E0E0C0E0E0E0E08C
:10890000E0C0E0E0E0E0E0C0E0E0E044E0C0E0E063
:108910004444E0C0E0444444E0C044444444E044AF
:10892000444444E0E0C044444444E044444444E01B
:1089300044444444E0E0444444E0E0E04444E0E0B3
:10894000E0E044C0E0E0E0E0E0C0E0E0E0E0E0C023
:10895000E0E0E0E0E044444444E0E0C04444444417
:10896000E0C044444444E0C044444444E0C044447F
:108970004444E0C044444444E0C044444444E044EB
:10898000444444E0E044444444E0E0444444444437
:10899000E0C044444444E0C0E0444444E0C0E0E07B
:1089A0004444E0C0E0E0E044E0C0E0E0E0E0E0C0FB
:1089B000E0E0E0E044444444E0E0444444E0E0E0FB
:1089C0004444E0E0E0E0444444E0E0E04444444423
:1089D0004444444444444444444444444444E0C03F
:1089E000E0444444E0C0E0E0E0E0E0C0E0E0E0E09B
:1089F000E0C0E0E0E044E0C0E04444444444444497
:108A00004444444444444444444444444444444426
:108A100044E0E0E0E044444444E04444444444E06E
:108A200044444444E0E0444444E0E0E04444E0E0C2
:108A3000E0E044C0E0E0E0E0E0C0E0E0E0E0E0C032
:108A4000E0E0E0E0616161616161616161AF6161CC
:108A5000AFAFAFAFAF61AFAFAFAFAFAFAFAFAFAF74
:108A6000AFAFAFAFAFAFAF61616161AF6161616186
:108A700061616161616161616161616161616161E6
:108A800061616161616161616161616161616161D6
:108A900061616161616161616161616161616161C6
:108AA000616161616161616161616161FF61616118
:108AB00061FFFFFF616161FFFFFF61616161FF6154
:108AC00061616161FF6161616161616161616161F8
:108AD000FF616161616161616161FFFF61FFFF6170
:108AE000FFFF61FFFF61FF6161FF616161616161C2
:108AF0006161616161616161616161616161616166
:108B00006161616161616161616161616161616155
:108B100061FF61FF6161FFFFFFFFFF6161FF61FFB7
:108B2000616161FF61FF6161FFFFFFFFFF6161FF45
:108B300061FF616161616161616161FF61616161E9
:108B400061FFFFFF6161FF616161616161FFFF6161
:108B50006161616161FF6161FFFFFF61616161618D
:108B6000FF616161616161616161FFFF6161FF617D
:108B7000FFFF6161FF61616161FF61616161FF61CF
:108B8000616161FF61616161FF6161FFFF61FF61BF
:108B900061FFFF6161616161616161FF61616161EB
:108BA000FF61FF616161FF61FF61616161FF61619F
:108BB0006161FF61FF61FF61FF6161FF616161FFF1
:108BC000FF61FF6161616161616161FFFF6161611D
:108BD00061FFFF61616161FF6161616161616161AB
:108BE0006161616161616161616161616161616175
:108BF000616161616161616161616161FF616161C7
:108C000061FF6161616161FF6161616161FF61617A
:108C1000616161FF6161616161FF61616161616108
:108C2000FF61616161616161616161FF61616161F8
:108C30006161FF6161616161FF6161616161FF614A
:108C400061616161FF6161616161FF61616161FF3A
:108C50006161616161616161616161616161616104
:108C600061FF61FF616161FFFFFF6161FFFFFFFF66
:108C7000FF6161FFFFFF616161FF61FF6161616130
:108C800061616161616161616161616161616161D4
:108C90006161FF6161616161FF616161FFFFFFFF10
:108CA000FF616161FF6161616161FF6161616161DA
:108CB00061616161616161616161616161616161A4
:108CC0006161616161616161616161616161616194
:108CD000616161FFFF61616161FFFF61616161FF6E
:108CE0006161616161616161616161616161616174
:108CF000616161616161616161616161FFFFFFFFEC
:108D0000FF616161616161616161616161616161B5
:108D10006161616161616161616161616161616143
:108D20006161616161616161616161616161616133
:108D3000616161616161616161FFFF61616161FF49
:108D4000FF61616161616161616161616161616175
:108D500061616161FF61616161FF61616161FF6129
:108D6000616161FF61616161FF61616161616161B7
:108D70006161616161616161616161FFFFFF616109
:108D8000FF616161FF61FF6161FFFF61FF61FF6181
:108D9000FF61FFFF6161FF61FF616161FF6161FF71
:108DA000FFFF61616161616161616161FF616161D9
:108DB00061FFFF6161616161FF6161616161FF612B
:108DC00061616161FF6161616161FF61616161FFB9
:108DD000FFFF616161616161616161FFFFFF61616D
:108DE000FF616161FF6161616161FF616161FFFF5D
:108DF000616161FF61616161FF6161616161FFFFEB
:108E0000FFFFFF6161616161616161FFFFFF61619E
:108E1000FF616161FF6161616161FF6161FFFFFF8E
:108E2000616161616161FF61FF616161FF6161FFBA
:108E3000FFFF6161616161616161616161FF616148
:108E40006161FFFF616161FF61FF6161FF6161FF5E
:108E50006161FFFFFFFFFF61616161FF616161614E
:108E600061FF6161616161616161FFFFFFFFFF613E
:108E7000FF6161616161FF6161616161FFFFFFFF2E
:108E8000616161616161FF61FF616161FF6161FF5A
:108E9000FFFF61616161616161616161FFFF61614A
:108EA00061FF61616161FF6161616161FFFFFFFFFE
:108EB0006161FF616161FF61FF616161FF6161FF8C
:108EC000FFFF6161616161616161FFFFFFFFFF6140
:108ED00061616161FF61616161FF61616161FF61A8
:108EE000616161FF6161616161FF6161616161FF98
:108EF0006161616161616161616161FFFFFF616188
:108F0000FF616161FF61FF616161FF6161FFFFFFFF
:108F10006161FF616161FF61FF616161FF6161FF2B
:108F2000FFFF616161616161616161FFFFFF61611B
:108F3000FF616161FF61FF616161FF6161FFFFFFCF
:108F4000FF6161616161FF61616161FF616161FF99
:108F5000FF61616161616161616161616161616163
:108F600061616161616161FFFF61616161FFFF6179
:108F7000616161616161616161FFFF61616161FF07
:108F8000FF61616161616161616161616161616133
:108F900061FFFF61616161FFFF6161616161616149
:108FA000616161FFFF61616161FFFF61616161FF9B
:108FB0006161616161616161616161616161FF6103
:108FC000616161FF61616161FF61616161FF6161B7
:108FD00061616161FF616161616161FF6161616145
:108FE0006161FF61616161616161616161616161D3
:108FF000616161616161FFFFFFFFFF61616161614B
:109000006161616161616161FFFFFFFFFF6161613A
:109010006161616161616161616161FF61616161A2
:109020006161FF616161616161FF616161616161F4
:10903000FF61616161FF61616161FF61616161FFA8
:109040006161616161616161616161FFFFFF616136
:10905000FF616161FF6161616161FF616161FFFFEA
:1090600061616161FF616161616161616161616152
:10907000FF61616161616161616161FFFFFF616168
:10908000FF616161FF61FF61FFFFFF61FF61FF61E0
:10909000FF61FF61FFFFFF61FF616161616161FF6E
:1090A000FFFF616161616161616161FFFFFF61619A
:1090B000FF616161FF61FF616161FF61FF6161618A
:1090C000FF61FFFFFFFFFF61FF616161FF61FF6102
:1090D0006161FF61616161616161FFFFFFFF61616A
:1090E000FF616161FF61FF616161FF61FFFFFFFF80
:1090F0006161FF616161FF61FF616161FF61FFFFAC
:10910000FFFF616161616161616161FFFFFF616139
:10911000FF616161FF61FF6161616161FF616161C7
:109120006161FF6161616161FF616161FF6161FFB7
:10913000FFFF6161616161616161FFFFFFFF61616B
:10914000FF616161FF61FF616161FF61FF616161F9
:10915000FF61FF616161FF61FF616161FF61FFFFAD
:10916000FFFF6161616161616161FFFFFFFFFF619D
:10917000FF6161616161FF6161616161FFFFFFFF2B
:109180006161FF6161616161FF6161616161FFFF57
:10919000FFFFFF61616161616161FFFFFFFFFF61CF
:1091A000FF6161616161FF6161616161FFFFFFFFFB
:1091B0006161FF6161616161FF6161616161FF61C5
:1091C0006161616161616161616161FFFFFF6161B5
:1091D000FF616161FF61FF6161616161FF61FFFFCB
:1091E000FF61FF616161FF61FF616161FF6161FFBB
:1091F000FFFFFF61616161616161FF616161FF6149
:10920000FF616161FF61FF616161FF61FFFFFFFF5E
:10921000FF61FF616161FF61FF616161FF61FF618A
:109220006161FF6161616161616161FFFFFF6161B6
:109230006161FF6161616161FF6161616161FF6144
:1092400061616161FF6161616161FF61616161FF34
:10925000FFFF616161616161616161616161FF6124
:1092600061616161FF6161616161FF6161616161B2
:10927000FF61FF616161FF61FF616161FF6161FF2A
:10928000FFFF6161616161616161FF616161FF6156
:10929000FF6161FF6161FF61FF616161FFFF61610A
:1092A0006161FF61FF616161FF6161FF6161FF6198
:1092B0006161FF61616161616161FF616161616162
:1092C000FF6161616161FF6161616161FF616161B4
:1092D0006161FF6161616161FF6161616161FFFF06
:1092E000FFFFFF61616161616161FF616161FF6158
:1092F000FFFF61FFFF61FF61FF61FF61FF6161616E
:10930000FF61FF616161FF61FF616161FF61FF6199
:109310006161FF61616161616161FF616161FF6163
:10932000FFFF6161FF61FF61FF61FF61FF6161FF3D
:10933000FF61FF616161FF61FF616161FF61FF6169
:109340006161FF6161616161616161FFFFFF616195
:10935000FF616161FF61FF616161FF61FF616161E7
:10936000FF61FF616161FF61FF616161FF6161FF39
:10937000FFFF6161616161616161FFFFFFFF616129
:10938000FF616161FF61FF616161FF61FFFFFFFFDD
:109390006161FF6161616161FF6161616161FF61E3
:1093A0006161616161616161616161FFFFFF6161D3
:1093B000FF616161FF61FF616161FF61FF61616187
:1093C000FF61FF61FF61FF61FF6161FF616161FF3B
:1093D000FF61FF61616161616161FFFFFFFF6161C9
:1093E000FF616161FF61FF616161FF61FFFFFFFF7D
:1093F0006161FF6161FF6161FF616161FF61FF6147
:109400006161FF6161616161616161FFFFFF6161D4
:10941000FF616161FF61FF616161616161FFFFFF88
:10942000616161616161FF61FF616161FF6161FFB4
:10943000FFFF6161616161616161FFFFFFFFFF61CA
:109440006161FF6161616161FF6161616161FF6132
:1094500061616161FF6161616161FF6161616161C0
:10946000FF616161616161616161FF616161FF6112
:10947000FF616161FF61FF616161FF61FF616161C6
:10948000FF61FF616161FF61FF616161FF6161FF18
:10949000FFFF6161616161616161FF616161FF6144
:1094A000FF616161FF61FF616161FF61FF61616196
:1094B000FF61FF616161FF6161FF61FF6161616186
:1094C000FF616161616161616161FF616161FF61B2
:1094D000FF616161FF61FF61FF61FF61FF61FF612A
:1094E000FF61FF61FF61FF61FF61FF61FF6161FF7C
:1094F00061FF6161616161616161FF616161FF6182
:10950000FF616161FF6161FF61FF61616161FF6135
:10951000616161FF61FF6161FF616161FF61FF6125
:109520006161FF61616161616161FF616161FF6151
:10953000FF616161FF61FF616161FF6161FF61FF67
:1095400061616161FF6161616161FF6161616161CF
:10955000FF616161616161616161FFFFFFFF6161E5
:10956000616161FF61616161FF61616161FF616111
:109570006161FF6161616161FF6161616161FFFF63
:10958000FFFF616161616161FF6161FFFFFF616117
:10959000FF616161FF61FF616161FF61FF616161A5
:1095A000FF61FFFFFFFFFF61FF616161FF61FF611D
:1095B0006161FF616161616161616161FFFF6161C1
:1095C00061FF6161FF61FF61FFFF61FFFF61FF619B
:1095D00061FFFF61FFFF61FF61FF6161FF61616129
:1095E000FFFF616161616161616161FFFF616161F3
:1095F000616161FF6161616161FF6161616161FF81
:10960000FF61616161FF6161616161FF616161FFD2
:10961000FF616161504C4159004F5054494F4E53C6
:109620000041424F5554005C203230313020464CCE
:109630005B56494F205A4156414E0057454C434FC7
:109640004D452E0A484F57204D414E592046414D19
:10965000494C494553204152450A504C4159494EC5
:109660004720544849532054494D453F00504C45EC
:109670004153452053454C4543542057484943489E
:109680000A434F4E54524F4C4C455220454143489B
:109690002046414D494C590A57494C4C2055534599
:1096A0002E0046414D494C49455300444F4E45001C
:1096B00046414D494C593A00464952535400000026
:1096C0005345434F4E440000544849524400000063
:1096D000464F555254480000464946544800000041
:1096E0005349585448000000534556454E544800CD
:1096F00045494748544800002046414D494C592CA3
:109700000A454E54455220594F5552204E414D4521
:109710002E0A592044454C455445532E0A50524573
:109720005353205354415254205748454E20444FE0
:109730004E452E002C0A41524520594F5520535575
:1097400052453F00594553004E4F005345434F4E3D
:109750004453002C0A505245535320535441525401
:1097600020544F20434F4E54494E55452E005349E7
:109770004E474C4500444F55424C450054524950C9
:109780004C45004F4646004F4E00004D555349434F
:109790003A005346583A0050524F4752414D4D49B6
:1097A0004E4720425920464C5B56494F205A41565D
:1097B000414E004152543A20464C5B56494F205A84
:1097C0004156414E004D555349433A204944455274
:1097D000414C444F204C5549532044412053494C5F
:1097E000564100434F444520554E4445522054486D
:1097F0004520474E552047504C2056330041525487
:1098000020414E44204D5553494320554E44455226
:109810002054484500435245415449564520434F42
:109820004D4D4F4E53004154545249425554494FA7
:109830004E2D534841524520414C494B4500332E53
:109840003020554E504F52544544204C4943454ECC
:109850005345005155455354494F4E533A20534EAA
:1098600045532046414D494C5920464555440041F9
:109870004E44205448452057494E4E4552204953A6
:109880003A0A00495427532041205449452E0019D3
:109890000A31323334353637383930414243444562
:1098A000464748494A4B4C4D4E4F505152535455E0
:1098B000565758595A202726000011241FBECFEFB3
:1098C000D0E1DEBFCDBF14BE88E10FB6F89480931F
:1098D0006000109260000FBE11E0A0E0B1E0EAE489
:1098E000FFED02C005900D92A831B107D9F71EE037
:1098F000A8E1B1E001C01D92A439B107E1F70E94CF
:109900005C56882311F40E947356F894E2EFF9E054
:1099100080E881939BE0EE3FF907D9F782EF99E069
:109920009093FF0B8093FE0B1092000C1092030C8F
:1099300010920D0C1092170C1092210C81E0809364
:10994000230C8093240C8093220C1092810015BC70
:109950009FEF97B994B998E99AB95C9A9CE091B94C
:109960009BEF92B91092DA0996E09093DB0910927E
:1099700085001092840093E0909389009DE8909375
:10998000880099E09093810092E090936F0092E4B8
:1099900094BD17BC85BD93E89093B0001092B300BE
:1099A0008093B10081E185B91092EE091092DE0931
:1099B0001092DF091092E9091092E8091092ED095E
:1099C0001092EC091092F0090E94F35580E00E9479
:1099D000D45580FF03C084E00E94D1550E947C5B77
:1099E00078940E94C25C0E94E56D0C94A36F0C9465
:1099F0000000EFEC00C000C0EA95E1F700C000C035
:109A0000C8E1D1E000EEA02E662776E0D1D03EE29C
:109A10003A95F1F70E94344D31E13A95F1F7AA9465
:109A200089F0C8956395683029F0C895C895C895A0
:109A30000000ECCF6627002430E5C30FD01DC89589
:109A40000000E4CF35E03A95F1F700C0B1D011E065
:109A50000091DD0901270093DD0900FF1093DC0967
:109A6000E2E0E09336000895DE014D915D91679F3D
:109A7000C001480F591FFA0128E2059108B94D911C
:109A8000059108B95D91059108B900C0059108B923
:109A9000480F591F059108B90591FA012A9508B98F
:109AA00061F700C00000002708B90895E64DF54DA4
:109AB000034E5A4D28980E949A4FEBE0EA95F1F731
:109AC00000C0E7E0E0938900EBE1E0938800E0E08C
:109AD000F6E0BED0289AE0FF30D0E0FF2DC02F93F3
:109AE0003F934F935F936F937F938F939F93AF9326
:109AF000BF9378941124E091E009F091E109E11518
:109B0000F10509F009950E947D5B0E9430560E9484
:109B1000C74E1124E091E209F091E309E115F10546
:109B200009F00995BF91AF919F918F917F916F91AE
:109B30005F914F913F912F910895EF93E091DB0951
:109B4000E93E80F4E93070F0EDE1FF2700800F92EC
:109B5000EA95E1F70E94F94CE1E0FF270F900192AE
:109B6000EE31E0F3EF910895FF93EF93EFB7EF93AA
:109B7000E0918400EE50F1E0EF1700F0F395FA3039
:109B8000D8F305D0EF91EFBFEF91FF9118950F92A9
:109B90001F92ECEAFAE90090DA09000C1124E00DBA
:109BA000F11D05901490F00109951F900F900895F4
:109BB00028980E949A4FE5E1EA95F1F7E091DB09D8
:109BC000EA95E093DB09289A00C0089528980E943E
:109BD000BC4F289A0000E1E0F6E03AD0E3E0E093E1
:109BE0008900EDE8E0938800089528980E94BC4F12
:109BF000E9EA0000EA95E9F700C00000F6E0E2E0DB
:109C000027D0289A089528980E94BC4F289A0000CF
:109C1000E3E0FDEF1DD0E091DB09E53091F4E09148
:109C2000DD09E1300000F091EE0919F4F091EE0940
:109C3000F195E3E0E0938900EDE8EF0FE093880011
:109C40000895E3E0E0938900EDE8E093880008954B
:109C50000090DB090A9410905F0011FC0F2E009217
:109C6000DB090090DA0911FC0E2E0092DA09E0E01F
:109C700011FCE1E008950000000000000000000079
:109C800000000000000000000000000000000000D4
:109C900000000000000000000000000000000000C4
:109CA00000000000000000000000000000000000B4
:109CB00000000000000000000000000000000000A4
:109CC0000000000000000000000000000000000094
:109CD0000000000000000000000000000000000084
:109CE0000000000000000000000000000000000074
:109CF0000000000000000000000000000000000064
:109D000099277727833008F00895ECE8FFE9660F7C
:109D1000771FE60FF71FA591B491E3E0FCE02AE07E
:109D2000289FE00DF11DA183B28311240895909125
:109D3000220C9170880F892B8093220C089599270B
:109D40007727E3E0FCE02AE0289FE00DF11D6E3F5D
:109D500031F46091220C6E7F6093220C0BC06F3F38
:109D600031F46091220C6E6F6093220C03C071EA93
:109D7000760F75831124089599277727E3E0FCE097
:109D80002AE0289FE00DF11D6083112408950E94B0
:109D90002E580090000C002019F4A2EFB9E002C088
:109DA000A8EFBAE021E002260092000C22E0209306
:109DB000010C2F923F924F925F926F927F928F92FF
:109DC0009F92AF92BF92CF92DF92EF92FF920F934A
:109DD0001F93CF93DF935091210C6091230C7091CE
:109DE000240C8091250C2090040C3090050C4090A0
:109DF000070C5090080C6090060C1091030C7090AA
:109E00000E0C80900F0C9090100CA090110CB09044
:109E1000120C20910D0CC090180CD090190CE090F1
:109E20001B0CF0901C0C00911A0C3091170C9FEF3A
:109E3000620C431CF2014491410300240008C12D2F
:109E4000D02D970CA81CF501449142030024000872
:109E5000C10DD01D0C0DED1CF701449143030024EE
:109E60000008C10DD01D8A956AF44091220C842F00
:109E70008695062E0694062600FA7695679576F95D
:109E800040FF66F940E860FD4FE745030024000805
:109E9000C10DD01D0024C038D0050CF0CFE70A94C6
:109EA000C038D0050CF4C0E8C058CD939A9509F09D
:109EB000BFCF4091010C4A954093010C97E009F007
:109EC000B7CF6092060C4092070C9092100CA092B3
:109ED000110C00931A0CE0921B0C6093230C7093EE
:109EE000240C8093250CDF91CF911F910F91FF904F
:109EF000EF90DF90CF90BF90AF909F908F907F902A
:109F00006F905F904F903F902F900895E091FE0BDF
:109F1000F091FF0B019100000093B3000BE0EE3FC6
:109F2000F00702EF19E008F0F801E093FE0BF09360
:109F3000FF0B08950C949C4F0C949E4F0F931F930E
:109F40002F93E091FE0BF091FF0B01910093B30072
:109F50000BE0EE3FF00708F400C010F0E2EFF9E08C
:109F6000E093FE0BF093FF0B26E02A95F1F700C07B
:109F70002F911F910F9108950000E091DB09E0FF00
:109F8000DDCFE1E1EA95F1F700C008952200240059
:109F9000260028002B002D00300033003600390049
:109FA0003D004000440048004C00510056005B005A
:109FB000600066006C0073007900810088009000EA
:109FC0009900A200AC00B600C100CC00D800E500AA
:109FD000F3000101100121013201440157016C011C
:109FE00081019801B001CA01E5010202210241028A
:109FF00064028802AE02D7020303300361039403B4
:10A00000CB03050442048304C70410055D05AF05B6
:10A0100005066106C206290796070908830805098F
:10A020008E09200ABA0A5D0B0A0CC10C840D510E70
:10A030002B0F121007110A121D1340147415BA16B3
:10A0400014188319071BA31C571E24200E22142446
:10A0500039267F28E82A752D293006330F364539F1
:10A06000AD3C49401B442848734CFE50CF55EA5A3A
:10A0700051600C661D6C8B725A79928037885090B3
:10A08000E598FDA19FABD3B5A3C000000000000080
:10A0900000000000000000000000000000000000C0
:10A0A00000000000000000000000000000000000B0
:10A0B00000000000000000000000000000000000A0
:10A0C0000000000000000000000000000000000090
:10A0D0000000000000000000000000000000000080
:10A0E0000000000000000000000000000000000070
:10A0F0000000000000000000000000000000000060
:10A10000000306090C101316191C1F2225282B2EDC
:10A11000313336393C3F414447494C4E51535558F1
:10A120005A5C5E60626466686A6B6D6F70717374AE
:10A13000757678797A7A7B7C7D7D7E7E7E7F7F7F67
:10A140007F7F7F7F7E7E7E7D7D7C7B7A7A7978764D
:10A1500075747371706F6D6B6A68666462605E5C63
:10A160005A585553514E4C494744413F3C39363378
:10A17000312E2B2825221F1C191613100C0906033B
:10A1800000FDFAF7F4F0EDEAE7E4E1DEDBD8D5D242
:10A19000CFCDCAC7C4C1BFBCB9B7B4B2AFADABA80D
:10A1A000A6A4A2A09E9C9A9896959391908F8D8C30
:10A1B0008B8A888786868584838382828281818157
:10A1C0008181818182828283838485868687888A51
:10A1D0008B8C8D8F9091939596989A9C9EA0A2A41B
:10A1E000A6A8ABADAFB2B4B7B9BCBFC1C4C7CACDE6
:10A1F000CFD2D5D8DBDEE1E4E7EAEDF0F4F7FAFD03
:10A20000808182838485868788898A8B8C8D8E8FD6
:10A21000909192939495969798999A9B9C9D9E9FC6
:10A22000A0A1A2A3A4A5A6A7A8A9AAABACADAEAFB6
:10A23000B0B1B2B3B4B5B6B7B8B9BABBBCBDBEBFA6
:10A24000C0C1C2C3C4C5C6C7C8C9CACBCCCDCECF96
:10A25000D0D1D2D3D4D5D6D7D8D9DADBDCDDDEDF86
:10A26000E0E1E2E3E4E5E6E7E8E9EAEBECEDEEEF76
:10A27000F0F1F2F3F4F5F6F7F8F9FAFBFCFDFEFF66
:10A28000000102030405060708090A0B0C0D0E0F56
:10A29000101112131415161718191A1B1C1D1E1F46
:10A2A000202122232425262728292A2B2C2D2E2F36
:10A2B000303132333435363738393A3B3C3D3E3F26
:10A2C000404142434445464748494A4B4C4D4E4F16
:10A2D000505152535455565758595A5B5C5D5E5F06
:10A2E000606162636465666768696A6B6C6D6E6FF6
:10A2F000707172737475767778797A7B7C7D7E7FE6
:10A3000000020406080A0C0E10121416181A1C1E5D
:10A3100020222426282A2C2E30323436383A3C3E4D
:10A3200040424446484A4C4E50525456585A5C5E3D
:10A3300060626466686A6C6E70727476787A7C7E2D
:10A340007F7D7B79777573716F6D6B69676563610D
:10A350005F5D5B59575553514F4D4B4947454341FD
:10A360003F3D3B39373533312F2D2B2927252321ED
:10A370001F1D1B19171513110F0D0B0907050301DD
:10A38000FFFDFBF9F7F5F3F1EFEDEBE9E7E5E3E1CD
:10A39000DFDDDBD9D7D5D3D1CFCDCBC9C7C5C3C1BD
:10A3A000BFBDBBB9B7B5B3B1AFADABA9A7A5A3A1AD
:10A3B0009F9D9B99979593918F8D8B89878583819D
:10A3C00080828486888A8C8E90929496989A9C9E9D
:10A3D000A0A2A4A6A8AAACAEB0B2B4B6B8BABCBE8D
:10A3E000C0C2C4C6C8CACCCED0D2D4D6D8DADCDE7D
:10A3F000E0E2E4E6E8EAECEEF0F2F4F6F8FAFCFE6D
:10A400007F7F7F7F7F7F7F7F7F7F7F7F7F7F7F7F5C
:10A410007F7F7F7F7F7F7F7F7F7F7F7F7F7F7F7F4C
:10A420007F7F7F7F7F7F7F7F7F7F7F7F7F7F7F7F3C
:10A430007F7F7F7F7F7F7F7F7F7F7F7F7F7F7F7F2C
:10A700000309131E28313A40464C5054585B5E6191
:10A71000636567696B6C6E6F707172737475767751
:10A72000777879797A7A7B7B7C7C7C7D7D7D7E7E77
:10A730007E7E7F7F7F7F7F7F7F7F7F7F7F7F7F7F2B
:10A740007F7F7F7F7F7F7F7F7F7F7F7F7F7E7E7E1C
:10A750007E7D7D7D7C7C7C7B7B7A7A79797877774E
:10A76000767574737271706F6E6C6B696765636117
:10A770005E5B5854504C46403A31281E1309030082
:10A78000C6CCD5DBDFE3E5E7E9EAEBECEDEEEFEF96
:10A79000F0F0F0F1F1F1F1F2F2F2F2F2F2F2F2F3A2
:10A7A000F3F3F3F3F3F3F3F3F3F3F3F3F3F3F3F379
:10A7B000F3F3F3F3F3F3F3F3F3F3F3F3F3F3F3F369
:10A7C000F3F3F3F3F3F3F3F3F3F3F3F3F3F3F3F359
:10A7D000F3F3F3F3F3F3F3F3F3F3F3F3F3F3F3F349
:10A7E000F2F2F2F2F2F2F2F2F1F1F1F1F0F0F0EF56
:10A7F000EFEEEDECEBEAE9E7E5E3DFDBD5CCC60015
:10A8000000283D42302D2C2B2C2D2E2F303233356D
:10A8100037393B3D3F414345484A4C4E50535557CD
:10A82000595B5D5F61636567696B6C6E70717374B2
:10A83000757778797A7B7C7D7D7E7E7F7F7F7F7F59
:10A840007F7F7F7F7F7F7E7E7D7D7C7B7A7978773F
:10A8500075747371706E6C6B69676563615F5D5B66
:10A8600059575553504E4C4A484543413F3D3B395B
:10A8700037353332302F2E2D2C2B2C2D30423D28C6
:10A8800000E9E5FED4D7D7D7D6D4D2D0CECCCAC82B
:10A89000C6C3C1BFBDBAB8B6B4B1AFADABA9A7A569
:10A8A000A3A19F9E9C9A999795949391908F8D8C3C
:10A8B0008B8A89888887868585848484838383833B
:10A8C0008383838383848484858586878888898A33
:10A8D0008B8C8D8F909193949597999A9C9E9FA124
:10A8E000A3A5A7A9ABADAFB1B4B6B8BABDBFC1C33C
:10A8F000C6C8CACCCED0D2D4D6D7D7D7D4FEE5E9F5
:10A90000F9F8F9F5EBE1DDDEE0E2E4E5E6E5E4E2C5
:10A91000DED9D2CAC1B7ACA299918A8683818080E0
:10A920008182838586888A8C8D8F90929395969765
:10A9300098999A9B9B9C9D9D9D9E9E9E9F9F9F9F4D
:10A940009F9F9F9E9E9E9D9D9D9C9B9B9A99989745
:10A9500096959392908F8D8C8A888685838281804C
:10A96000808183868A9199A2ACB7C1CAD2D9DEE22E
:10A97000E4E5E6E5E4E2E0DEDDE1EBF5F9F8F90037
:10A980000708070B151F2322201E1C1B1A1B1C1E49
:10A9900022272E363F49545E676F767A7E7F7F7F0F
:10A9A0007F7E7D7B7A7876747371706E6D6B6A6969
:10A9B0006867666565646463636262626161616160
:10A9C0006161616262626363636465656667686949
:10A9D0006A6B6D6E7071737476787A7B7D7E7F7F23
:10A9E0007F7F7E7A766F675E54493F362E27221E20
:10A9F0001C1B1A1B1C1E2022231F150B07080700F7
:10AA00001F313D444E5354565A5F64696E747679D3
:10AA10007C7F7F7F7F7F7F7F7F7F7F7F7F7F7F7F49
:10AA20007F7F7F7F7F7F7F7F7F7F7F7F7F7F7F7F36
:10AA30007F7F7F7F7F7F7F7F7F7F7F7F7F7F7F7F26
:10AA40007F7F7F7F7F7F7F7F7F7F7F7F7F7F7F7F16
:10AA50007F7F7F7F7F7F7F7F7F7F7F7F7F7F7F7F06
:10AA60007F7F7F7F7F7F7F7F7F7F7F7F7F7F7F7FF6
:10AA70007F7F7F7F7F7F7F7F7F7F7F7C7871684C48
:10AA80002C1C120C0A0B0A05FDF3E9DFD4CAC0B76F
:10AA9000AEA69E97918B8685828080808080808004
:10AAA00080808080808080808080808080808080A6
:10AAB0008080808080808080808080808080808096
:10AAC0008080808080808080808080808080808086
:10AAD0008080808080808080808080808080808076
:10AAE0008080808080808080808080808080808066
:10AAF000808080808087919DACC4CBD4DDF2FAFA4F
:10AB0000E0E6F4E0A8E1B1E06091D8097091D909DC
:10AB10006D937D933197E1F7112408959927552777
:10AB200028E2220F629F880F080E191EA8E1B1E0EB
:10AB3000A00DB11D6091D8097091D90920E3429F01
:10AB4000600D711D6D937C931124089599277727CB
:10AB500028E2220F629F880F080E191EA8E1B1E0BB
:10AB6000A00DB11D6091E4097091E50920E3429FB9
:10AB7000600D711D529F700D6D937C93112408958B
:10AB80008093D8099093D90908958093E40990930C
:10AB9000E50908958091DC09089511241092DC09DB
:10ABA00008958093EE090895882329F48091E60999
:10ABB0009091E70908958091EA099091EB09089531
:10ABC000F999FECF92BD81BD60BDF894FA9AF99AC9
:10ABD00078940895F999FECF92BD81BDF894F89AC2
:10ABE00080B578940895129AC895C895129840E057
:10ABF00080E090E020E030E03695279596958795A7
:10AC00001398C895C895009B3068019B9068139A6B
:10AC1000C895C8954F5F403179F73093E709209385
:10AC2000E6099093EB098093EA098091E6099091F7
:10AC3000E7098F30910539F08091EA099091EB098D
:10AC40008F30910561F428E088E190E00FB6F89428
:10AC5000A895809360000FBE20936000FFCF0895F9
:10AC60001092370C009903C081E08093370C019952
:10AC700005C08091370C82608093370C0E94F35599
:10AC800008959091370C90FD02C080E009C020919A
:10AC9000E6093091E709832F881F8827881F8F5F77
:10ACA00091FF09C02091EA093091EB0937FF02C0FA
:10ACB00088600895846008951F9380E090E00E946A
:10ACC000EA55182F81E090E00E94EA5590E0382F75
:10ACD00020E0210F311D85E52A35380709F491E080
:10ACE000892F1F910895CF93DF93C0E0D0E0FE013C
:10ACF000E059FF4F6491CE010E94E0552196C03289
:10AD0000D105A9F7C0E2D0E0CE016FEF0E94E05577
:10AD1000CE0101966FEF0E94E055A09688E0C0300A
:10AD2000D80791F7DF91CF91089590E026E130E0C8
:10AD3000829FF001839FF00D929FF00D1124E65C3D
:10AD4000F34F628708956093220C089590E026E106
:10AD500030E0829FF001839FF00D929FF00D11244F
:10AD6000E65CF34F13861182089590E026E130E00F
:10AD7000829FF001839FF00D929FF00D1124E65CFD
:10AD8000F34F81E0838B089590E026E130E0829FCD
:10AD9000F001839FF00D929FF00D1124E65CF34FBC
:10ADA0006187089590E026E130E0829FF001839F63
:10ADB000F00D929FF00D1124E65CF34F648308952B
:10ADC00090E026E130E0829FF001839FF00D929F9A
:10ADD000F00D1124E65CF34F658308959093950C74
:10ADE0008093940C8FE680939A0C1092F109EAE319
:10ADF000FCE021E08FEF98E1208310868683878333
:10AE000014861182958376963CE0E239F307A1F728
:10AE1000089510923B0C1092510C1092670C1092F6
:10AE20007D0C019690939E0C80939D0C9093390C11
:10AE30008093380C9093A10C8093A00C10929C0CE2
:10AE400010929B0C1092930C1092920C1092960CF4
:10AE500081E08093F1091092990C1092980C08955A
:10AE6000E4E4FCE09091000186E1989FC001112488
:10AE70008E0F9F1F2AEF04C0308137FF2083769604
:10AE8000E817F907C9F71092F1090895DC012D912F
:10AE90003C911197A9014F5F5F4F11965C934E93C0
:10AEA000F901249130E027FF15C02F7730703695D7
:10AEB000322F222737952795CA014F5F5F4FFC013C
:10AEC0008491982F9F77290F311D87FDF0CF119620
:10AED0005C934E93C9010895FC01108A12868FEF8E
:10AEE00081876087138A118A91E09387128A14827E
:10AEF00086834283089580939A0C08950E949F4E02
:10AF00000895EF92FF920F931F93DF93CF9300D09A
:10AF1000CDB7DEB7182F062FE82EFF2486E190E08C
:10AF2000E89EF001E99EF00DF89EF00D1124E65C1C
:10AF3000F34F8385882321F08181882309F085C020
:10AF4000222391F486E190E0E89EF001E99EF00D65
:10AF5000F89EF00D1124E65CF34F138A8285882356
:10AF600009F073C0108671C0133059F481E091E08C
:10AF70009093240C8093230C81E08093220C042F67
:10AF80000DC0812F60E02A8349830E949F4E812F4C
:10AF90004981642F0E94804E49812A810F3789F4AC
:10AFA00086E190E0E89EF001E99EF00DF89EF00D3C
:10AFB0001124E65CF34F8091970C878788E99CE029
:10AFC0002CC089E0089FC0011124E091940CF091FD
:10AFD000950CE80FF91F339685919491009771F4C1
:10AFE00086E190E0E89EF001E99EF00DF89EF00DFC
:10AFF0001124E65CF34F158A148A11C0FC013491C8
:10B0000066E170E0E69EF001E79EF00DF69EF00D21
:10B010001124E65CF34F37870196958B848B86E18C
:10B0200090E0E89EF001E99EF00DF89EF00D1124ED
:10B03000E65CF34F0487118286E1189FC00111245A
:10B04000865C934F622F0E946C570F900F90CF91A8
:10B05000DF911F910F91FF90EF900895CF92DF92B3
:10B06000EF92FF921F93CF93DF93E3E4FCE08181A3
:10B07000992787FD90952081820F911D8F3F910523
:10B0800019F014F08FEF90E097FF02C080E090E09D
:10B09000808376968CE0EB39F80749F78091F109C7
:10B0A000882309F05FC17AC140919D0C50919E0C9C
:10B0B000DA011196B0939E0CA0939D0CFA01449175
:10B0C0004F3F71F5BD016F5F7F4F70939E0C609392
:10B0D0009D0CFD01A491AF3219F41092F10950C1F9
:10B0E000A63009F032C1FB0131969F012F5F3F4F1F
:10B0F00030939E0C20939D0C8491833529F43093DA
:10B10000A10C2093A00C21C1853409F01EC18091AF
:10B11000A00C9091A10C90939E0C80939D0C15C156
:10B1200047FF02C04093960C842F8F70242F30E08D
:10B13000207F30702039310541F0203B3105A1F0EE
:10B14000203C310509F076C05EC09D012F5F3F4F66
:10B15000FD014491B9016F5F7F4F70939E0C609326
:10B160009D0CF901249181C09D012F5F3F4FFD018E
:10B17000A491A9014F5F5F4F50939E0C40939D0C8B
:10B18000F9019491A73071F4282F30E02C9FF00141
:10B190002D9FF00D3C9FF00D1124E65CF34F990FAD
:10B1A0009783D3C0AB3071F4282F30E02C9FF0018F
:10B1B0002D9FF00D3C9FF00D1124E65CF34F990F8D
:10B1C0009683C3C0AC3571F4282F30E02C9FF0017A
:10B1D0002D9FF00D3C9FF00D1124E65CF34F990F6D
:10B1E0009483B3C0A43609F0B0C0282F30E02C9F60
:10B1F000F0012D9FF00D3C9FF00D1124E65CF34F04
:10B20000990F9583A2C09D012F5F3F4F30939E0CF5
:10B2100020939D0CFD01249190E08C9FD0018D9F87
:10B22000B00D9C9FB00D1124A65CB34F1C962C93BF
:10B230001C978BC02091960C822F8F7030E0207F5E
:10B2400030702039310541F0203B310511F1203CAF
:10B25000310509F07AC06EC09D012F5F3F4F3093DA
:10B260009E0C20939D0CFD012491682F70E06C9F33
:10B27000F0016D9FF00D7C9FF00D1124E65CF34F03
:10B280009081992309F461C0220F64850E9481573F
:10B290005CC09D012F5F3F4F30939E0C20939D0C0F
:10B2A000FD012491473081F490E08C9FD0018D9F67
:10B2B000B00D9C9FB00D1124A65CB34FE22FEE0F92
:10B2C0001796EC93179741C04B3081F490E08C9F18
:10B2D000D0018D9FB00D9C9FB00D1124A65CB34F83
:10B2E000E22FEE0F1696EC9316972FC04C3581F493
:10B2F00090E08C9FD0018D9FB00D9C9FB00D1124CC
:10B30000A65CB34FE22FEE0F1496EC9314971DC07A
:10B310004436D9F490E08C9FD0018D9FB00D9C9F56
:10B32000B00D1124A65CB34FE22FEE0F1596EC93EF
:10B3300015970BC090E08C9FF0018D9FF00D9C9FA6
:10B34000F00D1124E65CF34F44878DE99CE00E94E8
:10B35000465790939C0C80939B0C1092930C1092E8
:10B36000920C02C0C6E1D0E08091920C9091930CB7
:10B3700020919B0C30919C0C8217930709F494CE7A
:10B3800001969093930C8093920C8091980C9091DD
:10B39000990C01969093990C8093980C13E0E12EF0
:10B3A0001CE0F12ECBE3DCE010E0BFEFCB2ED12C84
:10B3B0008A89882309F05BC08B899C89009709F4EE
:10B3C00053C09F858E85981708F049C04DC08B8566
:10B3D000EB89FC898F37E1F4DF018D91BC8BAB8B5E
:10B3E0008F3FF1F061811196BC8BAB8BE82FF0E0C1
:10B3F000EE0FFF1FE057FF4F0190F081E02D812FEE
:10B400000995EB89FC8981918E87FC8BEB8B26C09B
:10B41000BF016F5F7F4F7C8B6B8B84918F3F21F4DB
:10B4200018821C8A1B8A20C09B012F5F3F4F3C8BD8
:10B430002B8BFB01649190E0880F991F80579F4FE1
:10B44000FC0125913491812FF9010995EB89FC8943
:10B45000CF0101969C8B8B8BE491EE871F869F8595
:10B460008E85981709F4B3CF8F858F5F8F878A8574
:10B47000882319F480E090E068C088898F3F11F03C
:10B480008F5F888B8F81882309F459C038853323D7
:10B4900009F455C09E81992309F451C020919A0C5A
:10B4A000222309F44CC0989FC001112480509F4F63
:10B4B000692F7727432F50E0649FC001659F900D4F
:10B4C000749F900D112480509F4F692F77274D81D5
:10B4D00050E0649FC001659F900D749F900D1124F2
:10B4E00080509F4F492F552730E0429FC001439F16
:10B4F000900D529F900D112480509F4F892F9927B6
:10B500003B813323F1F0EA81F0E0E050FF452491E4
:10B510002058239F9001112420503F4F232F332781
:10B52000A601421B530B489F9001499F300D589F25
:10B53000300D112420503F4F832F992702C080E007
:10B5400090E02A813C81230F2A83F70180831F5FCB
:10B550008AE090E0E80EF91E6696143009F028CFD4
:10B56000DF91CF911F91FF90EF90DF90CF900895E2
:10B57000EF92FF920F931F93CF93DF9329E0829F67
:10B5800090011124C091940CD091950CC20FD31F3F
:10B590009E012D5F3F4FF901A591B491FE01949159
:10B5A0009150923010F413E01DC09091510C9923EA
:10B5B000B1F090915D0C981711F4442381F49091AF
:10B5C000670C992371F09091730C981711F4442330
:10B5D00041F42091610C9091770C921710F411E0D6
:10B5E00001C012E0E12EFF24FD01949126E130E03C
:10B5F000E29EE001E39ED00DF29ED00D1124C65CC8
:10B60000D34F9F871196BD8BAC8B8D8701E009834B
:10B6100086E1189FC0011124865C934F40E50E948B
:10B620006C57133049F481E091E09093240C80939F
:10B63000230C0093220C15C08BE090E0E89EF001F3
:10B64000E99EF00DF89EF00D1124EE0FFF1FE45C53
:10B65000F34F812F60810E94804E812F6A890E9462
:10B660009F4EDF91CF911F910F91FF90EF90089522
:10B670000F931F93082F162F0E94804E202F30E02B
:10B680008BE090E0289FF001299FF00D389FF00D8E
:10B690001124EE0FFF1FE45CF34F10831F910F91F5
:10B6A0000895482F50E02BE030E0429FF001439F87
:10B6B000F00D529FF00D1124EE0FFF1FE45CF34FCD
:10B6C0009081961B9083692F0E94804E0895482F89
:10B6D00050E02BE030E0429FF001439FF00D529F7D
:10B6E000F00D1124EE0FFF1FE45CF34F9081690F02
:10B6F00060830E94804E0895089508950F931F93CC
:10B70000CF93DF938C01C0E0D0E007C00E94CA5500
:10B710008823E1F30E94CD552196C017D107B4F3D9
:10B72000DF91CF911F910F91089540520E948E5545
:10B730000895EF92FF921F93CF93DF93EC01162FA2
:10B74000E42EF52EF70144910894E11CF11C4423EA
:10B7500041F08C2F21964F774052612F0E948E55D9
:10B76000F1CFDF91CF911F91FF90EF900895CF928D
:10B77000DF92EF92FF920F931F93CF93DF93062FE9
:10B78000142FE22EC82EE6016E01D92EE601FF2409
:10B79000112311F4FF2049F4812F6AE00E949B6E6F
:10B7A000492F405F8C2F602F09C0EE2021F08C2F95
:10B7B000602F40E103C08C2F602F40E00E948E5527
:10B7C000F394219743E0D42EFD1431F0812F6AE0E9
:10B7D0000E949B6E182FDCCFDF91CF911F910F91AC
:10B7E000FF90EF90DF90CF900895AF92BF92CF92ED
:10B7F000DF92EF92FF920F931F93CF93DF93062F69
:10B8000069017A01A82EE5015E01B92EE50110E07B
:10B81000C114D104E104F10411F4112369F4C70146
:10B82000B6012AE030E040E050E00E94CE6E462FA4
:10B83000405F8C2F602F03C08C2F602F40E00E9450
:10B840008E551F5F21971A3069F0C701B6012AE0B3
:10B8500030E040E050E00E94CE6EC22ED32EE42EA7
:10B86000F52ED6CFDF91CF911F910F91FF90EF90E2
:10B87000DF90CF90BF90AF9008957F928F929F926C
:10B88000AF92BF92CF92DF92EF92FF920F931F93EE
:10B89000CF93DF93E82EF62EEA016901480100E01C
:10B8A00010E00EC08E2D8A0D672DA4010E94A655B2
:10B8B0000894A11CB11CAC16BD06A4F30F5F1F4F6A
:10B8C0000C151D052CF4AA24BB24702E7F0CF3CF7D
:10B8D000DF91CF911F910F91FF90EF90DF90CF906C
:10B8E000BF90AF909F908F907F9008956F927F92BE
:10B8F0009F92AF92BF92CF92DF92EF92FF920F93FF
:10B900001F93CF93DF93A82EB62EEA01FA01E5909C
:10B91000F490FA013296C590D49010E015C0E60D6F
:10B92000F71D3296EE0FFF1FEC0FFD1F459154914E
:10B93000802F8A0D692D0E94A6550F5FE02FF0E041
:10B94000EE15FF0564F31F5F812F90E08C159D05B8
:10B950005CF48E9D30018F9D700C9E9D700C1124A7
:10B9600000E0912E9B0CEACFDF91CF911F910F91B8
:10B97000FF90EF90DF90CF90BF90AF909F907F901F
:10B980006F900895CF93DF938DEB90E00E94EE5679
:10B99000C6ECD0E0CE010E94C555CE010E94C05534
:10B9A0000E9480558FE090E00E947E5B80E06FEF08
:10B9B00041E00E94B85AC6E1D8E082E16CE0AE01F5
:10B9C0000E94765C83E090E00E947E5B82E16CE006
:10B9D0004AE458E00E94765C82E090E00E947E5B40
:10B9E00082E16CE0AE010E94765C80E290E00E9411
:10B9F0007E5B0E9480558AE090E00E947E5BDF9132
:10BA0000CF91089590E0880F991FFC01E15DF34FFD
:10BA100020813181855D934FFC0180819181822B52
:10BA2000932B807C81F0207C19F06093500D09C02D
:10BA30008091500D81508093500D882321F44093C4
:10BA4000500D81E0089580E0089590E0880F991FDF
:10BA5000FC01E15DF34F20813181855D934FFC0155
:10BA600080819181822B932B80739070009799F045
:10BA7000207330702115310519F06093500D09C005
:10BA80008091500D81508093500D882321F4409374
:10BA9000500D81E0089580E00895CF93DF93DC019D
:10BAA00088E590E0A89FB001A99F700DB89F700D28
:10BAB0001124FB01EC56F24F249190E00AC0E855A6
:10BAC000F34F20839F5FFB01E90FF11DEC56F24F0E
:10BAD0002491E92FF0E02B3391F7E855F34FEF0174
:10BAE000219788818F3319F08EE280839F5FC92F61
:10BAF000D0E0FE01E855F34F108228E18AE00AC049
:10BB00002150E22FF0E0E855F34F30813032C1F799
:10BB10008083285E422F50E04F5F5F4F4C175D07D8
:10BB200084F32CE230E0A29FA001A39F500DB29FAE
:10BB3000500D112441505040440F551F80E020E02B
:10BB4000FB01E90FF11DEC56F24F9F5F34913B333F
:10BB500011F03323E9F4A82FB0E0ED01E4E0CC0FBD
:10BB6000DD1FEA95E1F7CA0FDB1FCD5AD24FDE0188
:10BB7000A20FB11D11971C92DA01A90FB11DAC568D
:10BB8000B24FFD01A491A88B8F5F3323C1F612C081
:10BB9000A82FB0E0FD01E295F295F07FFE27E07F4F
:10BBA000FE27EA0FFB1FE20FF11DED5AF24F308323
:10BBB0002F5FC6CF80934E0DDF91CF910895609196
:10BBC0004E0D4091A60C5091A70C20E030E023C010
:10BBD000FA01022E02C0F695E7950A94E2F7E0FD1D
:10BBE00018C0F901A4E0EE0FFF1FAA95E1F7E20FDC
:10BBF000F31FED5AF24FACE0BEE090817C919717B5
:10BC000041F4992359F0319611969EE0AD31B90770
:10BC1000A1F72F5F3F4F822F2617D0F20895EF92A2
:10BC2000FF920F931F93CF93DF93082F31E0E32E02
:10BC3000F12C02C0EE0CFF1C8A95E2F7CDEFDDE09F
:10BC400018E0898190E08E219F21002E02C09595F9
:10BC500087950A94E2F7E881F0E0EE21FF21002EBB
:10BC600002C0F595E7950A94E2F7EE0FFF1FE80F83
:10BC7000F91FEE0FFF1FE75FFE4F40815181812FBB
:10BC80006AE00E94765CEA81F0E0EE21FF21002E5E
:10BC900002C0F595E7950A94E2F7EE0FFF1FEE0F4D
:10BCA000FF1FEF5FFE4F40815181812F6CE00E94AA
:10BCB000765C1B5F2396113221F680E090E06FE006
:10BCC00070E048E250E024E030E005E510E00E943A
:10BCD0003D5C85E06EE044E654E70E94765CDF91CF
:10BCE000CF911F910F91FF90EF900895CF92DF9227
:10BCF000EF92FF920F931F93F82EE62ED42EC22EB2
:10BD000090E070E050E030E002E010E00E943D5C26
:10BD10008F2D6E2D41E050E00E94A6551F2D115031
:10BD20001D0D812F6E2D49E050E00E94A655EA942A
:10BD3000EC0C8F2D6E2D41E250E00E94A655812F14
:10BD40006E2D45E250E00E94A6551F910F91FF9085
:10BD5000EF90DF90CF9008950F931F9380E090E0D5
:10BD600060E070E048E250E02CE130E000E010E0FC
:10BD70000E943D5C8CE065E04CEF52E70E94765CEF
:10BD800084E06CE040E22BE00E94765E85E090E08B
:10BD90006DE070E047E957E90E94995B85E090E02B
:10BDA0006EE070E043EB57E90E94995B85E090E01C
:10BDB0006FE070E045EC57E90E94995B85E090E008
:10BDC00060E170E043EE57E90E94995B85E090E006
:10BDD00061E170E04DEF57E90E94995B85E090E0EA
:10BDE00062E170E045E158E90E94995B85E090E0EE
:10BDF00063E170E046E258E90E94995B85E090E0DB
:10BE000064E170E04EE358E90E94995B85E090E0C0
:10BE100065E170E043E558E90E94995B89E068E1DB
:10BE200046E123E00E94765E8BE090E069E170E0FD
:10BE300047E256E90E94995B80912B0C90912C0C63
:10BE40009093340C8093330C80912D0C90912E0C98
:10BE50009093360C8093350C81E090E00E947E5BDD
:10BE600080E00E94D4559C0190932C0C80932B0C65
:10BE70008091330C9091340C80959095822393237C
:10BE80009093300C80932F0C81E00E94D4559C013C
:10BE900090932E0C80932D0C8091350C9091360C44
:10BEA00080959095822393239093320C8093310C4C
:10BEB00080912F0C81FD0DC080912B0C90912C0C4A
:10BEC0009093340C8093330C3093360C2093350CC4
:10BED000C3CF1F910F910895FF920F931F93CF939C
:10BEE000DF9380E090E060E070E048E250E02CE119
:10BEF00030E000E010E00E943D5C8CE065E04CEF3B
:10BF000052E70E94765C8EE062E14CE025E00E9400
:10BF1000765E81E190E063E170E044E156E90E94E1
:10BF2000995B81E190E064E170E049E156E90E94AB
:10BF3000995B81E190E065E170E041E256E90E94A1
:10BF4000995B89E068E146E123E00E94765E8BE040
:10BF500090E069E170E047E256E90E94995B8091C8
:10BF60002B0C90912C0C9093340C8093330C80917B
:10BF70002D0C90912E0C9093360C8093350CC0E0D4
:10BF8000D0E0FF2481E090E00E947E5B21968FE06C
:10BF900090E063E170E041E050E023E030E002E057
:10BFA00010E00E943D5C6F2D6D5E8FE04FE650E02B
:10BFB0000E94A65580E00E94D4559C0190932C0CC1
:10BFC00080932B0C8091330C9091340C809590953C
:10BFD000822393239093300C80932F0C81E00E9456
:10BFE000D4559C0190932E0C80932D0C8091350C90
:10BFF0009091360C80959095822393239093320CE8
:10C000008093310C80912F0C9091300C81309105F0
:10C0100081F08031910531F080329105B1F48F2D9E
:10C020008F5F02C08F2D8E5F63E00E949B6EF92EA2
:10C030000CC0BE0180E090E00E94636F8F2DDF9105
:10C04000CF911F910F91FF90089580912B0C9091AB
:10C050002C0C9093340C8093330C3093360C20933B
:10C06000350C90CFFF920F931F9380E090E060E03B
:10C0700070E048E250E02CE130E000E010E00E9487
:10C080003D5C8CE065E04CEF52E70E94765C8DE011
:10C0900062E14EE025E00E94765E80E190E063E19F
:10C0A00070E04BE857E90E94995B80E190E064E121
:10C0B00070E042E957E90E94995B80E190E065E118
:10C0C00070E04BEA56E90E94995B89E068E146E13D
:10C0D00023E00E94765E8BE090E069E170E047E249
:10C0E00056E90E94995B80912B0C90912C0C9093B7
:10C0F000340C8093330C80912D0C90912E0C9093E6
:10C10000360C8093350CFF2481E090E00E947E5B2A
:10C110008FE090E063E170E041E050E023E030E048
:10C1200002E010E00E943D5C6F2D6D5E8FE04FE6F7
:10C1300050E00E94A65587E190E063E170E043E0A3
:10C1400050E022E030E00E943D5C4091120150E05E
:10C1500041705070440F551F440F551F4D5758469E
:10C1600087E190E063E170E00E94995B40911201E9
:10C17000469550E041705070440F551F440F551FB5
:10C180004D57584687E190E064E170E00E94995B6A
:10C1900080E00E94D4559C0190932C0C80932B0C32
:10C1A0008091330C9091340C809590958223932349
:10C1B0009093300C80932F0C81E00E94D4559C0109
:10C1C00090932E0C80932D0C8091350C9091360C11
:10C1D00080959095822393239093320C8093310C19
:10C1E00080912F0C982F907CD9F021E030E00F2C1B
:10C1F00002C0220F331F0A94E2F7809112018227B6
:10C2000080931201FF20D1F480FF05C082E798E0FF
:10C210000E94095713C082E798E00E9430570EC071
:10C2200084FF03C082E0F80E09C085FF02C0F394CA
:10C2300005C080FF03C082E0F816B1F080912B0C9E
:10C2400090912C0C9093340C8093330C80912D0C96
:10C2500090912E0C9093360C8093350C8F2D63E0CB
:10C260000E949B6EF92E50CF1F910F91FF90089561
:10C270002F923F924F925F926F927F928F929F92F6
:10C28000AF92BF92CF92DF92EF92FF920F931F93E4
:10C29000DF93CF9300D000D000D0CDB7DEB79E8320
:10C2A0008D83E62E4983722E86E063E14CE127E020
:10C2B0000E94765ECC24DD2420E01AC0E22FE00F3D
:10C2C000F0E0EF56F7464491C8010496880F991F95
:10C2D000B5012C830E94955B0F5F1F4F2C810D30A1
:10C2E000110561F7235F0894C11CD11C273241F06E
:10C2F00000E010E086E1A82EB12CAC0CBD1CDECF16
:10C30000772011F4FF241AC0AD808E81CA2CD82E5C
:10C310000DE010E007C0C8016FE070E00E94955B7F
:10C320000F5F1F4FFC2CFA18F6014081442331F0B7
:10C330000894C11CD11C0A31110569F780911301C1
:10C3400090E002C095958795EA94E2F7662463949D
:10C35000682280912B0C90912C0C9093340C80933C
:10C36000330C80912D0C90912E0C9093360C809371
:10C37000350C8981869504E1402E512C481A5108CC
:10C3800014E1C12EC81AEE24DD249924BDE28B2EBF
:10C39000862D90E0880F991FFBE22F2EFCE03F2EA8
:10C3A000280E391E9C01215D334F3B832A8381E097
:10C3B00090E00E947E5B93943EE1391510F48A94DC
:10C3C000992487FE0DC08F2D772009F490C0F39437
:10C3D000882309F08CC080E2ED81FE81808387C0D4
:10C3E00080E00E94D4559C0190932C0C80932B0CE0
:10C3F0008091330C9091340C8095909582239323F7
:10C400009093300C80932F0C81E00E94D4559C01B6
:10C4100090932E0C80932D0C8091350C9091360CBE
:10C4200080959095822393239093320C8093310CC6
:10C43000862D68E046E00E94255D882339F4862D2C
:10C4400068E044E00E94025D8823A1F0F101808150
:10C4500086FF03C0FCE0EF0E68C087FF02C0E394D4
:10C4600064C085FF02C0D39460C084FF5EC022E038
:10C47000D20E5BC0EA81FB81808180FF21C02DE06C
:10C48000D29EF0011124EE0DF11DEF56F7464491B6
:10C490008F2D90E0ED81FE81E80FF91F408377201A
:10C4A00021F00D966FE070E004C0840D951D64E1ED
:10C4B00070E00E94955BF3943981F316B1F517C0D3
:10C4C00081FF11C0FF2079F0FA94772021F08F2DA1
:10C4D000835F6FE003C08F2D8C0D64E142E050E07C
:10C4E0000E94A65522C083FF20C0FF20F1F0ED81FD
:10C4F000FE81EF0DF11D108226960FB6F894DEBF77
:10C500000FBECDBFCF91DF911F910F91FF90EF90A4
:10C51000DF90CF90BF90AF909F908F907F906F9063
:10C520005F904F903F902F90089580912B0C9091A9
:10C530002C0C9093340C8093330C80912D0C9091A3
:10C540002E0C9093360C8093350C8E2D6DE00E944E
:10C550009B6EE92E8D2D63E00E949B6ED92EAA243E
:10C56000BB24C501880F991F079666E170E041E082
:10C5700050E023E030E002E010E00E943D5C0894CF
:10C58000A11CB11C8DE0A816B10459F78E2D880F9F
:10C590006D2D6A5E895F4FE650E00E94A6558FE0E0
:10C5A00090E060E170E0482D20E00E94B75BFFCE94
:10C5B0008F929F92AF92BF92CF92DF92EF92FF92B3
:10C5C0000F931F93DF93CF930F92CDB7DEB74C013C
:10C5D000162FE42EFF24EE0CFF1CF701ED5CF34F49
:10C5E000D701A55DB34F8D919C919183808384E0A9
:10C5F00062E04AE128E00E94765E80E263E040EA81
:10C6000053E70E94765C20E0DD2453E0C52E05E070
:10C610004FE7B42E8FE29CE0E80EF91E233050F471
:10C6200081E090E029830E947E5B29812F5F233087
:10C6300009F03BC04D2D50E0AD2CA394112331F0F7
:10C64000480D591DDA2CFA01449105C0480D591DB9
:10C65000FA014081DA2C442309F462C04A3019F40B
:10C66000C39405E008C0802F0F5F40526C2D2983D2
:10C670000E948E5529812330C1F4EA2DF0E0E1704B
:10C68000F070E157F746449181E264E050E00E9487
:10C69000A65560911201669561706B9D602D112405
:10C6A00082E041E00E94B85A20E080E029830E94A5
:10C6B000D455AC0190932C0C80932B0C8091330CAF
:10C6C0009091340C80959095842395239093300C11
:10C6D00080932F0C81E00E94D455AC0190932E0CD6
:10C6E00080932D0C8091350C9091360C809590950F
:10C6F000842395239093320C8093310CF701808131
:10C70000298180FD24E080912B0C90912C0C90933A
:10C71000340C8093330C5093360C4093350C7ECF01
:10C720000F90CF91DF911F910F91FF90EF90DF90CD
:10C73000CF90BF90AF909F908F900895DF92EF922F
:10C74000FF920F931F9380E090E060E070E048E27A
:10C7500050E02CE130E000E010E00E943D5C8BE313
:10C7600096E961E040E00E94D8628DE06EE04EE024
:10C7700024E00E94765E82E190E06FE070E042EAA1
:10C7800056E90E94995B80E190E060E170E04BEA3D
:10C7900056E90E94995B80912B0C90912C0C909300
:10C7A000340C8093330C80912D0C90912E0C90932F
:10C7B000360C8093350CFF24E8E0EE2E72E0D72E85
:10C7C00081E090E00E947E5B80E00E94D4559C0155
:10C7D00090932C0C80932B0C8091330C9091340C03
:10C7E00080959095822393239093300C80932F0C07
:10C7F00081E00E94D4559C0190932E0C80932D0CC7
:10C800008091350C9091360C8095909582239323DE
:10C810009093320C8093310C80912F0C87FF06C0CF
:10C82000FF2021F4809111018F5F07C086FF08C0AF
:10C83000FF2031F48091110181508093110111C0CA
:10C8400085FF02C0F3940DC084FF02C0FA9409C0B2
:10C8500080FF03C091E0F916D1F181FF02C080E0B2
:10C8600037C080912B0C90912C0C9093340C8093BA
:10C87000330C3093360C2093350C809111018930A4
:10C8800018F0D092110104C0823010F4E09211012E
:10C8900081E0F8228EE090E06FE070E041E050E04F
:10C8A00022E030E002E010E00E943D5C6F2D615F0D
:10C8B0008EE04FE650E00E94A6554091110150E0F5
:10C8C00040585F4F80E16FE00E94A65579CF81E02C
:10C8D0001F910F91FF90EF90DF900895EF92FF92DC
:10C8E0000F931F93CF93DF9380E090E060E070E0C0
:10C8F00048E250E02CE130E000E010E00E943D5CB6
:10C900008DE696E961E040E00E94D8622091110135
:10C910002D5F89E06EE046E10E94765E10E02BC05C
:10C92000AFE0EA2EF12CEC0EFD1EAE01F3E0440F59
:10C93000551FFA95E1F7485459468CE090E0B7014D
:10C940000E94995B84E190E0B70140EB56E90E94B8
:10C95000995B612F615F4091130150E002C05595D2
:10C960004795CA95E2F7417050704F575F4F8CE181
:10C970000E94A6551F5F80911101C12FD0E01817AA
:10C9800078F2BE01615F7F4F8CE090E04BEA56E9A0
:10C990000E94995B80912B0C90912C0C9093340CFD
:10C9A0008093330C80912D0C90912E0C9093360C2B
:10C9B0008093350CFF2481E090E00E947E5B80E054
:10C9C0000E94D45590932C0C80932B0C81E00E94F4
:10C9D000D455AC0190932E0C80932D0CE0912B0C30
:10C9E000F0912C0C8091330C9091340C80959095A3
:10C9F0008E239F239093300C80932F0C2091350C25
:10CA00003091360C20953095242335233093320C09
:10CA10002093310C20911101F21688F4382F307CCC
:10CA200071F061E070E00F2C02C0660F771F0A946E
:10CA3000E2F78091130186278093130110C0F2164C
:10CA400011F480FD49C084FF02C0F20E08C085FFCA
:10CA500002C0F39404C081FF02C080E03EC0F093A6
:10CA6000340CE093330C5093360C4093350C30E08B
:10CA70002F5F3F4F8F2D90E0B9010E94BB6EF82EC3
:10CA80008AE090E06FE070E041E050E002E010E00A
:10CA90000E943D5C6F2D615F8AE04FE650E00E948E
:10CAA000A65510E013C0612F615F4091130150E063
:10CAB000012E02C0559547950A94E2F741705070D7
:10CAC0004F575F4F8CE10E94A6551F5F8091110167
:10CAD000181708F070CFE7CF81E0DF91CF911F9159
:10CAE0000F91FF90EF900895CF92DF92EF92FF9217
:10CAF0000F931F93DF93CF93CDB7DEB76E970FB62B
:10CB0000F894DEBF0FBECDBFDC013C9120E0FE01FA
:10CB100031960DC0422F50E0DF01A40FB51F3C93AA
:10CB2000480F591FDA0111963C9111972F5F33235B
:10CB300089F780E030E07E010894E11CF11CA82F09
:10CB4000B0E0AD014C5C5846FA019491FD01EE0D48
:10CB5000FF1DE20FF31F90838F5F992381F7C09031
:10CB60001301DD2402C0D594C7946A95E2F7F1E081
:10CB7000CF2280E090E060E070E048E250E02CE1FD
:10CB800030E000E010E00E943D5CC70160E04C2D09
:10CB90000E94D86280E16EE048E024E00E94765E68
:10CBA00083E190E06FE070E048E457E90E94995B10
:10CBB00083E190E060E170E044E457E90E94995B12
:10CBC0008C2D0E94D4550097D9F7FF24DD24CC0C7E
:10CBD000DD1C8FE29CE0C80ED91E81E090E00E942F
:10CBE0007E5B80E00E94D4559C0190932C0C809336
:10CBF0002B0C8091330C9091340C8095909582236E
:10CC000093239093300C80932F0C81E00E94D45595
:10CC10009C0190932E0C80932D0C8091350C90915B
:10CC2000360C80959095822393239093320C8093B9
:10CC3000310CD6018D919C911197AC0140735070CD
:10CC40004115510511F0F39414C080FF12C08F2DCF
:10CC5000F11081E06E960FB6F894DEBF0FBECDBF27
:10CC6000CF91DF911F910F91FF90EF90DF90CF90C8
:10CC7000089580912B0C90912C0C9093340C809300
:10CC8000330C3093360C2093350CB1E0FB2281E15C
:10CC900090E06FE070E041E050E022E030E002E040
:10CCA00010E00E943D5C6F2D615F81E14FE650E036
:10CCB0000E94A65592CFAF92BF92DF92EF92FF9261
:10CCC0000F931F93DF93CF93CDB7DEB7C354D040FC
:10CCD0000FB6F894DEBF0FBECDBFD82E282F30E0A0
:10CCE000A90103E0440F551F0A95E1F7FA01E85442
:10CCF000F946949180E0BE016F5F7F4F4F5F5F4FB9
:10CD00000CC0E82FF0E0DB01AE0FBF1F9C93E40FD7
:10CD1000F51FE854F94694918F5F992391F7A82F56
:10CD2000B0E0BE016F5F7F4F092F10E0A8014850AF
:10CD30005946FA014491F801E60FF71FEA0FFB1F6D
:10CD400040839F5F442381F7790114E0EE0CFF1CC0
:10CD50001A95E1F7E21AF30A8CE19EE0E80EF91E5B
:10CD60005E010894A11CB11C80E090E060E070E0DE
:10CD700048E250E02CE130E000E010E00E943D5C31
:10CD80008D2D0E940F5E81E190E060E170E04BE448
:10CD900057E90E94995B4091130150E00D2C02C0AD
:10CDA000559547950A94E2F74170C50160E00E94ED
:10CDB000D862C7016D2D4EE021E00E943861C701A5
:10CDC0006D2D0E947465882379F2CD5BDF4F0FB61D
:10CDD000F894DEBF0FBECDBFCF91DF911F910F91B1
:10CDE000FF90EF90DF90BF90AF900895EF92FF9289
:10CDF0000F931F93CF93DF93182F062FEA01E12E95
:10CE0000F92EEE2DE11BCE018E0F911DFC0140810C
:10CE1000442349F08E2D0894E11CF11C4052602FF0
:10CE20000E948E55EECFDF91CF911F910F91FF9011
:10CE3000EF9008952F923F924F925F926F927F9260
:10CE40008F929F92AF92BF92CF92DF92EF92FF921A
:10CE50000F931F93DF93CF93CDB7DEB7AA970FB68B
:10CE6000F894DEBF0FBECDBF282E3324809113016E
:10CE700090E0022C02C0959587950A94E2F7282F3E
:10CE800021702AA780E090E060E070E048E250E086
:10CE90002CE030E000E010E00E943D5C80E090E09B
:10CEA0006CE070E048E250E020E130E001E610E0A4
:10CEB0000E943D5C7CE1672E7EE0772E6EE2462E7E
:10CEC0006DE0562EAA24BB245EE0952E43E0842E0E
:10CED0003CC0C82CDD24E92CFF24C601B7014FE07B
:10CEE00050E022E030E002E010E00E943D5CC6012C
:10CEF000B701A3010E94F6660894E11CF11CD2015F
:10CF00002D913D914D915C91C6010E96B7010E9405
:10CF1000F55BC6010596B70144E20E94955BB3E05C
:10CF2000AB16B10429F43EE0932E26E1822E02C016
:10CF3000E3E09E0E0894A11CB11C8FE090E0680E07
:10CF4000791EA4E0B0E04A0E5B1E8091110190E0D2
:10CF5000A816B90608F4BDCFF10194E0EE0FFF1F4B
:10CF60009A95E1F7E219F309E45EF14F908180E0D0
:10CF7000AE014F5F5F4F0DC0282F30E0DA01A20FE6
:10CF8000B31F9C932E0F3F1FD90111969C911197AF
:10CF90008F5F992389F7682F70E09E012F5F3F4FC5
:10CFA000A92FB0E0AD014D5A5846FA014491FD0158
:10CFB000E20FF31FE60FF71F40839F5F442381F7C3
:10CFC000C90160E04AA50E94D86280912B0C909123
:10CFD0002C0C9093340C8093330C80912D0C9091F9
:10CFE0002E0C9093360C8093350CFAA50F2F10E081
:10CFF000000F111F015D134F81E090E00E947E5BE6
:10D0000080E00E94D4559C0190932C0C80932B0CB3
:10D010008091330C9091340C8095909582239323CA
:10D020009093300C80932F0C81E00E94D4559C018A
:10D0300090932E0C80932D0C8091350C9091360C92
:10D0400080959095822393239093320C8093310C9A
:10D05000D8018C9183FD0DC080912B0C90912C0CEC
:10D060009093340C8093330C3093360C2093350C12
:10D07000C3CFAA960FB6F894DEBF0FBECDBFCF9137
:10D08000DF911F910F91FF90EF90DF90CF90BF90B5
:10D09000AF909F908F907F906F905F904F903F9058
:10D0A0002F9008953F924F925F926F927F928F924E
:10D0B0009F92AF92BF92CF92DF92EF92FF920F9327
:10D0C0001F93DF93CF93CDB7DEB7A4970FB6F89435
:10D0D000DEBF0FBECDBFD090130181E0D82280E02B
:10D0E00090E060E070E048E250E02CE030E000E0EA
:10D0F00010E00E943D5C80E090E06CE070E048E26F
:10D1000050E020E130E001E610E00E943D5C7CE16F
:10D11000672E7EE0772E6EE2462E6DE0562E882436
:10D1200099245EE0C52E43E0342E3CC0A32CBB24E2
:10D13000EC2CFF24C501B7014FE050E022E030E0C5
:10D1400002E010E00E943D5CC501B701A3010E940E
:10D15000F6660894E11CF11CD2012D913D914D9190
:10D160005C91C5010E96B7010E94F55BC50105965D
:10D17000B70144E20E94955BB3E08B16910429F459
:10D180003EE0C32E26E1322E02C0E3E0CE0E08942C
:10D19000811C911C8FE090E0680E791EA4E0B0E045
:10D1A0004A0E5B1E40911101842F90E0881699066B
:10D1B00008F4BCCFE2E3FDE031E020E031C0E080E4
:10D1C000F18002811381822F6AE00E949B6EA92F59
:10D1D000B0E0AA0FBB1FAA0FBB1FA25DB24F8D917B
:10D1E0009D910D90BC91A02D8E159F05A007B107B4
:10D1F00010F4232F13C0A22FB0E0AA0FBB1FAA0F59
:10D20000BB1FA25DB24F8D919D910D90BC91A02D41
:10D21000E816F9060A071B0709F4265F3F5F3496F4
:10D22000341768F22A3008F045C0EFE6F8E9949127
:10D2300080E0BE016F5F7F4F0BC0482F50E0FB01C5
:10D24000E40FF51F908340595746FA0194918F5F80
:10D25000992399F730E0F901A4E0EE0FFF1FAA959A
:10D26000E1F7E21BF30BE45EF14F508140E0682FE1
:10D2700070E0CE0101960CC0DC01A20FB31FA60F17
:10D28000B71F5C932E0F3F1FD90111965C91119728
:10D29000242F30E04F5F552379F7680F791F260F51
:10D2A000371F5EE2F9015083640F711DDB011C9290
:10D2B00060E003C083E898E961E04D2D0E94D862E8
:10D2C00080912B0C90912C0C9093340C8093330C08
:10D2D00080912D0C90912E0C9093360C8093350CF0
:10D2E0000D2D10E0000F111F015D134F81E090E044
:10D2F0000E947E5B80E00E94D4559C0190932C0C90
:10D3000080932B0C8091330C9091340C80959095E8
:10D31000822393239093300C80932F0C81E00E9402
:10D32000D4559C0190932E0C80932D0C8091350C3C
:10D330009091360C80959095822393239093320C94
:10D340008093310CF801808183FD0DC080912B0CFE
:10D3500090912C0C9093340C8093330C3093360CBA
:10D360002093350CC3CFA4960FB6F894DEBF0FBE42
:10D37000CDBFCF91DF911F910F91FF90EF90DF9084
:10D38000CF90BF90AF909F908F907F906F905F9065
:10D390004F903F9008957F928F929F92AF92BF924D
:10D3A000CF92DF92EF92FF920F931F93CF93DF9371
:10D3B000782E80E090E060E070E048E250E02CE100
:10D3C00030E001E610E00E943D5C0EE0E02E13E04C
:10D3D000D12EFF24B1E1CB2E5EC0CF2DD0E08091C5
:10D3E000A60C9091A70C9E0102C0969587952A9550
:10D3F000E2F780FF2BC08D2C9924AE2CBB24C401F6
:10D40000B5014FE050E022E030E002E010E00E9481
:10D410003D5CFC9CA00111244D5A524FC401B50142
:10D420000E94F666B5016F5F7F4FFE01A4E0EE0F2C
:10D43000FF1FAA95E1F7EC0FFD1FED5AF24FC40153
:10D440000E96408920E00E94B75B1AC08D2D90E0B7
:10D450006E2D70E04FE050E022E030E002E610E098
:10D460000E943D5CAE01F3E0440F551FFA95E1F7D1
:10D47000485459468D2D90E06E2D70E00E94995BC6
:10D4800033E0F31629F4EEE0EE2E76E1D72E02C05B
:10D4900083E0E80EF39480914E0DF81608F49DCFCA
:10D4A00080E190E06AE070E047E050E021E030E0A9
:10D4B00002E010E00E943D5C872D90E00197AC01F6
:10D4C00063E0440F551F6A95E1F7481B590B425919
:10D4D000584680E190E06AE070E00E94995BDD24AC
:10D4E000D3948EC0ED2CFF2430E02E193F0980919B
:10D4F000A60C9091A70C02C0969587952A95E2F705
:10D5000080FD7DC08EE190E00E947E5B6091120103
:10D5100066956170619584E041E00E94B85A8091FF
:10D520004E0D90E08E199F09843091051CF423E084
:10D5300030E002C026E130E064E070E00E94BB6EA3
:10D54000BC01660F771F680F791F625F7F4FC901AB
:10D550004FE050E022E030E002E010E00E943D5C4D
:10D5600020914E0D30E02E193F09243031051CF476
:10D57000E3E0F0E002C0E6E1F0E0C90164E070E061
:10D580000E94BB6EBC01660F771F680F791F625F38
:10D590007F4FA90184E0440F551F8A95E1F7420FA0
:10D5A000531F4D5A524FCF010E94F66620914E0DE7
:10D5B00030E02E193F09243031051CF4E1E1F0E0A0
:10D5C00002C0E4E2F0E0C90164E070E00E94BB6EDA
:10D5D000BC01660F771F680F791F615F7F4FD9010C
:10D5E00014E0AA0FBB1F1A95E1F7A20FB31FAD5AA3
:10D5F000B24FCF0150964C9120E00E94B75BD3947C
:10D6000020914E0D2D1508F06DCF88E790E00E9417
:10D610007E5BDF91CF911F910F91FF90EF90DF9094
:10D62000CF90BF90AF909F908F907F9008956F9212
:10D630007F928F929F92AF92BF92CF92DF92FF9292
:10D640000F931F93DF93CF930F92CDB7DEB7F82ED2
:10D6500080E090E060E070E048E250E02CE130E0F3
:10D6600000E010E00E943D5C8F2D0E940F5E4FE0B5
:10D67000F49EA0011124445E514F8DE090E06FE0D4
:10D6800070E00E94F66661E0662E712C0F2C02C0DD
:10D69000660C771C0A94E2F700E010E085E090E069
:10D6A0000E947E5B5FEFA52E5DE0B52ECC24DD24CD
:10D6B00098E0802E99249601217030702825392514
:10D6C000D501EC91F0E0E621F7210F2C02C0F59591
:10D6D000E7950A94E2F7EE0FFF1FE20FF31FEE0F3C
:10D6E000FF1FEF5FFE4F40815181892F6CE09983CE
:10D6F0000E94765C99819B5F0894C11CD11CE3E079
:10D70000F0E0AE0EBF1E9132B1F61F5F60911201C4
:10D7100066956170619583E041E00E94B85A1031CE
:10D7200019F081E00827BACF8EE190E00E947E5B7D
:10D730000F90CF91DF911F910F91FF90DF90CF90CD
:10D74000BF90AF909F908F907F906F9008956F9251
:10D750007F928F929F92AF92BF92CF92DF92EF9281
:10D76000FF920F931F93CF93DF93782E662E80E066
:10D7700090E060E070E048E250E02CE130E001E64B
:10D7800010E00E943D5C5EE0E52E43E0D42EFF24D5
:10D7900031E1C32E5EC0CF2DD0E08091A60C9091D8
:10D7A000A70C9E0102C0969587952A95E2F780FF07
:10D7B0002BC08D2C9924AE2CBB24C401B5014FE0A5
:10D7C00050E022E030E002E010E00E943D5CFC9C72
:10D7D000A00111244D5A524FC401B5010E94F666B2
:10D7E000B5016F5F7F4FFE0124E0EE0FFF1F2A950A
:10D7F000E1F7EC0FFD1FED5AF24FC4010E96408980
:10D8000020E00E94B75B1AC08D2D90E06E2D70E075
:10D810004FE050E022E030E002E610E00E943D5C84
:10D82000AE0193E0440F551F9A95E1F748545946CD
:10D830008D2D90E06E2D70E00E94995B33E0F31621
:10D8400029F48EE0E82E06E1D02E02C083E0E80E37
:10D85000F39480914E0DF81608F49DCF1DE0E12E53
:10D8600010E009C08E2D62E048E555E70E94765C25
:10D8700025E0E20E1F5F80914F0D181798F380E1AD
:10D8800090E06AE070E047E050E021E030E002E044
:10D8900010E00E943D5C872D90E00197AC01B3E061
:10D8A000440F551FBA95E1F7481B590B425958468A
:10D8B00080E190E06AE070E00E94995B0E94DF5D89
:10D8C000F82E8EE190E00E947E5B80914E0D60917B
:10D8D0001201F81608F088C066956170619584E0C1
:10D8E00041E00E94B85A33E03F1518F083E090E021
:10D8F00002C086E190E0CF2CDD24960123703070C9
:10D90000E901CC0FDD1FC20FD31FFEE0AF2EB12CFB
:10D91000AC0EBD1EB5014FE050E022E030E002E069
:10D9200010E00E943D5C83E08F1518F083E090E0EA
:10D9300002C086E190E041E1F49EA00111244D5A1D
:10D94000524FB5010E94F66623E02F1518F081E1D1
:10D9500090E002C084E290E0BE01615F7F4FE6018B
:10D96000E4E0CC0FDD1FEA95E1F7CC0DDD1DCD5ACB
:10D97000D24F488920E00E94B75B988984E69802DC
:10D98000C00111249C01442737FD4095542F8091FC
:10D99000A20C9091A30CA091A40CB091A50C820FA5
:10D9A000931FA41FB51F8093A20C9093A30CA09368
:10D9B000A40CB093A50C21E030E002C0220F331F6D
:10D9C000CA94E2F78091A60C9091A70C820F931F46
:10D9D0009093A70C8093A60C8AE590E00E947E5B52
:10D9E000862D0E94176B16C066956170619585E063
:10D9F00041E00E94B85A80914F0D8F5F80934F0D88
:10DA00008E2D62E048E555E70E94765C8AE590E05D
:10DA10000E947E5BDF91CF911F910F91FF90EF905D
:10DA2000DF90CF90BF90AF909F908F907F906F903E
:10DA30000895AF92BF92CF92DF92EF92FF920F9331
:10DA40001F93CF93DF93F82EE62E10924F0D109276
:10DA5000A70C1092A60C1092A20C1092A30C10927C
:10DA6000A40C1092A50C0E945E6F27E231E040E00A
:10DA700050E00E94F06EDC01CB01EEEFFCE020E014
:10DA800030E007C0419151914817590761F32F5F6A
:10DA90003F4F28173907B0F32091510D3091520DA7
:10DAA000F901EE0FFF1FE250F34F918380832F5F48
:10DAB0003F4F3093520D2093510D0E944D5D8FE0EA
:10DAC000F89EE0011124C45ED14FEAE0CE2ED12CA5
:10DAD0007FEFA72E73E0B72E2FC080E090E060E0CC
:10DAE00070E048E250E02CE130E000E010E00E94FD
:10DAF0003D5C8F2D0E940F5E8DE090E06FE070E046
:10DB0000AE010E94F66681E190E060E170E04BE4D6
:10DB100057E90E94995B88EA9CE060E040E00E943F
:10DB2000D8628CE09EE06F2D4FE020E00E943861CB
:10DB30008E2D6F2D0E94A76B80914F0D8330A8F41E
:10DB400080914E0D9601281B3109C901950102C033
:10DB5000359527958A95E2F7C9012091A60C309159
:10DB6000A70C2817390708F4B8CFCF2DD0E0CC0F79
:10DB7000DD1FCC0FDD1FC25DD24F6E2D70E080E047
:10DB800090E02091A20C3091A30C4091A40C5091F4
:10DB9000A50C0E947C6E288139814A815B81620FCD
:10DBA000731F841F951F688379838A839B838E2DBF
:10DBB0000E94CB69DF91CF911F910F91FF90EF9061
:10DBC000DF90CF90BF90AF9008950F931F93CF93A6
:10DBD000DF9384E79AE80E94C05584E795E70E94A6
:10DBE000C5558EE59DE00E94EE5680EB0E947B5766
:10DBF000ECE1FEE010823F968EE0E439F807D1F7C1
:10DC00000E94415682FD02C01092130182E798E003
:10DC10000E9409570E946C5F882331F0813009F41B
:10DC200065C08230B9F765C00E949E63882319F4ED
:10DC3000CDEFDDE005C00E946E648823A9F3F8CF24
:10DC400018810E945E6F20E031E040E050E00E94C9
:10DC5000F06E610F688319810E945E6F20E031E0F1
:10DC600040E050E00E94F06E610F69831A810E94CB
:10DC70005E6F20E031E040E050E00E94F06E610F06
:10DC80006A8323968EE0CC30D807D1F610E010C01E
:10DC9000812F0E945B66E12FF0E0EE0FFF1FEE0F79
:10DCA000FF1FE25DF24F10821182128213821F5F0A
:10DCB00080911101181760F31092520D1092510DBE
:10DCC00001E00FC0812F0E941A67812F602F0E94F0
:10DCD000196D1F5F809111011817A0F30F5F0430B9
:10DCE00011F010E0F7CF0E94526894CF0E9432608A
:10DCF00091CF0E94AC5E8ECF629FD001739FF001E6
:10DD0000829FE00DF11D649FE00DF11D929FF00DCB
:10DD1000839FF00D749FF00D659FF00D9927729F02
:10DD2000B00DE11DF91F639FB00DE11DF91FBD018D
:10DD3000CF0111240895991B79E004C0991F96170B
:10DD400008F0961B881F7A95C9F780950895AA1B3D
:10DD5000BB1B51E107C0AA1FBB1FA617B70710F0D6
:10DD6000A61BB70B881F991F5A95A9F78095909508
:10DD7000BC01CD01089597FB092E07260AD077FD37
:10DD800004D0E5DF06D000201AF4709561957F4F2E
:10DD90000895F6F7909581959F4F0895A1E21A2E68
:10DDA000AA1BBB1BFD010DC0AA1FBB1FEE1FFF1F3F
:10DDB000A217B307E407F50720F0A21BB30BE40B8F
:10DDC000F50B661F771F881F991F1A9469F76095D6
:10DDD0007095809590959B01AC01BD01CF01089590
:10DDE00097FB092E05260ED057FD04D0D7DF0AD0A9
:10DDF000001C38F450954095309521953F4F4F4F7A
:10DE00005F4F0895F6F790958095709561957F4FD7
:10DE10008F4F9F4F0895A0E0B0E0E1E1FFE60C9442
:10DE2000746FEC01E880F9800A811B81E114F10430
:10DE30000105110541F484E2E82E89EDF82E8BE509
:10DE4000082F87E0182FC801B7012DE133EF41E01B
:10DE500050E00E94F06E27EA31E440E050E00E947A
:10DE60007C6E5B016C01C801B7012DE133EF41E02D
:10DE700050E00E94F06ECA01B9012CEE34EF4FEF72
:10DE80005FEF0E947C6E9B01AC012A0D3B1D4C1D77
:10DE90005D1D57FF04C0215030404040504828834A
:10DEA00039834A835B835F77B901CA01CDB7DEB797
:10DEB000EAE00C94906F0E940B6F089584E191E06A
:10DEC0000E940B6F08956093140170931501809365
:10DED00016019093170108952F923F924F925F92EF
:10DEE0006F927F928F929F92AF92BF92CF92DF926A
:10DEF000EF92FF920F931F93CF93DF93CDB7DEB7CF
:10DF0000CA1BDB0B0FB6F894DEBF0FBECDBF099462
:10DF10002A88398848885F846E847D848C849B84B9
:10DF2000AA84B984C884DF80EE80FD800C811B81C7
:10DF3000AA81B981CE0FD11D0FB6F894DEBF0FBEF6
:0ADF4000CDBFED010895F894FFCF66
:10DF4A0004147428743C745074D8730074C473EC49
:08DF5A00730203AA010000009C
:00000001FF
